:100000000C94B40F0C94D50F0C94D50F0C94D50F01
:100010000C94D50F0C94D50F0C94D50F0C94D50FD0
:100020000C94D50F0C94D50F0C9411680C942E6879
:100030000C94D50F0C94D50F0C94EF680C941C699C
:100040000C9449690C9476690C94A3690C94D0695A
:100050000C94FD690C942A6A0C94576A0C94846A77
:100060000C94D50F0D94C7340D94FE340C94D50F19
:100070000C94D50F0C94D50F0C94D50F0C94D50F70
:100080000C94D50F0C94D50F0C94D50F0C94D50F60
:100090000C94D50F0C94D50F0C94D50F0D941560BE
:1000A0000D9447600D9479600D94AB600D946110D0
:1000B0000C94D50F0C94D50F0C94D50F0C94736C35
:1000C0000C94A06C0C94CD6C0C94FA6C0C94276D71
:1000D0000C94546D0C94816D0C94AE6D0C94DB6D8E
:1000E0000C94086E0C94D50F0D94EB330D942234C0
:1000F0000C94D50F0C94D50F0C94D50F0C94D50FF0
:100100000C94D50F0C94D50F0D943B150C94D50F72
:100110000C94D50F0C94D50F0C94D50F0D944D5F06
:100120000D947F5F0D94B15F0D94E35F0C94D50F38
:100130000C94D50F0C94B16A0C94DE6A0C940B6B82
:100140000C94386B0C94656B0C94926B0C94BF6B95
:100150000C94EC6B0C94196C0C94466C0C94D50FAD
:100160000D9459340D9490340C94D50F0C94D50FF4
:100170000C94D50F0C94D50F0C94D50F0C94D50F6F
:100180000C94D50F0C94D50F0C94D50F0C94D50F5F
:100190000C94D50F0C94D50F0C94D50F0C94D50F4F
:1001A0000D942E100C94D50F0C94D50F0C94D50FE4
:1001B0000C94356E0C94626E0C948F6E0C94BC6E25
:1001C0000C94E96E0C94166F0C94D50F0C94D50F0B
:1001D0000C94D50F0C94D50F0C94D50F0D94353588
:1001E0000D946C350C94D50F0C94D50F0C94D50F41
:1001F0000C94D50F0C94AE7A0C94697B8E1011116F
:10020000A0101111B2101111C410DE10C410F8109A
:10021000F810BF12D312E7120D133313AE139B1352
:10022000AE137513751376187618AE18EB182F19D0
:100230006C18181A341A711ACF19CF19341A181ADF
:100240002F19EB18AE187618761835223F2249225E
:1002500053225D226722712276227B22852285220B
:10026000762271225D22532249223F2235224D27D8
:100270004D275427542767278A274D278A27542735
:1002800054274D278A27542754274D274D27C32706
:10029000C327CB27CB27E0270728C3270728CB274F
:1002A000CB27C3270728CB27CB27C327C32717284C
:1002B000B8284028B828B8289128B828692869287B
:1002C0009128B8284028B8281728EB28F6280529AF
:1002D0002029362958299E29A729C2297E297E2925
:1002E000A7299E29362920290529F628EB282561EA
:1002F0009C619C61B5609C619C619C619C619C61FE
:100300009C619C619C619C619C619C619C619C6105
:100310009C61CA609C619C619C619C619C619C61C8
:100320009C611F617D619C619C618A619C619C6193
:100330009C619C619C619C6138619C619C6196613F
:100340009C6199619C619C619C619C6193619C61D1
:100350009C619C619C619C619C619C619C619C61B5
:100360009C619C619C619C619C619C619C619C61A5
:100370009C619C619C619C619C619C619C619C6195
:100380009C619C619C619C619C619C619C619C6185
:100390009C619C619C619C619C619C619C619C6175
:1003A0009C6122618275857588758B758E759175D6
:1003B0009475017D147D277D3A7D4D7D607D737D33
:1003C0007B827B82F8813D823D82B081B0813D821B
:1003D0003D823D823D823D823D823D823D823D8225
:1003E0003D823D823D823D823D823D82B0813D82A3
:1003F0003D823D823D823D8287872E89C387F48777
:100400002E892E892E892E892E892E892E892E8934
:100410002E892E892E892E892E892E892E892E8924
:100420002E892E892E892E892E892E892E892E8914
:100430002E892E892E892E892E892E892E892E8904
:100440002E892E892E892E892E892E892E892E89F4
:100450002E892E892E892E892E89C1882E892F8852
:100460002E892E89F0882E892E892E892E892E8913
:100470002E892E892E892E8972882E893E882E8972
:100480004C882E89A088DF920F9148919291F89123
:10049000439258928A92AC92CD9292941F93279352
:1004A000449383939693E093029419942E948D949D
:1004B0008D948D948D948D948D948D948D948D9434
:1004C0008D9445944D9458946D94739463BD94BDEC
:1004D0003FBD4BBD94BD94BD94BD94BD94BD94BD32
:1004E00094BD94BD94BD94BD94BD94BD94BD94BD84
:1004F00057BD94BD94BD94BD94BD94BD94BD94BDB1
:1005000094BD94BD94BD94BD94BD94BD63BD94BD94
:100510003FBD4BBD94BD94BD94BD94BD94BD94BDF1
:1005200094BD94BD94BD94BD94BD94BD94BD94BD43
:1005300057BDFCC8FFC850C950C950C950C950C99F
:1005400050C950C950C950C950C950C950C950C9E3
:1005500050C950C950C950C950C950C936C950C9ED
:1005600050C950C950C950C950C91CC950C950C9F7
:1005700050C950C950C902C950C950C950C950C901
:1005800050C950C950C950C950C950C950C950C9A3
:1005900050C950C950C950C950C950C936C950C9AD
:1005A00050C950C950C950C950C91CC950C950C9B7
:1005B00050C950C950C902C9F9CBF6CB0BCC0BCCF2
:1005C0000BCC0BCC0BCC0BCC0BCC0BCC0BCC0BCC73
:1005D0000BCC0BCC0BCC0BCC0BCC42CB15CB33CBFD
:1005E0000BCC0BCCB9CBFCCA0BCC0BCC0BCC0BCCB7
:1005F0000BCC24CBFCCB0BCC0BCC4CCB0BCC0BCCFB
:100600000BCC0BCC0BCC0BCC0BCC0BCC0BCC0BCC32
:100610000BCC0BCC0BCC0BCC0BCC42CB15CB33CBBC
:100620000BCC0BCCB9CBFCCA0BCC0BCC0BCC0BCC76
:100630000BCC24CBFCCB0BCC0BCC4CCB04CF47CF7F
:1006400056CF56CF56CF56CF56CF56CF56CF56CF82
:1006500056CF56CF56CF56CF56CF31CE56CFE8CE07
:10066000E2CE4ACEFECE56CF56CF5ACE31CE56CF60
:10067000F8CE13CF3ECEF2CE4CCFEECE50CE09CF39
:10068000DCCE55CE56CF0ECF2DCE51CF56CF56CF36
:1006900044CE56CF56CF56CF56CF56CF56CFE8CEB4
:1006A000E2CE4ACEFECE56CF56CF5ACE31CE56CF20
:1006B000F8CE13CF3ECEF2CE4CCFEECE50CE09CFF9
:1006C000DCCE55CE56CF0ECF2DCE51CF56CF56CFF6
:1006D00044CE0DCE76D466D468D46AD46CD46ED4AD
:1006E00070D472D493D483D485D487D489D48BD452
:1006F0008DD48FD4A0D4CED4A8D4CED4A8D4CED4E4
:10070000A8D4CED4A8D4CED4A8D4CED4CED4CED44B
:10071000CED4CED4CED4CED4AFD4B6D4C2D4C2D418
:10072000FEE72DE639E684E6B5E799E6DBE6FFE687
:1007300028E783E7AAEFAAEF34F06CF14CF274F3E8
:100740005EF44CF55EF498F698F64CF55EF44CF2D7
:100750006CF134F0AAEFAAEFCEF8CEF80FF96DF9EC
:10076000ACF9FAF92FFA6EFA2FFABCFABCFA6EFA63
:100770002FFAACF96DF90FF9CEF8CEF819FD84FD1A
:10078000EFFDA8FE54FFD003DA03E003DA03D80339
:10079000D803E003DA0354FFA8FEEFFD84FD19FD42
:1007A0000D9444000D9404200D94C6200D9439211D
:1007B0000D94E5020D942D010D941F220D94B92185
:1007C0000D94E4010D94A1214E414E494E495459D6
:1007D000494E46CDCCCC3D0AD7233C17B7D138770C
:1007E000CC2B329595E6241FB14F0A000020410022
:1007F00000C84200401C4620BCBE4CCA1B0E5AAE6C
:10080000C59D74444D2E4D00444D53004444003268
:1008100035304D4F686D0032354D4F686D003630C4
:10082000487A003530487A004E6F6E2D496E74005C
:1008300048692D4C4F004750530054696D65004482
:10084000697374616E6365005075736820427574D6
:10085000746F6E00496D70657269616C004D6574EE
:1008600072696300494E4300444543004F4E004FB8
:100870004646007B0976096C096509590952094603
:10088000093509270914090109EC08DB08C808BA69
:1008900008AB08A1089708434950532641435647DF
:1008A0000044435647264143564700434950532688
:1008B00044435647264143564700327844435647FF
:1008C00026327841435647004349505326327844F4
:1008D00043564726327841435647003278496D7077
:1008E0002E20434950532641435647003278496DE4
:1008F000702E43495053264443564726414356479A
:1009000000327843495053263278444356472641B3
:10091000435647003278496D702E20434950532684
:1009200032784443564700506172616C6C656C20AC
:1009300043495053003278496D702E20434950533B
:100940002644435647003278496D702E2043495063
:100950005300347844435647004349505326327875
:100960004443564700327844435647004349505366
:1009700026444356470044435647004349505300DA
:100980004B128911C7100510430F810EBF0DFD0CCE
:100990003B0C790B180BFD0CBF0D430F0510C71056
:1009A00089114B12AC12EA1128116610A40FE20E45
:1009B000200E5E0D9C0CDA0B180B5E0D200EA40FA2
:1009C00066102811EA11AC1253616D706C652F73BB
:1009D00065633A004552524F5220202020202000CB
:1009E000432D434950532C20522D434950532C2022
:1009F00000000000000000000000000000000000F7
:100A000000000000000000000000000000000000E6
:100A100000000000000000000000000000000000D6
:100A200000000000000000000000000000000000C6
:100A300000000000000000000000000000000000B6
:100A4000004C6F2D434950532C2048692D43495089
:100A5000532C2000000000000000000000000000F7
:100A60000000000000000000000000000000000086
:100A70000000000000000000000000000000000076
:100A80000000000000000000000000000000000066
:100A90000000000000000000000000000000000056
:100AA0000000434950532C200000000000000000CB
:100AB0000000000000000000000000000000000036
:100AC0000000000000000000000000000000000026
:100AD0000000000000000000000000000000000016
:100AE0000000000000000000000000000000000006
:100AF00000000000000000000000000000000000F6
:100B00000000004143564752506F6C2C2041435621
:100B10004752526D732C2000414356474C506F6C26
:100B20002C20414356474C526D732C20414356476D
:100B300052506F6C2C204143564752526D732C20FB
:100B400000000000000000000000000000000000A5
:100B50000000000000000000000000000000000095
:100B60000000000000000000000000000000000085
:100B7000000000000000000000522D4443564720B2
:100B80004F6E2C204C2D44435647204F6E2C204C4A
:100B90006F2D43495053204F6E2C2048692D4349F7
:100BA0005053204F6E2C20522D44435647204F6601
:100BB000662C204C2D44435647204F66662C204C13
:100BC0006F2D43495053204F66662C2048692D43B2
:100BD000495053204F66662C2000522D44435647FF
:100BE000204F66662C204C2D44435647204F6666A6
:100BF0002C204C6F2D43495053204F66662C2048C3
:100C0000692D43495053204F66662C20522D444392
:100C10005647204F6E2C204C2D44435647204F6E94
:100C20002C204C6F2D43495053204F6E2C20486987
:100C30002D43495053204F6E2C2000432D434950E3
:100C400053204F6E2C20522D43495053204F6E2C71
:100C500020432D43495053204F66662C20522D438C
:100C6000495053204F66662C200000000000000011
:100C70000000000000000000000000000000000074
:100C80000000000000000000000000000000000064
:100C9000000000000000000000000000432D434958
:100CA0005053204F66662C20522D43495053204FFD
:100CB00066662C20432D43495053204F6E2C205202
:100CC0002D43495053204F6E2C200000000000009F
:100CD0000000000000000000000000000000000014
:100CE0000000000000000000000000000000000004
:100CF00000000000000000000000000000522D4431
:100D0000435647204F6E2C204C6F2D4349505320A3
:100D10004F6E2C2048692D43495053204F6E2C2094
:100D2000522D44435647204F66662C204C6F2D436E
:100D3000495053204F66662C2048692D4349505333
:100D4000204F66662C20000000000000000000001C
:100D50000000000000000000000000000000522D14
:100D600044435647204F66662C204C6F2D43495014
:100D700053204F66662C2048692D43495053204F1D
:100D800066662C20522D44435647204F6E2C204C33
:100D90006F2D43495053204F6E2C2048692D4349F5
:100DA0005053204F6E2C2000000000000000000077
:100DB0000000000000000000000000000000004CE7
:100DC0006F2D43495053204F6E2C2048692D4349C5
:100DD0005053204F6E2C204C6F2D43495053204FC1
:100DE00066662C2048692D43495053204F66662C77
:100DF00020000000000000000000000000000000D3
:100E000000000000000000000000000000000000E2
:100E100000000000000000000000000000000000D2
:100E20004C6F2D43495053204F66662C2048692D46
:100E300043495053204F66662C204C6F2D43495038
:100E400053204F6E2C2048692D43495053204F6E3C
:100E50002C20000000000000000000000000000046
:100E60000000000000000000000000000000000082
:100E70000000000000000000000000000000000072
:100E800000522D44435647204F6E2C204C2D444396
:100E90005647204F6E2C20462D44435647204F6E18
:100EA0002C20422D44435647204F6E2C20522D4477
:100EB000435647204F66662C204C2D44435647200E
:100EC0004F66662C20462D44435647204F66662CBD
:100ED00020422D44435647204F66662C20000000D8
:100EE0000000522D44435647204F66662C204C2D5F
:100EF00044435647204F66662C20462D44435647B0
:100F0000204F66662C20422D44435647204F66668C
:100F10002C20522D44435647204F6E2C204C2D44FC
:100F2000435647204F6E2C20462D44435647204FB2
:100F30006E2C20422D44435647204F6E2C2000003B
:100F4000000000522D44435647204F6E2C204C2D5C
:100F500044435647204F6E2C2043495053204F6E38
:100F60002C20522D44435647204F66662C204C2D92
:100F700044435647204F66662C2043495053204F28
:100F800066662C2000000000000000000000000049
:100F90000000000000000000000000000000000051
:100FA00000000000522D44435647204F66662C2017
:100FB0004C2D44435647204F66662C2043495053DE
:100FC000204F66662C20522D44435647204F6E2CEE
:100FD000204C2D44435647204F6E2C2043495053FC
:100FE000204F6E2C200000000000000000000000D8
:100FF00000000000000000000000000000000000F1
:101000000000000000522D44435647204F6E2C2014
:101010004C2D44435647204F6E2C20522D444356AE
:1010200047204F66662C204C2D44435647204F6680
:10103000662C2000000000000000000000000000FE
:1010400000000000000000000000000000000000A0
:101050000000000000000000000000000000000090
:10106000000000000000522D44435647204F6666A2
:101070002C204C2D44435647204F66662C20522D81
:1010800044435647204F6E2C204C2D444356472056
:101090004F6E2C2000000000000000000000000047
:1010A0000000000000000000000000000000000040
:1010B0000000000000000000000000000000000030
:1010C00000000000000000522D44435647204F6EA0
:1010D0002C2043495053204F6E2C20522D44435610
:1010E00047204F66662C2043495053204F66662C9C
:1010F00020000000000000000000000000000000D0
:1011000000000000000000000000000000000000DF
:1011100000000000000000000000000000000000CF
:101120000000000000000000522D44435647204FAD
:1011300066662C2043495053204F66662C20522D62
:1011400044435647204F6E2C2043495053204F6E46
:101150002C20000000000000000000000000000043
:10116000000000000000000000000000000000007F
:10117000000000000000000000000000000000006F
:10118000000000000000000000522D44435647209C
:101190004F6E2C20522D44435647204F66662C201C
:1011A000000000000000000000000000000000003F
:1011B000000000000000000000000000000000002F
:1011C000000000000000000000000000000000001F
:1011D000000000000000000000000000000000000F
:1011E00000000000000000000000522D444356475C
:1011F000204F66662C20522D44435647204F6E2CBC
:1012000020000000000000000000000000000000BE
:1012100000000000000000000000000000000000CE
:1012200000000000000000000000000000000000BE
:1012300000000000000000000000000000000000AE
:10124000000000000000000000000043495053204F
:101250004F6E2C2043495053204F66662C200000CF
:10126000000000000000000000000000000000007E
:10127000000000000000000000000000000000006E
:10128000000000000000000000000000000000005E
:10129000000000000000000000000000000000004E
:1012A000000000000000000000000000434950530F
:1012B000204F66662C2043495053204F6E2C20004F
:1012C000000000000000000000000000000000001E
:1012D000000000000000000000000000000000000E
:1012E00000000000000000000000000000000000FE
:1012F00000000000000000000000000000000000EE
:101300000000000000000000000000000044656CC8
:1013100061792054696D653B0046696C65204E61BA
:101320006D653A2000436861696E6167652C200035
:10133000004C6F63616C54696D652C204C6F636168
:101340006C444D592C204C61742D4465672C204C05
:1013500061742D4D696E2C204E532C204C6F6E2DD8
:101360004465672C204C6F6E2D4D696E2C204557BF
:101370002C20466978537461742C204E756D53612E
:10138000742C2050444F502C20416C745F4D2C2005
:1013900043686B2C20436F6D6D000000000000005F
:1013A00000000000000000000000000000004C6F82
:1013B00063616C54696D652C204C6F63616C444DA6
:1013C000592C204C61742D4465672C204E532C20E1
:1013D0004C6F6E2D4465672C2045572C204669784C
:1013E000537461742C204E756D5361742C205044DD
:1013F0004F502C20416C745F4D2C2043686B2C2087
:10140000436F6D6D00000000000000000000000050
:1014100000000000000000000000000000000000CC
:1014200000000000000000000000004C6F63616CD1
:1014300054696D652C204C6F63616C444D592C20B0
:101440004C61742D4465672C204C61742D4D696E80
:101450002C204C61742D5365632C204E532C204C52
:101460006F6E2D4465672C204C6F6E2D4D696E2C70
:10147000204C6F6E2D5365632C2045572C204669F8
:1014800078537461742C204E756D5361742C205008
:10149000444F502C20416C745F4D2C2043686B2CC2
:1014A00020436F6D6D000000484558434F5244453E
:1014B000522043414C4942482E5458540000007772
:1014C00077772E636174682D746563682E636F6D22
:1014D0000000000000004C494D495445442039307B
:1014E000352D3835372D313035300000004341542B
:1014F000484F44494320544543484E4F4C4F475969
:101500000000007B702C30302C662C007B702C305F
:10151000302C657D007B702C30302C6F7D00686333
:1015200069746F6F6C20706169722000456E74651C
:10153000722050494E203A2000686369636F6E66DE
:101540006967206E616D65200061742B6274642A86
:10155000007175697400736D6172745A0061742B47
:1015600072756E00456E746572204143564720289F
:1015700027462720666F722046726F6E742C2027D4
:10158000422720666F72204261636B290A0D206139
:101590006E6420737570706C79203332302B363462
:1015A000302073696E65776176652077697468208D
:1015B0005065616B546F5065616B20766F6C746120
:1015C0006765206F6620302E385600456E74657250
:1015D0002053434F504520766F6C746167652069D6
:1015E0006E206D5620284E4E4E4E4E2900456E748C
:1015F0006572204349505320766F6C746167652093
:10160000696E206D562A313020284E4E4E4E4E299E
:1016100000456E746572204443564720766F6C74A3
:1016200061676520696E206D562A313020284E4E44
:101630004E4E4E29004469736320434F55504F4E20
:10164000204F4E203D20004469736320434F555086
:101650004F4E204F4646203D2000494E5354414EA8
:1016600054204F4E203D2000494E5354414E5420AB
:101670004F4646203D2000AD16A616A2169E169A8D
:1016800016961687168716432D53474E44205B3512
:101690002D3430565D00432D4200432D4600432D2E
:1016A0005200432D4C00522D53474E4400432D53BE
:1016B000474E440020616E6420656E74657220762A
:1016C0006F6C7461676520696E206D562A31302019
:1016D000284E4E4E4E4E2900506C65617365206356
:1016E0006F6E6E65637420004572726F722C206D90
:1016F000697373696E6720414443206E756D2028BD
:10170000302D3729000A0D5363616C696E674361A0
:101710006C6962204F66667365743A200045727288
:101720006F722C20656E74657220766F6C746167C1
:101730006520696E206D562A313020284E4E4E4E5F
:101740004E2900F117D217BC17B0178C1779175113
:101750001743535B302F312F322F332F345D5B769D
:10176000767676765D202D204443205363616C6944
:101770006E672043616C6962004342202D20426104
:1017800074746572792043616C696200435A5B30FE
:101790002F312F322F332F345D202D204443205AF8
:1017A00065726F4F66667365742043616C69620091
:1017B00056202D20566E756D626572004C5B696E09
:1017C000785D5B4F4E2F4F46465D202D204C656463
:1017D0007300416E6E202D205265616420414443A8
:1017E0003120666F72206E6E207365636F6E647356
:1017F0000041202D20526561642041444331004561
:1018000052524F52004F4B004341544820544543DD
:101810004820484558434F52444552205630312EB7
:101820003231000100020003000400050006000A36
:10183000000C000F0014001E003C007800B400F003
:10184000002C01680100000000120002000100B835
:101850000B0F27010064006801100E010010271013
:101860002710271027102710270100010001000171
:1018700000F8010200010002000100F40100000074
:10188000000100000000000A00F1D8000001000182
:1018900000C8000000640064006400640064006428
:1018A00000000000000000000050FE0000000000EA
:1018B0000000000100000000000100000000000A1C
:1018C00000000001000100020058020000FA00FAC6
:1018D00000FA00FA00780078000000000000000123
:1018E00000000001000100000000000100010000F4
:1018F0008000190080001900800019008000190084
:101900008000190080001900800019008000190073
:10191000000100FF03E600E6004F19411933192CBE
:1019200019244A42494E2C39342C3100244A53415F
:10193000564500244A4153432C47504753412C31CC
:1019400000244A4153432C4750524D432C3100242C
:101950004A4153432C47504747412C310024504DB6
:10196000544B3636372A33350024504D544B3331DF
:10197000342C302C312C302C312C312C302C302C80
:10198000302C302C302C302C302C302C302C302C77
:10199000302C302C302C302A323900756E6C6F6749
:1019A000206C62616E64747261636B7374617461E4
:1019B000006C6F67206C62616E64747261636B733C
:1019C00074617461206F6E74696D652031300075CB
:1019D0006E6C6F6720707372706F7361006C6F67ED
:1019E00020707372706F7361206F6E74696D652003
:1019F000313000646174756D20757365720020303C
:101A00002E3020302E3020302E3020302E300075F9
:101A1000736572646174756D2000646174756D2006
:101A2000776773383400756E6C6F67206770616C10
:101A30006D006C6F67206770616C6D206F6E7469EC
:101A40006D6520313000AF1AA01A911A821A7A1AE5
:101A5000611A541A245047524D432C2C2C39362CE1
:101A600000245047524D432C412C2C3130302C2C2B
:101A70002C2C2C2C2C2C2C2C2C00245047524D433D
:101A80004500245047524D4F2C5047524D542C3056
:101A900000245047524D4F2C5047524D462C310098
:101AA000245047524D4F2C47504753562C3000245A
:101AB0005047524D4F2C2C3400101B011BF21AE3DF
:101AC0001AD41AC51A445A203D2000000000000014
:101AD000000000004459203D2000000000000000EC
:101AE0000000004458203D200000000000000000DD
:101AF0000000466C6174203D2000000000000000E2
:101B0000004D616A6F7241203D200000000000001E
:101B10005354505220444154554D2E545854005C57
:101B20001C4F1C421C351C281C1B1C0E1C011CF4C9
:101B30001BE71BDA1BCD1BC01BB31BA61B991B8C01
:101B40001B7F1B721B651B581B4B1B4143564732A7
:101B500020524D53203D2000414356473120524DE5
:101B600053203D200042415454202043616C203DCD
:101B7000200041432020205343616C203D20004140
:101B8000432020205A43616C203D200041444337CC
:101B9000205653636C203D200041444337205A4374
:101BA000616C203D200041444336205653636C2035
:101BB0003D200041444336205A43616C203D2000C3
:101BC00041444335205653636C203D20004144433B
:101BD00035205A43616C203D200041444334205657
:101BE00053636C203D200041444334205A43616CD0
:101BF000203D200041444333205653636C203D2058
:101C00000041444333205A43616C203D200041444D
:101C10004332205653636C203D2000414443322020
:101C20005A43616C203D20004144433120565363A8
:101C30006C203D200041444331205A43616C203DDB
:101C4000200041444330205653636C203D20004126
:101C5000444330205A43616C203D200046696C6546
:101C600020496E646578203D20000A1FF41EDE1EA8
:101C7000C81EB21E9C1E861E701E5A1E441E2E1E9C
:101C8000181E021EEC1DD61DC01DAA1D941D7E1D12
:101C9000681D521D3C1D261D101DFA1CE41CCE1C87
:101CA000B81C454E44000000000000000000000089
:101CB00000000000000000004443564720446566D1
:101CC0006563742056616C203D2000000000444391
:101CD00056472044656665637420456E203D2000AC
:101CE0000000000053796E632054797065203D2018
:101CF0000000000000000000000043495053205243
:101D0000616E6765202B2F2D3556203D2000000089
:101D100047505320436F6F726420666F726D617419
:101D2000203D200000004C6F63616C4750535469A4
:101D30006D654F6666736574203D20004143204603
:101D400072657175656E6379203D200000000000AA
:101D5000000042726F6B656E5769726520416C615D
:101D6000726D203D200000004C6F7720506F742072
:101D7000416C61726D203D20000000000000496E42
:101D800070757420496D706564616E6365203D20D7
:101D900000000000444356474D44656C4F4E203DC3
:101DA00020000000000000000000444356474D445E
:101DB000656C4F4646203D200000000000000000FA
:101DC00043495053324D44656C4F4E203D20000036
:101DD00000000000000043495053324D44656C4FF1
:101DE0004646203D200000000000000043495053BB
:101DF000314D44656C4F4E203D2000000000000036
:101E0000000043495053314D44656C4F4646203DD8
:101E10002000000000000000537461727457697460
:101E200068203D20000000000000000000004F6618
:101E30006654696D65205B6D7365635D203D2000B0
:101E400000000000546F74616C4379636C65205B23
:101E50007365635D203D2000000054696D65205668
:101E6000616C7565203D200000000000000000004E
:101E7000436861696E61676520446972656374696E
:101E80006F6E203D20005374617274204368616955
:101E90006E616765203D2000000000004469737496
:101EA000616E63652056616C7565203D2000000001
:101EB00000004D6561737572656D656E7420556EB9
:101EC000697473203D20000053746F726167652050
:101ED000416374696F6E203D20000000000053755F
:101EE000727665792054797065203D2000000000ED
:101EF000000000004F70657261746F72204E616D5A
:101F000065203D2000000000000053757276657961
:101F1000204E616D65203D200000000000000000A3
:101F200054532D5453204F4E203D200054532D54D4
:101F300053204F4646203D20004E45572054532005
:101F40004F4E203D20004E4557205453204F4646CB
:101F5000203D20005453204F4E203D20005453205C
:101F60004F4646203D20000011241FBECFEFCDBFBD
:101F7000DFE5DEBF00E00CBF1FE2A0E0B0E2EEE86C
:101F8000F3ED02E00BBF02C007900D92AA3FB1072C
:101F9000D9F724E5AAEFBFE201C01D92A63BB20724
:101FA000E1F70E940F3F0D94C5690C940000CF9398
:101FB000DF93CDB7DEB72B97CDBFDEBFBE016F5F1E
:101FC0007F4F80E092E00F942D61AE01485F5F4F3C
:101FD00068E080E092E00F9489618A819B819F781C
:101FE0009B8395E09D83817E8A831C82BE016F5F07
:101FF0007F4F80E092E00F94DD6081E0888788E188
:102000008987AE01485F5F4F68E080E092E00F94FF
:10201000506180E092E00F943E5F2B96CDBFDEBF13
:10202000DF91CF9108959FB7F894E0E0F2E08081CE
:10203000806280839FBF0895009781F020910602FF
:1020400023FF0EC020913C0230913D02FC01208311
:10205000318388E08093060281E0089580E008954E
:1020600080E00895CF92DF92EF92FF92CF93DF93BB
:102070000097D1F061157105C9F0EB01FC01A08159
:10208000B18128EE33E00F94DD646B017C0183E1C4
:102090000E9441D09B01AC01C701B6010F94886436
:1020A0002883398381E003C080E001C080E0DF91B4
:1020B000CF91FF90EF90DF90CF900895EDE1F9E39D
:1020C0001082118214821582128213821682178264
:1020D0008BE00E9465D0672B682B692B19F4109256
:1020E000253903C081E080932539EDE1F9E31186BC
:1020F00012860895CF93DF93EC01892B09F491C0E8
:10210000862F90E0FC013197EB30F10508F089C093
:102110008827E250FF4F8F4F0D94C6648091253978
:10212000811107C088819981809321399093223948
:1021300078C08A819B81809321399093223971C024
:1021400080912539811107C08A819B818093213933
:102150009093223966C08E819F818093213990931C
:1021600022395FC080912539811107C08C819D8102
:10217000809321399093223954C08A859B8580931E
:102180002139909322394DC08091253981110BC09E
:1021900088819981EDE1F9E3848395838A819B812C
:1021A000868397833EC08C819D81EDE1F9E3848332
:1021B00095838E819F818683978333C08091253953
:1021C00081110BC08A819B81EDE1F9E384839583C2
:1021D0008C819D818683978324C0EDE1F9E3888516
:1021E0009985848395838A859B858683978319C087
:1021F0008091253981110BC08C819D81EDE1F9E33E
:10220000848395838E819F81868397830AC0EDE1C5
:10221000F9E38C859D85848395838E859F85868350
:102220009783DF91CF910895EDE1F9E38481958162
:102230008083918386819781828393830895EDE1E2
:10224000F9E381E0818712860895EDE1F9E31186D3
:102250001286089580912739089583E10E9465D000
:10226000672B682B692B19F080912639089580E03F
:102270000895CF92DF92EF92FF926B01072E000C30
:10228000EE08FF08C216D306E406F5067CF48617AE
:102290009707E4F0092E000CAA0BBB0BE1E028170E
:1022A00039074A075B07ACF4E0E013C06C01092E64
:1022B000000CEE08FF08C216D306E406F50644F04B
:1022C000E1E0681779072CF4E0E003C0E0E001C02A
:1022D000E0E08E2FFF90EF90DF90CF900895FF9277
:1022E0000F931F93CF93DF93CDE1D9E301E219E37D
:1022F000F12CE991F991309719F1AF010F2E000CF3
:10230000660B770BDB01CA0177231CF40196A11D34
:10231000B11DB595A795979587959A01AB01280FA3
:10232000391F4A1F5B1FBF01FF2314F46F5F7F4FEC
:10233000759567958A819B819CDF813009F0F394C4
:10234000C017D107B1F6FF2011F079DF01C07DDFA2
:102350006BDFDF91CF911F910F91FF900895EDE119
:10236000F9E381E090E0A0E0B0E08787908BA18B5B
:10237000B28B838B948BA58BB68B178A13861486AE
:1023800015861686108E0895EDE1F9E381E0878BBE
:10239000108E0895EDE1F9E3178A108E089580916B
:1023A0003539089584E10E9465D0672B682B692B2D
:1023B00019F080913439089580E00895EDE1F9E352
:1023C00087859089A189B289838B948BA58BB68BE5
:1023D00083859485A585B6858787908BA18BB28BE5
:1023E0000895609328397093293980932A399093FE
:1023F0002B3908958F929F92AF92BF92CF92DF9226
:10240000EF92FF92EDE1F9E3C388D488E588F6887E
:1024100087859089A189B289C816D906EA06FB0684
:1024200091F48090283990902939A0902A39B09061
:102430002B39C4DFC814D904EA04FB0411F4A4DF67
:1024400004C0A8DF02C0BADFFCCFFF90EF90DF909E
:10245000CF90BF90AF909F908F9008958BE10E9496
:1024600065D06093363970933739809338399093BB
:102470003939AAE3B9E3EDE1F9E385E299E31D9285
:1024800011A212A232968E179F07C9F7EDE1F9E368
:1024900011A612A6089581E090914639911101C0CC
:1024A00080E008958AE10E9465D0672B682B692B34
:1024B00039F081E090914639911103C080E0089590
:1024C00080E008950F931F938B019C018091363912
:1024D00090913739A0913839B09139390097A105D9
:1024E000B10529F1880F991FAA1FBB1FAC01BD01BF
:1024F000440F551F661F771F440F551F661F771F18
:10250000840F951FA61FB71FB901A80133233CF400
:1025100044275527BA01401B510B620B730B21E076
:1025200084179507A607B7071CF020E001C020E03C
:10253000822F1F910F9108950F931F93CF93DF93D5
:10254000009709F40BC1ADE1B9E35D961C925D976C
:102550005E961C925E975F961C925F9790961C9277
:10256000462F50E0FA013297EA30F10508F0F6C044
:10257000EC018827E75FFE4F8F4F0D94C664809172
:102580002539811108C06C817D818E819F819ADF00
:1025900080933A39E3C0688179818A819B8192DF97
:1025A00080933A39DBC080912539811108C0688554
:1025B00079858A859B8586DF80933A39CFC068818B
:1025C00079818A819B817EDF80933A39C7C080916F
:1025D0002539811111C0688579858A859B8572DFCF
:1025E0000DE119E3F801858F6C857D858E859F85CA
:1025F00069DFF801868FB2C0688179818A819B8109
:1026000061DF0DE119E3F801858F6C817D818E8199
:102610009F8158DFF801868FA1C0809125398111F3
:1026200011C06C857D858E859F854CDF0DE119E39A
:10263000F801858F688979898A899B8943DFF80148
:10264000868F8CC0688179818A819B813BDF0DE117
:1026500019E3F801858F6C817D818E819F8132DF46
:10266000F801868F7BC08091253981111FC0688950
:1026700079898A899B8926DF0DE119E3F801858F25
:102680006C897D898E899F891DDFF801868F688D11
:10269000798D8A8D9B8D16DFF801878F6C8D7D8DEE
:1026A0008E8D9F8D0FDFF80180A358C068817981DE
:1026B0008A819B8107DF0DE119E3F801858F6C8129
:1026C0007D818E819F81FEDEF801868F6885798508
:1026D0008A859B85F7DEF801878F6C857D858E85E1
:1026E0009F85F0DEF80180A339C0809125398111E2
:1026F00011C0688979898A899B89E4DE0DE119E333
:10270000F801858F6C897D898E899F89DBDEF801D0
:10271000868F24C0688179818A819B81D3DE0DE117
:1027200019E3F801858F6C817D818E819F81CADEDE
:10273000F801868F13C080912539811108C06C85FE
:102740007D858E859F85BEDE80933A3907C068817E
:1027500079818A819B81B6DE80933A39DF91CF916E
:102760001F910F910895843040F5EDE1F9E341A503
:1027700052A5242F30E0082E02C0359527950A94E3
:10278000E2F720FF0AC0252F30E0082E02C0359561
:1027900027950A94E2F720FD10C021E030E0B9014E
:1027A00002C0660F771F8A95E2F7CB01EDE1F9E3EE
:1027B000462B41A78095852382A70895843090F405
:1027C00021E030E0A90102C0440F551F8A95E2F7CD
:1027D000CA018095EDE1F9E391A5982391A792A50F
:1027E000892382A70895BF92CF92DF92EF92FF9242
:1027F0000F931F93CF93DF930AE319E3CDE1D9E35E
:102800006E017801B12CF70181917F01F60121A1C0
:1028100090E0820F911D22A1820F911D039719F460
:102820008B2DA1DF02C08B2DC9DFB394F2E0CF0E58
:10283000D11C84E0B812E7CF25E239E389A18AA34D
:10284000F80181918F0189A32296C217D307B1F7AE
:10285000DF91CF911F910F91FF90EF90DF90CF907C
:10286000BF900895843060F42091463930E0A9018A
:1028700002C0559547958A95E2F7CA01817008957F
:1028800080E00895843060F42091473930E0A90158
:1028900002C0559547958A95E2F7CA01817008955F
:1028A00081E00895843000F5662379F0EDE1F9E3E5
:1028B00021E030E0A90102C0440F551F8A95E2F7DC
:1028C000CA0192A5892B82A70895EDE1F9E321E0E1
:1028D00030E0A90102C0440F551F8A95E2F7CA01F2
:1028E000809592A5892382A70895CF93833009F11B
:1028F00028F4813031F0823061F02CC0883008F14A
:1029000029C080913439882329F181E080933539B9
:1029100021C0C1DD8823F1F061E080E0C3DF61E028
:1029200081E0C0DF61E082E0BDDF61E083E0BADF2B
:1029300011C080912639882369F081E0809327397E
:1029400009C0CCEFC80F8C2F8DDF882319F061E010
:102950008C2FA8DFCF910895009781F0FC01DC0156
:10296000AD5BBD4F80818C936083643021F481E046
:102970000D94F815089580E00D94F81508950097CA
:1029800019F0FC018081089580E00895009741F0DE
:10299000613021F421E0FC0122AB0895FC0112AA70
:1029A0000895009719F0FC0182A9089580E0089528
:1029B000009741F0613021F421E0FC0123AB089540
:1029C000FC0113AA0895009719F0FC0183A908954A
:1029D00080E008958F929F92AF92BF92DF92EF9224
:1029E000FF920F931F93CF93DF934115510509F485
:1029F0006BC08A017B01C82F0E945BD4D82F8C2F1B
:102A00000E9478D4D82EDD2309F460C0882309F40D
:102A10005FC08D2F0E9441D04B015C018D2D0E9423
:102A200041D0672B682B692B39F4F8011082118291
:102A30001282138280E04DC09701280D391D032EAC
:102A4000000C440B550BC63050F4A0E1B7E20F94D4
:102A5000E364F801608371838283938309C0A8EEE5
:102A6000B3E00F94E364F8016083718382839383FE
:102A70008D2D0E9441D09B01AC01F80160817181D4
:102A8000828193810F94AA6488279927DC01821B95
:102A9000930BA40BB50BF80180839183A283B383BE
:102AA0008C2F0E941ED8F80180809180A280B38074
:102AB000DC01CB01880D991DAA1DBB1D808391836C
:102AC000A283B38381E005C080E003C080E001C041
:102AD00080E0DF91CF911F910F91FF90EF90DF90F9
:102AE000BF90AF909F908F900895CF93DF93009702
:102AF00009F460C0EC010F94C928813091F58C83F2
:102B00000F9420118823F9F08091493F811119C059
:102B100089E0E4EEF0E2A0EDB4E401900D928A9534
:102B2000E1F7E0EDF4E401900020E9F73197AF011F
:102B3000405D544421E060ED74E48AEA99E30F9427
:102B40008B310F9459110F942311882399F18EEB37
:102B500098E40E946CDE0F941D118A830F946A1111
:102B600029C01C820F94F5288823F9F08091493FF1
:102B7000811119C089E0EDEEF0E2A0EDB4E401901E
:102B80000D928A95E1F7E0EDF4E401900020E9F779
:102B90003197AF01405D544421E060ED74E48AEA6E
:102BA00099E30F948B310F94F8280F94E128811149
:102BB0000F94E428DF91CF9108950F931F93CF9343
:102BC000DF93009709F463C0EC010F94402B882336
:102BD00081F18B8181115BC08091493F811126C0B9
:102BE0000F940929182F0F941D111F921F931F92E4
:102BF0008F938FEF90E29F938F9300ED14E41F93D8
:102C00000F930F94F366F80101900020E9F73197D4
:102C1000AF01405D544420E0B8018AEA99E30F9483
:102C20008B318DB79EB708968DBF9EBF81E08B8399
:102C30002EC08B81813059F51B828091493F8111D3
:102C400026C00F940929C82F0F941D111F92CF93EE
:102C50001F928F9386EF90E29F938F93C0EDD4E401
:102C6000DF93CF930F94F36609900020E9F7219743
:102C7000AE01405D544420E060ED74E48AEA99E3DB
:102C80000F948B318DB79EB708968DBF9EBFDF9195
:102C9000CF911F910F910895CF92DF92EF92FF9203
:102CA0000F931F93CF93DF93009709F4AAC0611588
:102CB000710509F4A6C08B01EC010E940ADE88238D
:102CC00009F49FC00F9488296B017C010F942D2B70
:102CD00086E10E9465D0AB01BC0183E29DE30E94C6
:102CE000A0DED701C6010197A109B109883E934032
:102CF000A105B10508F03FC00E9474C8823088F178
:102D00008091493F81112DC00F941D111F928F9307
:102D100080912B541F928F93FF92EF92DF92CF926C
:102D200082E191E29F938F930F2EF0EDEF2EF4E46A
:102D3000FF2EF02DFF92EF920F94F366F7010190B2
:102D40000020E9F73197AF01405D544421E0B7011D
:102D50008AEA99E30F948B318DB79EB70C968DBF9D
:102D60009EBF25ED35E44FEE57E469E277E4C801F4
:102D70000E946EEA43C0D701C601895E9340A10953
:102D8000B10984369105A105B105C0F58FEE95E432
:102D90000E9402DE811132C08091493F811125C01D
:102DA000FF92EF92DF92CF928EE191E29F938F9309
:102DB0000F2EF0EDEF2EF4E4FF2EF02DFF92EF92A8
:102DC0000F94F366F70101900020E9F73197AF0106
:102DD000405D544421E0B7018AEA99E30F948B31B6
:102DE0008DB79EB708968DBF9EBF25ED35E44FEE9B
:102DF00057E469E277E4C8010E946EEACE010E94BE
:102E000023DEDF91CF911F910F91FF90EF90DF9024
:102E1000CF900895FC01892B39F0118689E0DF01FC
:102E20001D928A95E9F712860895FC01892B41F0DD
:102E3000118689E0DF011D928A95E9F712861386D3
:102E400008950F931F93CF93DF93CBE4D9E303EA65
:102E500019E3CE01DFDF2B96C017D107D1F78FED35
:102E60009CE3E3DF8BEE9CE3E0DF0F94A62DDF9184
:102E7000CF911F910F910895FC01892B31F081E0D2
:102E80009285913019F080E0089580E008951F93B5
:102E9000CF93DF93CDB7DEB76097CDBFDEBF9C0188
:102EA000FE013196AE014F5E5F4F21933193255F56
:102EB0003F4FE417F507C9F7892B31F110E010C037
:102EC000E12FF0E0EE0FFF1F81E090E08C0F9D1FDF
:102ED000E80FF91F80819181CFDF8823D1F01F5F38
:102EE0000F942D2C181760F382E00E9465D06B3090
:102EF00068F08091EA3C882359F081E09091F63C9B
:102F0000911107C080E005C080E003C081E001C0EE
:102F100080E06096CDBFDEBFDF91CF911F91089515
:102F2000CF92DF92EF92FF920F931F93CF93DF9395
:102F3000CDB7DEB72597CDBFDEBF19821A821B82BF
:102F40001C824115510559F16A017B01182FCA01F4
:102F500061DFAE014F5F5F4FB701812F3BDD8823FB
:102F6000C9F009811A812B813C814BE0BE016B5F66
:102F70007F4FC6010F940F39F60101900020E9F749
:102F80003197EC19FD09D6011996EC93199781E058
:102F90001A968C9369817A818B819C8103C060E051
:102FA00070E0CB012596CDBFDEBFDF91CF911F91A1
:102FB0000F91FF90EF90DF90CF9008958F929F92A6
:102FC000AF92BF92EF92FF920F931F93CF93DF9335
:102FD0000097A1F06115710589F0142F7B01EC01B8
:102FE0000F942B164B015C01113009F4FAD99501AD
:102FF00084014BE0B701CE010F946137DF91CF918F
:103000001F910F91FF90EF90BF90AF909F908F9086
:103010000895AF92BF92CF92DF92EF92FF920F93FB
:103020001F93CF93DF93CDB7DEB76097CDBFDEBFE1
:103030008C01CE0101967C014096F701619371935A
:10304000655F7F4FE817F907C9F70115110509F406
:1030500075C282E00E9465D0D62E96E0D91206C0D5
:10306000C8010F94772781116FC243C38FEF8D0D75
:10307000823030F4C8010F947727811111C039C311
:103080008FEE8D0D823030F4C8010F9477278111B7
:1030900007C02FC3C8010F947727882309F429C3D9
:1030A00080E2E3E7F0E4DF011D928A95E9F780E131
:1030B000E8EBFBE3DF011D928A95E9F78D2D90E0A7
:1030C000FC013197E231F10508F03AC28827ED5E44
:1030D000FE4F8F4F0D94C66458010F2EF3E7CF2E8D
:1030E000F0E4DF2EF02D01E010E00EC10F94742704
:1030F000C82E49815A81F8016081718111DF0F2E3C
:10310000F3E7EF2EF0E4FF2EF02DD7016D937D93C2
:103110008D939C9313974B815C81F801628173813D
:103120008C2DFEDED70114966D937D938D939C9329
:103130001797B2E0DB1206C2809173409091744001
:10314000A0917540B09176408093B83B9093B93B85
:10315000A093BA3BB093BB3B81E0CBC258010F2E8A
:10316000F3E7CF2EF0E4DF2EF02D01E010E00BC0EE
:103170001F5F0F5FE2E0EE0EF11CF2E0AF0EB11C3C
:1031800084E0C80ED11C112309F4FBC1123009F4EC
:10319000EAC1D7014D915C91F5016081718180E0B8
:1031A000BFDED6016D937D938D939C93139704306E
:1031B000F8F28091734090917440A0917540B09165
:1031C00076408093B83B9093B93BA093BA3BB093C1
:1031D000BB3B81E08EC258010F2EF3E7CF2EF0E407
:1031E000DF2EF02D01E010E00BC01F5F0F5FB2E09B
:1031F000EB0EF11CE2E0AE0EB11CF4E0CF0ED11CE0
:10320000112309F4DBC1123009F4CAC1D7014D9171
:103210005C91F5016081718182E082DED6016D935F
:103220007D938D939C9313970430F8F2E8EBFBE3C6
:10323000A3E7B0E44D915D916D917C91139740832C
:1032400051836283738314968D919D910D90BC91EF
:10325000A02D84839583A683B78381E04AC2580159
:103260000F2EF3E7CF2EF0E4DF2EF02D01E010E07B
:103270000BC01F5F0F5FB2E0EB0EF11CE2E0AE0E81
:10328000B11CF4E0CF0ED11C112309F4B8C11330E6
:1032900009F4A3C1113009F4A2C1143009F4A1C189
:1032A000D7014D915C91F5016081718180E038DE3C
:1032B000D6016D937D938D939C9313970630C8F23E
:1032C000E8EBFBE3A3E7B0E44D915D916D917C9158
:1032D0001397408351836283738314968D919D91DC
:1032E0000D90BC91A02D84839583A683B78381E044
:1032F00000C21F5F0F5FB2E0EB0EF11CE2E0AE0E0A
:10330000B11CF4E0CF0ED11C112309F487C1143095
:1033100009F492C1812F8B7F813009F48FC18230F3
:1033200009F48EC1D7014D915C91F50160817181E5
:1033300085E0F6DDD6016D937D938D939C93139775
:103340000830B8F2E8EBFBE3A3E7B0E44D915D9100
:103350006D917C911397408351836283738314969C
:103360004D915D916D917C91179744835583668350
:10337000778318964D915D916D917C911B97408755
:103380005187628773871C968D919D910D90BC919A
:10339000A02D84879587A687B78781E0AAC15801A9
:1033A0000F2EF3E7CF2EF0E4DF2EF02D01E010E03A
:1033B0000BC01F5F0F5FB2E0EB0EF11CE2E0AE0E40
:1033C000B11CF4E0CF0ED11C112309F458C1143004
:1033D00009F445C1812F8B7F813009F442C1D701A7
:1033E0004D915C91F5016081718180E099DDD6019C
:1033F0006D937D938D939C9313970830D0F2E8EBF7
:10340000FBE3A3E7B0E44D915D916D917C9113973F
:10341000408351836283738314968D919D910D90A7
:10342000BC91A02D84839583A683B78381E061C17D
:10343000680103E710E45E01B9E0AB0EB11CF701CF
:10344000419151917F01D6016D917D916D0180E097
:1034500067DDF80161937193819391938F01EA1471
:10346000FB0469F781E045C158010F2EF3E7CF2E29
:10347000F0E4DF2EF02D01E010E00BC01F5F0F5FC6
:10348000F2E0EF0EF11C82E0A80EB11C94E0C90E30
:10349000D11C112309F410C1133009F4FFC0D70166
:1034A0004D915C91F5016081718180E039DDD6013B
:1034B0006D937D938D939C9313970630F8F28091D2
:1034C000734090917440A0917540B0917640809384
:1034D000B83B9093B93BA093BA3BB093BB3B81E020
:1034E00008C158010F2EF3E7CF2EF0E4DF2EF02DA8
:1034F00001E010E00BC01F5F0F5FB2E0EB0EF11CAC
:10350000E2E0AE0EB11CF4E0CF0ED11C112309F4A1
:10351000E2C0D7014D915C91F5016081718181E03C
:10352000123009F480E0FCDCD6016D937D938D931D
:103530009C9313970430F8F281E0DBC080E0D9C09F
:1035400080E0D7C081E0D5C080E2E3E7F0E4DF01AE
:103550001D928A95E9F780E1E8EBFBE3DF011D921C
:103560008A95E9F7B9CDF70140815181D5016D9177
:103570007C9183E0D5DCF601608371838283938341
:10358000F7CDD7014D915C91F5016081718183E0A8
:10359000C7DCD6016D937D938D939C931397E8CDF3
:1035A000F70140815181D5016D917C9183E0B8DCB8
:1035B000F601608371838283938317CED7014D9187
:1035C0005C91F5016081718183E0AADCD6016D9385
:1035D0007D938D939C93139708CE83E003C082E084
:1035E00001C082E0F70140815181D5016D917C914C
:1035F00097DCF60160837183828393833ACED7018F
:103600004D915C91F5016081718183E089DCD60187
:103610006D937D938D939C9313972BCEF7014081EF
:103620005181D5016D917C9183E07ADCF601608354
:103630007183828393835DCE83E003C082E001C007
:1036400084E0D7014D915C91F5016081718168DC66
:10365000D6016D937D938D939C9313974ACE83E00F
:1036600001C082E0F70140815181D5016D917C91CB
:1036700057DCF60160837183828393839ACED701EE
:103680004D915C91F5016081718183E049DCD60147
:103690006D937D938D939C9313978BCEF70140810F
:1036A0005181D5016D917C9183E03ADCF601608314
:1036B000718382839383E2CED7014D915C91F501B2
:1036C0006081718183E02CDCD6016D937D938D93B5
:1036D0009C931397D3CEF70140815181D5016D9111
:1036E0007C9180E01DDCF60160837183828393838B
:1036F00002CF6096CDBFDEBFDF91CF911F910F91BA
:10370000FF90EF90DF90CF90BF90AF9008950F940F
:10371000DD24882329F00F94EE2484E0809327068B
:103720000895CF93DF93009799F1EC018881813060
:10373000A8F0833018F0863019F010C0E8DF25C0FB
:103740008091280682FD03C084E0809325060F94B3
:1037500077248823D1F00F94882417C00F947724FE
:10376000882399F00F94882484E0809327060DC065
:103770008D8181110DC00F94BB24882349F00F94D3
:10378000CC2484E08093270603C08881863081F7AB
:10379000DF91CF9108950E9444E20F940D2A20E119
:1037A00037E240E050E00F948864672B682B692B68
:1037B000E1F40E9444E2813019F40C9458E1089538
:1037C0000E9444E2823021F481E00C9447E20895A3
:1037D0000E9444E2833019F40C944DE408950E9451
:1037E00044E2843011F40C94A1E408950F931F93E4
:1037F000CF93DF931F921F92CDB7DEB719821A8243
:103800000097B9F08C010E94A45690E006969E01A4
:103810002F5F3F4F43E060E0800F911F0F94C03552
:10382000882339F049815A8160E070E080E00E948D
:1038300050D00F900F90DF91CF911F910F9108956D
:103840009F92AF92BF92CF92DF92EF92FF920F932F
:103850001F93CF93DF931F92CDB7DEB7009709F484
:103860004BC05C0182E00E9465D0962E8501085D08
:103870001F4FBE016F5F7F4FC8010E9417EF882363
:1038800091F0F501C0A4D1A4E2A4F3A489E00E94C0
:1038900065D0AB01BC010AE619E42AE539E4898167
:1038A0000F94282A17C0BE016F5F7F4FC8010E9486
:1038B00063F8F501C0A4D1A4E2A4F3A489E00E94B6
:1038C00073D0AB01BC010AE619E42AE539E4898129
:1038D0000F94282AFAE0F91558F4F50140A551A5EE
:1038E00062A573A582E599E40F940D2D81E005C0D2
:1038F0000F94772D81E001C080E00F90DF91CF9190
:103900001F910F91FF90EF90DF90CF90BF90AF90FD
:103910009F900895CF92DF92EF92FF920F931F93A3
:10392000CF93DF931F92CDB7DEB7009779F18C016B
:10393000BE016F5F7F4F88960E945EFB882399F0DF
:10394000F801C0A4D1A4E2A4F3A489E00E9465D048
:10395000AB01BC010AE619E42AE539E489810F9438
:10396000282A81E014C0F801C0A4D1A4E2A4F3A4E1
:1039700089E00E9473D0AB01BC010AE619E42AE594
:1039800039E489810F94282A81E001C080E00F90FA
:10399000DF91CF911F910F91FF90EF90DF90CF902B
:1039A000089589E10E9465D0623059F482E00E9456
:1039B00065D0673041F0693031F0613021F081E04D
:1039C000089580E0089580E0089589E10F941B1721
:1039D000623059F482E00F941B17673041F0693070
:1039E00031F0613021F081E0089580E0089580E0B9
:1039F00008953F924F925F926F927F928F929F9223
:103A0000AF92BF92CF92DF92EF92FF920F931F93EC
:103A1000CF93DF93CDB7DEB76497CDBFDEBFB82EAF
:103A20008B017A0189E10E9465D0A62E011511054E
:103A300009F472C28091493F882339F00F2EFAEAC7
:103A4000CF2EF9E3DF2EF02D06C00F2EF1EBCF2E97
:103A5000FAE3DF2EF02D82E08A1508F4A12C8BE723
:103A6000F801808383E781838CE28283F2E3BF12D3
:103A700007C082E38A0DF80183838CE284830BC044
:103A8000F801B3828CE28483F0E3BF1609F4F1C13C
:103A900082E3B81218C28BE499E3FE0132969E01CC
:103AA0002E5E3F4F819391930B962E173F07D1F7D0
:103AB00088E08983E114F10469F086E0F701D80118
:103AC000159601900D928A95E1F70F2EFBE0FF2EDF
:103AD000F02D04C00F2EF5E0FF2EF02DF801EF0DB4
:103AE000F11D8CE2808382E00E9465D0762E872DC6
:103AF000072C000C990B9F937F928BE191E29F938F
:103B00008F93F394C8018F0D911D9F938F930F9402
:103B1000F366F80101900020E9F73197E01BF10B03
:103B20007F01FF24F801EE0DFF1D118221E0A701A6
:103B3000B801C6010F948B310F900F900F900F902A
:103B40000F900F908091493F811112C01A8A21E095
:103B500040E050E0BE016E5E7F4F8AEA99E30F9429
:103B60008B3120E0A701B8018AEA99E30F948B31E9
:103B700091E09A1508F402C11982912C0F2EFCE2F3
:103B80008F2EF02DF8013196EB8BFC8B0F2EF9E484
:103B90004F2EFFE35F2EF02D5BC00F942D2C69801C
:103BA000861509F45BC0F8018082E62CF12CF70140
:103BB000EE0FFF1F81E090E08C0F9D1FE80FF91FB3
:103BC000A180B280F501418550E0B5018B899C89C7
:103BD0000F94C566F50181856894332431F8380E59
:103BE0008F5FF801E80FF11D8082F7013196EE0F2B
:103BF000FF1F81E090E08C0F9D1FE80FF91FA1804F
:103C0000B280F501418550E0B501C801830D911DD9
:103C10000F94C566F501E1843E0C63946394698258
:103C2000E32CF12CF801EE0DFF1D118221E0A7011C
:103C3000B801C6010F948B31F2018081811107C058
:103C400020E0A701B8018AEA99E30F948B3193949D
:103C50000F942D2C8695981608F49FCFFAE0F7154F
:103C60000CF0D8C08CE078164CF09DE097150CF065
:103C700050C180EF870D833008F44BC1198280E07A
:103C80000F2EFCE23F2EF02D4801EFEF8E1A9E0A18
:103C90000F2EF9E44F2EFFE35F2EF02DF801308256
:103CA000E82EF12CF701EE0FFF1FEE0DFF1DEE0FBA
:103CB000FF1FEE0FFF1FE152F34C82858C3419F089
:103CC000823541F00EC080E39CE2F4018083918351
:103CD00012820FC081E39CE2F401808391831282FF
:103CE00008C085E0E0E3F1E2D40101900D928A95ED
:103CF000E1F7F80101900020E9F731975F01A01A80
:103D0000B10A3701660C771CB3016E0D7F1D660F7B
:103D1000771F660F771F6152734CFB01418550E09E
:103D2000C8018A0D911D0F94C566F301EE0DFF1DAC
:103D3000EE0FFF1FEE0FFF1FE152F34C8185A80E1F
:103D4000B12CF801EA0DFB1D118221E0A501B8019B
:103D5000C6010F948B31F2018081811107C020E0F0
:103D6000A501B8018AEA99E30F948B31E98081E0DB
:103D70008E0D8983823008F491CF4CC01982612C5A
:103D80000F2EFCE25F2EF02D4801FFEF8F1A9F0AE5
:103D90000F2EF9E4AF2EFFE3BF2EF02D36C00F94A7
:103DA0002D2C79808715B1F1F8015082E72DF0E0D4
:103DB000EE0FFF1F81E090E08C0F9D1FE80FF91FB1
:103DC000E180F280F701418550E0B701C4010F9412
:103DD000C566F701E184E39473947982F12CF801CC
:103DE000EE0DFF1D118221E0A701B801C6010F945D
:103DF0008B31F5018081811107C020E0A701B80156
:103E00008AEA99E30F948B3163940F942D2C869555
:103E1000681628F20F2EFCE2FF2EF02DF801F0823A
:103E200084E00E9465D0605DF8016183F28240E029
:103E3000BE016F5F7F4FC8010396C0D8898193E0B0
:103E4000980FF801E90FF11D9DE790838C5FE82E34
:103E5000F12CF801EE0DFF1D118221E0A701B80140
:103E6000C6010F948B318091493F882309F445C0E6
:103E700053C00F2EF8E2EF2EF7E4FF2EF02DF701DE
:103E8000408150E061EF76E4C80105960F94C56665
:103E9000F701808195E0980FF801E90FF11D9DE78A
:103EA00090838A5FE82EF12CF801EE0DFF1D118240
:103EB00021E0A701B801C6010F948B318091493FE1
:103EC00081112AC011C021E045E050E0B801C601CF
:103ED0000F948B318091493F81111EC0F0E3BF12D6
:103EE0000FC045E050E002C04E2D5F2D20E0B8012C
:103EF0008AEA99E30F948B310FC04E2D5F2D02C0DB
:103F000045E050E021E0B8018AEA99E30F948B3153
:103F100003C081E08983B4CE6496CDBFDEBFDF915C
:103F2000CF911F910F91FF90EF90DF90CF90BF90B6
:103F3000AF909F908F907F906F905F904F903F9049
:103F40000895CF93892B81F00E94B255CAE00E9458
:103F500075560E94AF55882321F00E94C5558111E6
:103F600005C0C150A1F703C0C0E001C0C1E08C2F63
:103F7000CF91089589E10E9465D0611104C00F942A
:103F80003411882371F081E04091305450913154C4
:103F90006091325470913354452B462B472B09F0D6
:103FA00080E008958F929F92AF92BF92CF92DF925E
:103FB000EF92FF920F931F93CF93DF930097A9F196
:103FC000EC0186E00E9465D04B015C0184E00E9418
:103FD00065D0162F87E00E9465D0062F812F0F94A1
:103FE0000F160F942B166B017C0186169706A806F8
:103FF000B906D9F0AB01BC0186E00E94B9D588238F
:10400000A1F00F94B815B701A60186E00E945BD01D
:10401000B701A60186E00F942E17602F812F0F9411
:104020000F1668E0CE010E94AC14DF91CF911F9172
:104030000F91FF90EF90DF90CF90BF90AF909F9047
:104040008F90089582E10E9465D028E0E2E6F4E5D1
:10405000DF01322F1D923A95E9F7EAE6F4E5DF0138
:104060001D922A95E9F721E030E0672B682B692B38
:1040700011F420E030E0F901E153FF4D80818560CB
:10408000E8E2F4E582AF83AF81E00895CF93DF9358
:104090000097A1F0613071F4EC01E3EBF0E4628190
:1040A0007381808191810F941458CA5CDD4F81E047
:1040B000888304C0FC01EA5CFD4F1082DF91CF9140
:1040C00008950097B1F0FC0180818430A1F40F9431
:1040D0006029823039F089E10E9465D0672B682B16
:1040E000692B59F00F943D2991E0811107C090E0B0
:1040F00005C090E003C090E001C090E0892F0895D2
:104100000F931F93CF93DF938C01EB01209709F45A
:1041100042C01882892B19F189E10E9465D0F8010B
:1041200080818130C0F0833018F08530D0F013C02A
:10413000611106C02097B9F087E4888380E02EC023
:104140006150623090F0209791F087E4888380E09E
:1041500025C0209771F082E4888380E01FC080E052
:104160001DC081E01BC080E019C081E017C080E065
:1041700015C080E013C081E011C080E00FC089E16C
:104180000E9465D0F8018081813018F3833080F27D
:10419000853088F3DECF892B91F7EFCFDF91CF9178
:1041A0001F910F910895009739F0FC018081815093
:1041B000843020F481E0089580E0089580E008953F
:1041C000009751F0FC018081813040F0843010F084
:1041D000853021F481E0089580E0089580E008951D
:1041E000CF92DF92EF92FF92CF93DF93009709F483
:1041F0005FC0EC0183E00E9465D06B017C01AB01E4
:10420000BC0155276627772783E00E94B9D588230C
:1042100009F44BC08C2DFE01E95CFD4FC08281305A
:1042200021F1823009F044C088E00E9465D0FE018F
:10423000E75CFD4F6083AB01BC01552766277727FC
:1042400088E00E94B9D5811105C081E0FE01E75CDC
:10425000FD4F8083FE01E85CFD4F1082C65CDD4FA0
:10426000188219821A821B8223C087E00E9465D0BF
:10427000F62E84E00E9465D0862F6F2D0F940F16C6
:1042800085E00E9465D00F94C016FE01E25CFD4FF0
:1042900060837183828393830F94D815C65CDD4F4E
:1042A000188219821A821B8203C0C95CDD4F1882F2
:1042B000DF91CF91FF90EF90DF90CF90089500971E
:1042C00061F1FC01E85CFD4F2081319630813217AD
:1042D00010F021111BC0FC01E85CFD4F3150308310
:1042E00032964081518162817381403821E55207C5
:1042F00021E06207710598F44F5F5F4F6F4F7F4F6A
:10430000408351836283738381E00895FC01E85CFC
:10431000FD4F2150208380E0089580E0089580E0E3
:1043200008950F931F93CF93DF93009741F1EC0112
:104330000F94EF15FE01E25CFD4F00811181228197
:1043400033816017710782079307D8F00F94D8154F
:10435000FE01E65CFD4F80819181A281B3818038AE
:1043600021E5920721E0A207B10568F40196A11D9D
:10437000B11D80839183A283B38381E005C080E077
:1043800003C080E001C080E0DF91CF911F910F91C9
:104390000895CF93DF93009709F43DC0FC01EA5CD8
:1043A000FD4F20812223B9F1EC018BDE813021F415
:1043B000CA5CDD4F18822FC089E10E9465D061116F
:1043C0001AC00F946029813031F1823089F4D2DD36
:1043D000882309F10F941A29CA5CDD4F18828FEEE9
:1043E00095E40E94FCDD8EEB98E40E9423DE13C06E
:1043F0000F944E2910C0BEDD882369F00F941A294E
:10440000CA5CDD4F18828FEE95E40E94FCDD8EEBD6
:1044100098E40E9423DEDF91CF910895FF920F93DD
:104420001F93CF93DF936115710509F47CC041158B
:10443000510509F478C08A01EB01F82E82E10F944E
:104440001B1721E0672B682B692B09F420E08F2DC7
:1044500090E0FC013197E231F10508F05BC088275C
:10446000EB5DFE4F8F4F0D94C6641882E22FF0E093
:10447000E153FF4D80818560F801808354C083E063
:104480008883E22FF0E0E153FF4D8081F8018083C3
:104490004AC01882E22FF0E0E153FF4D8081816035
:1044A000F801808340C083E08883E22FF0E0E1538D
:1044B000FF4D8081F801808336C01882E22FF0E042
:1044C000E153FF4D80818160F80180832CC083E03F
:1044D0008883E22FF0E0E153FF4D8081F801808373
:1044E00022C0188285E0F80180831DC0188281E017
:1044F000F801808318C01882E22FF0E0E153FF4DED
:1045000080818160F80180830EC0188281E0F8010B
:10451000808309C01882E22FF0E0E153FF4D8081D3
:104520008560F8018083DF91CF911F910F91FF90FB
:1045300008958F929F92AF92BF92CF92DF92EF92A7
:10454000FF920F931F93CF93DF93892B09F486C0BB
:1045500089E00E9465D09B01AC01A8EEB3E00F9406
:10456000E3646B017C010F947129C616D706E80637
:10457000F90609F475C0C701B60128EE33E040E042
:1045800050E00F948864F22ED22F2E3108F06AC0CA
:10459000213009F469C00F94712928EE33E040E01E
:1045A00050E00F948864822FF21638F46F2D0F9428
:1045B0005564C92F992309F45CC00F940929E82E8A
:1045C0006D2F0F945564D92F892F90E08E0D911D7A
:1045D000CA970CF04BC08D2E912CA12CB12C0F94AE
:1045E0008829162F072FD82EC92EA8EEB3E0A501D3
:1045F00094010F94E3644F2D0F94B629C091493F65
:10460000C11136C00F9488299F938F937F936F9326
:10461000CF92DF920F931F931F92DF931F92EF921F
:1046200085E391E29F938F9300ED14E41F930F9322
:104630000F94F366F80101900020E9F73197AF017C
:10464000405D544421E0B8018AEA99E30F948B312C
:104650008DB79EB740968DBF9EBF0BC0C0E009C00E
:10466000C0E007C0C1E005C0C0E003C0C1E001C0B8
:10467000C0E08C2FDF91CF911F910F91FF90EF90B1
:10468000DF90CF90BF90AF909F908F900895EF9262
:10469000FF920F931F93CF93DF932091493F2223E3
:1046A00039F00F2EFAEAEF2EF9E3FF2EF02D06C0B7
:1046B0000F2EF1EBEF2EFAE3FF2EF02D0097D1F144
:1046C000EC018BE7888388E689838CE28A8392E613
:1046D0009B838C837F936F9380E791E29F938F936B
:1046E000CE0105969F938F930F94F366FE01019080
:1046F0000020E9F73197EC1BFD0B8F01112721E01A
:10470000A801BE01C7010F948B310E9474C80F909D
:104710000F900F900F900F900F90873059F4809169
:10472000493F811107C021E0A801BE018AEA99E34F
:104730000F948B31DF91CF911F910F91FF90EF90EC
:1047400008958F929F92AF92BF92CF92DF92EF9295
:10475000FF920F931F93CF93DF93009709F470C0DC
:104760002091493F222339F00F2EFAEAEF2EF9E388
:10477000FF2EF02D06C00F2EF1EBEF2EFAE3FF2EE9
:10478000F02DEC018BE7888388E689838CE28A83AD
:1047900093E79B838C8307EF1CE3F801848C0E94D2
:1047A000C3A6982EA090483FB090453FF801C28024
:1047B000D0800F9434111F928F921F929F921F925C
:1047C000AF921F92BF921F92CF921F92DF921F92C1
:1047D0008F93F80185811F928F9384811F928F930D
:1047E00083811F928F9385E591E29F938F93CE01F2
:1047F00005969F938F930F94F366FE01019000201E
:10480000E9F73197EC1BFD0B8F01112721E0A8017F
:10481000BE01C7010F948B318DB79EB748968DBFEF
:104820009EBF8091493F81110BC0A80142505109A0
:10483000BE016F5F7F4F21E08AEA99E30F948B31CD
:10484000DF91CF911F910F91FF90EF90DF90CF906C
:10485000BF90AF909F908F900895DF92EF92FF925C
:104860000F931F93CF93DF9300D01F92CDB7DEB786
:104870008C010F94FF24882349F00F9410250E9487
:10488000131089E493E45DDF80E066C0CE010196F9
:104890000E941C10882309F45FC0F090A806E090E5
:1048A0006806D0902806BE016D5F7F4FCE0101964D
:1048B0000E943210882309F44CC00E9480C88823CB
:1048C000C9F18091493F811135C0D0FADD24D0F87B
:1048D0001F92DF92E4FAEE24E0F81F92EF92F6FACC
:1048E000FF24F0F81F92FF928A818F9389818F9322
:1048F0008C818F938B818F9384E791E29F938F9329
:104900000F2EF0EDEF2EF4E4FF2EF02DFF92EF923C
:104910000F94F366F70101900020E9F73197AF019A
:10492000405D544421E0B7018AEA99E30F948B314A
:10493000CDBFDEBF6B817C8189E493E4A8DE0115E5
:10494000110549F08B819C81F8018083918381E07E
:1049500003C081E001C081E02496CDBFDEBFDF91BE
:10496000CF911F910F91FF90EF90DF9008958823D2
:1049700021F081E08093483F08951092483F0895C8
:104980000F931F93CF93DF936115710571F000971B
:1049900061F0EB018C010F942125882331F00F94F5
:1049A0003225BE01C8010E94C590DF91CF911F91B1
:1049B0000F910895CF93DF93009751F0EC010F947E
:1049C0006D25882329F0CE010E9407930F947E2540
:1049D000DF91CF910895009791F0FC01EC5BFD4FC2
:1049E0002FEF3FE720833183329620E030E82083A9
:1049F000318332961082118232961082118208958C
:104A00000F93CF93DF930097A1F0662371F0EA0133
:104A1000FC01E45BFD4F81E08083C9010F947F2B93
:104A2000602FCE010E9468A804C0FC01E45BFD4F2A
:104A30001082DF91CF910F910895EF92FF920F9323
:104A40001F93CF93DF931F921F92CDB7DEB70097CE
:104A500009F498C06115710509F494C0FC0122A9FC
:104A6000211104C023A9222309F48CC08B017C01ED
:104A7000FC0112AA13AA0E946F110E94FA110E944F
:104A8000F313F70144A955A9B7016A5C7F4F9E0152
:104A90002F5F3F4FC8010F94EA5AC8010F94985CEA
:104AA000F701E75AFD4FD701AD5ABD4F8C91808376
:104AB000319611968C9180830F9488299F938F93C0
:104AC0007F936F9383E991E29F938F9300ED14E4BA
:104AD0001F930F930F94F366F80101900020E9F7FC
:104AE0003197AF01405D544421E0B8018AEA99E36F
:104AF0000F948B31CDBFDEBFF70124A935A9898181
:104B00009A812817390719F1C70106969F938F9349
:104B10008FE991E29F938F931F930F930F94F36606
:104B2000F80101900020E9F73197AF01405D54444E
:104B300021E0B8018AEA99E30F948B310E9415A90C
:104B40000F900F900F900F900F900F9002C00E9447
:104B5000A5A8E5E8F3E4808190E0DC01AB57BC4B0D
:104B600025853685880F991FFC01EB57FC4B418149
:104B700052811F960C9161E0C70142DF0E946B9544
:104B80000F94E52B0F900F90DF91CF911F910F9114
:104B9000FF90EF9008950F931F93CF93DF930097AB
:104BA00009F448C06115710509F444C08B01EC019A
:104BB000FC01E45BFD4F80818823C1F1DB018C9116
:104BC000882341F10F949B2B8823A1F1F801608188
:104BD00061506083611108C00E94DAA80E94C7A8D2
:104BE000C45BDD4F188226C070E0F801E60FF71FA6
:104BF000D8011D962D913C911E97660F771FA60F29
:104C0000B71F11964D915C911297078561E0CE0117
:104C1000F7DE10C00F949B2B882361F00E94DAA866
:104C20000E94C7A8C45BDD4F188204C00E94DAA8A6
:104C30000E94C7A8DF91CF911F910F9108958F9285
:104C40009F92BF92CF92DF92FF920F931F93CF93C9
:104C5000DF93009709F4DAC06115710509F4D6C035
:104C60002091493F222309F4C0C0CAEAD9E3BFC05A
:104C70008B014C010E94D211B82E0E945212D82EE4
:104C80000E942D11C82E8D2D90E08B0D911D8C0D45
:104C9000911D892B71F4F401E35BFD4F808181301C
:104CA00009F4B4C081E0808380E090E00F94B22BDF
:104CB000ADC0F401E35BFD4F8081823009F43EC05A
:104CC000BB2051F00E94CF11811108C061E0CE01DC
:104CD0000E94439501E003C000E001C000E0CC2049
:104CE00009F48AC00E942A11811186C063E0CE01B6
:104CF0000E94439501E080C0DD2081F0812F0E9459
:104D00003214882359F0812F0E944214811106C069
:104D100064E0610FCE010E94439501E01F5F1430F3
:104D200059F7002309F472C0E401C35BDD4F82E050
:104D3000888384EF91E00F94B22B68C00F94CE2B40
:104D4000882309F463C0BB2009F45DC00E94CF1121
:104D5000811159C00E942CA9CC2009F44FC0FF2416
:104D6000F39401C0F12C0E942A11811149C00E94C4
:104D70002CA916C0D0E0C0E0DD2069F08D2F0E9484
:104D80003214882341F08D2F0E944214811103C0F8
:104D90000E942AA9C1E0DF5FD43071F7CC23E1F093
:104DA00084EF91E00F94B22BD8018C9190E0F80140
:104DB000E80FF91F1D962D913C911E97880F991FA2
:104DC000A80FB91F11964D915C911297078561E06C
:104DD00087EF9CE315DE1AC0F401E35BFD4F808191
:104DE0008230A1F481E0808311C0C1EBDAE3FC01E1
:104DF0002081243059F43CCF10E07ECFFF24F3947F
:104E0000F110CECFB7CFC110ADCFB4CFDF91CF91DE
:104E10001F910F91FF90DF90CF90BF909F908F9048
:104E20000895009721F0FC01E35BFD4F6083089536
:104E3000CF93DF930097C1F0EC01198218820E9492
:104E4000E51C813031F482E0888389E1898391E037
:104E500006C0CE010E9491FC91E0811190E081E0BA
:104E6000992319F080E001C080E0DF91CF9108958F
:104E7000CF93892B09F44CC082E00E9465D0862F25
:104E800090E0FC013297E031F10508F043C088273B
:104E9000E95CFE4F8F4F0D94C66440E050E0BA01CC
:104EA00080E00E94F0D737C040E050E0BA0180E0D7
:104EB0000E94F0D7C82F40E050E0BA0181E00E9484
:104EC000F0D7C80F81E0C23031F180E024C040E06B
:104ED00050E0BA0180E00E94F0D7C82F40E050E0D7
:104EE000BA0181E00E94F0D7C80F40E050E0BA015B
:104EF00082E00E94F0D7C80F40E050E0BA0183E0A2
:104F00000E94F0D7C80F81E0C43029F080E003C0D0
:104F100080E001C080E0CF910895CF92DF92EF92C0
:104F2000FF92843098F4E82FF0E0EE0FFF1FEE0FB1
:104F3000FF1FE854F44CC080D180E280F3800E94CF
:104F4000C0D76C197D098E099F0903C060E070E02D
:104F5000CB01FF90EF90DF90CF900895CF93892BF6
:104F600009F453C082E00E9465D0862F90E0FC01D6
:104F70003297E031F10508F04AC08827E95BFE4F1F
:104F80008F4F0D94C66480E0C8DFAB01BC0180E0A8
:104F90000E94F0D73DC080E0C0DFAB01BC0180E0E3
:104FA0000E94F0D7C82F81E0B8DFAB01BC0181E0DF
:104FB0000E94F0D7C80F81E0C23051F180E028C0D4
:104FC00080E0ABDFAB01BC0180E00E94F0D7C82FCE
:104FD00081E0A3DFAB01BC0181E00E94F0D7C80FE4
:104FE00082E09BDFAB01BC0182E00E94F0D7C80FDA
:104FF00083E093DFAB01BC0183E00E94F0D7C80FD0
:1050000081E0C43029F080E003C080E001C080E08E
:10501000CF91089590E0FC013397EE30F10508F050
:10502000A7C08827E95AFE4F8F4F0D94C664E8E267
:10503000F4E5868D978DA0A1B1A1428D538D648D2D
:10504000758D841B950BA60BB70B86399105A105B1
:10505000B10508F48FC046A157A160A571A582A132
:1050600093A1A4A1B5A1481B590B6A0B7B0B81E04E
:10507000463951056105710508F483C080E0089543
:10508000E8E2F4E582A193A1A4A1B5A1468D578DD4
:1050900060A171A1841B950BA60BB70B86399105F6
:1050A000A105B10508F468C046A557A560A971A976
:1050B00082A593A5A4A5B5A5481B590B6A0B7B0B2C
:1050C00081E0463951056105710508F45AC080E058
:1050D0000895E8E2F4E582A193A1A4A1B5A1468DCB
:1050E000578D60A171A1841B950BA60BB70B863958
:1050F0009105A105B10508F441C042A953A964A9CD
:1051000075A986A597A5A0A9B1A9481B590B6A0B3B
:105110007B0B81E0463951056105710590F180E016
:105120000895E8E2F4E5868D978DA0A1B1A1428DA6
:10513000538D648D758D841B950BA60BB70B86392B
:105140009105A105B105E0F042A553A564A575A59B
:1051500086A197A1A0A5B1A5481B590B6A0B7B0B93
:1051600081E0463951056105710558F080E00895E8
:1051700080E0089581E0089581E0089581E0089538
:1051800081E00895CF9382E10E9465D0C1E0672B52
:10519000682B692B09F4C0E082E00E9465D088E0AA
:1051A000E2E6F4E5DF01982F1D929A95E9F7EAE629
:1051B000F4E5DF011D928A95E9F7862F90E0FC0166
:1051C0003197E231F10508F0EFC08827EB59FE4F27
:1051D0008F4F0D94C664EC2FF0E0E153FF4D8081BA
:1051E0008560E8E2F4E582AF83AFE8C0EC2FF0E041
:1051F000E153FF4D8081E8E2F4E582AF83AF83E0C5
:1052000080936A5480936B54D9C0862F03DFEC2FB0
:10521000F0E0E153FF4D908121E0811101C020E0D9
:10522000822F892BE8E2F4E582AF84AF83E080939C
:105230006A5480936C54892F816083AF85AFBEC060
:10524000EC2FF0E0E153FF4D8081E8E2F4E582AF1E
:1052500084AF93E090936A5490936C5483AF85AF7E
:1052600082E080936B5480936D54A8C0862FD2DE69
:10527000EC2FF0E0E153FF4D208191E0811101C05E
:1052800090E0892F822BE8E2F4E582AF85AF93E0CE
:1052900090936A5490936D5483AF86AF82E080936D
:1052A0006B5480936E54822F816084AF87AF86C029
:1052B000EC2FF0E0E153FF4D8081E8E2F4E582AFAE
:1052C00086AF93E090936A5490936E5483AF87AF08
:1052D00092E090936B5490936F5484AF8093685492
:1052E00094E090936C549093705485AF809369547C
:1052F00085E080936D548093715460C0862F8ADE60
:1053000091E0811101C090E0892F8F70E8E2F4E50F
:1053100082AF86AF93E090936A5490936E5483AFBC
:1053200087AF82E080936B5480936F5481E084AFA9
:105330008093685495AF9093695440C0E8E2F4E5D7
:1053400085E082AF84AF87E083AF85AF37C0862F1B
:1053500061DE91E0811101C090E0EC2FF0E0E153BB
:10536000FF4D8081892BE8E2F4E582AF85AF83E0D1
:1053700080936A5480936D5491E093AF96AF84AF5D
:1053800087AF1CC0EC2FF0E0E153FF4D80818160BE
:10539000E8E2F4E582AF84AF83AF85AF81E080932C
:1053A0006B5480936D540AC0EC2FF0E0E153FF4D35
:1053B00080818560E8E2F4E582AF83AF809162543A
:1053C00084700F94381581E0CF9108951F93CF9387
:1053D000DF930097E9F1EC011AAA1BAA0E9421179A
:1053E00087E00E9465D0162F84E00E9465D0862F4A
:1053F000612F0F940F1689E10E9465D0613071050D
:105400008105910521F481E00F949F2903C080E07C
:105410000F949F290E94D11C813031F4CE010E944B
:105420008A1C0E94222004C0CE010E94201CAADEF9
:105430000F94302C0F941B15CE010E94F0200F9476
:10544000BB2A0E945E100E94AF110E942E12198288
:10545000DF91CF911F910895CF93DF93009791F043
:10546000FC012081243071F4EC010E94D21FCE0196
:10547000ADDF0F942C291092443F63E0CE010E94CF
:10548000AC141982DF91CF910895882321F081E037
:105490008093493F08951092493F08958091493F74
:1054A0000895AF92BF92CF92DF92EF92FF920F9347
:1054B0001F93CF93DF93DC01009709F45AC0411585
:1054C000510509F458C02115310509F456C0FA01F7
:1054D000C081D0E0F901008110E06115710561F033
:1054E000FC017C01E60EF71E9191C90FD11D0C0F36
:1054F0001D1FEE16FF06C1F7F9017B016D01DA01F0
:10550000CC930083F601E60FF71F8CE280838BE1DA
:1055100081835B01A2E0AA0EB11CAC0CBD1C8C2FD8
:1055200082958F700F94A335F50180835701F3E0C6
:10553000AF0EB11CAC0CBD1C8C2F8F700F94A3351B
:10554000D5018C93E7012496CC0DDD1D802F82952B
:105550008F700F94A3358883D7011596E601CA0F83
:10556000DB1F802F8F700F94A3358883C7010696A9
:1055700005C0CB0103C0CB0101C0CB01DF91CF91AE
:105580001F910F91FF90EF90DF90CF90BF90AF9061
:1055900008953F924F925F926F927F928F929F9267
:1055A000AF92BF92CF92DF92EF92FF920F931F9331
:1055B000CF93DF93CDB7DEB76397CDBFDEBF7C015E
:1055C0006B013A01290189E10E9465D0B62E82E083
:1055D0000E9465D0162FE114F10409F446C1C114EC
:1055E000D10409F444C16B3008F449C16114710459
:1055F00009F43FC14114510409F43DC1FE01329642
:10560000CE014296C192D1922BE0C20ED11CE81776
:10561000F907C1F78DE0D701D6968C93D69782E033
:1056200090E0D4968D939C93D5978AE0D7968C93EF
:10563000F701F896EA8BFB8B41E0BE016F5F7F4F6D
:10564000CF010E94DE172981D701D4968D919C91BC
:10565000D597820F911D9C012F5F3F4FD4962D93BC
:105660003C93D597F701E80FF91F2CE226ABB1E088
:10567000BB1590F5B12C0F2EFCE2AF2EF02D61C0C2
:10568000EB2DF0E0EE0FFF1F81E090E08C0F9D1FEF
:10569000E80FF91FC180D280D701D4968D919C91DB
:1056A000D597C696F601418550E0B6018E0D9F1D37
:1056B0000F94C566D60119962C91F70184A995A976
:1056C000820F911D9C012F5F3F4F24AB35ABE80F3C
:1056D000F91FA6AAB39405C0B12C0F2EFCE2AF2E81
:1056E000F02D0F942D2CB81658F230C0EB2DF0E0B1
:1056F000EE0FFF1F81E090E08C0F9D1FE80FF91F58
:10570000C180D280D701D4968D919C91D597C696B1
:10571000F601418550E0B6018E0D9F1D0F94C566C0
:10572000D60119962C91F70184A995A9820F911D94
:105730009C012F5F3F4F24AB35ABE80FF91FA6AAA2
:10574000B3940F942D2C8695B81680F21B3008F474
:1057500066C01C3028F01E3028F01051133010F0B5
:1057600010E001C011E00F2EF4EB8F2EF1E29F2E1E
:10577000F02D5701F6E3AF0EB11C0F2EFCE23F2EC9
:10578000F02DC12ED12CC601880F991FC80ED91E2D
:10579000CC0CDD1CCC0CDD1CC60CD71CD6011A961B
:1057A0008C911F928F939F928F92F70184A995A954
:1057B000C6968E0D9F1D9F938F930F94F366F501F0
:1057C00001900020E9F73197EA19FB09D701D49637
:1057D000ED93FC93D597CF01C696F601418550E035
:1057E000B6018E0D9F1D0F94C566D60119962C919A
:1057F000F70184A995A9820F911D9C012F5F3F4F4E
:1058000024AB35ABE80FF91F36AA1F5F0F900F903E
:105810000F900F900F900F90123008F4B2CF01301C
:10582000D9F4D701D4968D919C91D597C6968201D3
:1058300001501F4FF801408150E0B2018E0D9F1DB5
:105840000F94C566D8012C91F70184A995A9820F00
:10585000911D84AB95AB18C0D701D496ED91FC9106
:10586000D597EE0DFF1D16AA0FC080E02EC080E078
:105870002CC080E02AC080E028C080E026C041140F
:10588000510409F0BBCEF9CFA7014D5A5D4FF70186
:10589000E75AFD4F8081FA01808397012C5A3D4FD2
:1058A00037968081D9018C93F70164A975A962505C
:1058B00071098A899B89F5DD0296D701D4968D936B
:1058C0009C93D59781E0D2968C936396CDBFDEBF33
:1058D000DF91CF911F910F91FF90EF90DF90CF90CC
:1058E000BF90AF909F908F907F906F905F904F9000
:1058F0003F9008952F923F924F925F926F927F92C6
:105900008F929F92AF92BF92CF92DF92EF92FF92CF
:105910000F93CF93DF93CDB7DEB76097CDBFDEBFD8
:10592000009709F46EC06115710509F46AC09B0106
:10593000FE013196DE01519621933193255F3F4F51
:10594000EA17FB07C9F76A017B011C01B12C12C0E1
:10595000EB2DF0E0EE0FFF1F81E090E08C0F9D1F1C
:10596000E80FF91F808191810E943C17882309F478
:1059700048C0B3940F942D2CB81650F30F94882977
:105980004B015C010F9471292B013C018FEE95E4D2
:105990000E9402DE082F81110BC09EE1890E911C2E
:1059A000A11CB11C84149504A604B70450F115C0C1
:1059B00040E050E069E473E480E30E94F91C2FEEBC
:1059C00035E4A601B701C101E4DD41EF56E469E425
:1059D00073E482E30E94F91C0EC000E02FEE35E470
:1059E000A601B701C101D5DD40E050E069E473E4F0
:1059F00082E30E94F91C8FEE95E40E94FCDD0E9478
:105A000021176096CDBFDEBFDF91CF910F91FF9040
:105A1000EF90DF90CF90BF90AF909F908F907F904E
:105A20006F905F904F903F902F900895009789F06E
:105A30006115710571F04115510559F021153105B8
:105A400041F0FC011082FB011082FA011082F90181
:105A5000108208952F923F924F925F926F927F92A1
:105A60008F929F92AF92BF92CF92DF92EF92FF926E
:105A70000F931F93CF93DF93CDB7DEB72597CDBF9D
:105A8000DEBF009709F461C04115510509F45FC0FC
:105A90002115310509F45DC0613BE4E07E0708F49F
:105AA0005AC02B01E0EB4E1AE4E05E0A612C712C27
:105AB000E2E04E165104610471040CF454C02C83CE
:105AC0003D831A018C01C12CD12C7601C3944B016A
:105AD000A12CB12CB501A4014C195D096E097F09F7
:105AE000C8010F94EA5C9E012F5F3F4F41E050E0F8
:105AF000BE016D5F7F4FC8010F949E5981112DC06B
:105B00008B818B3191F18FEFC81AD80AE80AF80A15
:105B1000C414D504E604F704ECF225C089819A8107
:105B20000497E8F0B10180ED94E40F949539982F33
:105B3000882341F16C817D8182ED94E40F94953945
:105B400091E081111FC090E01DC090E01BC090E06B
:105B500019C090E017C090E015C090E013C090E02D
:105B600011C090E00FC090E00DC09E012F5F3F4F2D
:105B700044E050E060ED74E4C8010F949E5988231E
:105B800069F2EFCF892F2596CDBFDEBFDF91CF9190
:105B90001F910F91FF90EF90DF90CF90BF90AF904B
:105BA0009F908F907F906F905F904F903F902F903D
:105BB00008950097A9F061157105B1F0FC019C01F1
:105BC000260F371F60E070E0CB0141914D3021F48A
:105BD0006F5F7F4F8F4F9F4F2E173F07B1F708958D
:105BE00060E070E0CB01089560E070E0CB010895C3
:105BF0002F923F924F925F926F927F928F929F92DD
:105C0000AF92BF92CF92DF92EF92FF920F931F93CA
:105C1000CF93DF9300D01F92CDB7DEB7009709F482
:105C200055C00115110509F453C0613B7440C0F41F
:105C3000F801108211821282138280E04CC0098127
:105C40001A81B801C101B5DF460E571E681E791EC4
:105C50000815190500F1C00ED11EE11CF11C0BC086
:105C60000B831C8349011A015C01C12CD12C7601E4
:105C7000412C512C3201B701A601C5010F94EA5CF9
:105C80009E012F5F3F4FA401B101C5010F949E59A2
:105C90008823A9F21FC0F6E24F1651046104710473
:105CA00040F4EB81FC81108211821282138281E028
:105CB00012C0F5E24F1A510861087108EB81FC81AE
:105CC000408251826282738281E005C080E003C01D
:105CD00080E001C080E02496CDBFDEBFDF91CF9190
:105CE0001F910F91FF90EF90DF90CF90BF90AF90FA
:105CF0009F908F907F906F905F904F903F902F90EC
:105D00000895009741F0FC01EB5AFD4F60817181CD
:105D100082819381089560E070E0CB01089500973F
:105D200039F0FC01EB5AFD4F10821182128213826E
:105D30000895CF93DF93009781F12091493F21117E
:105D40002CC0EC010F940726882339F1CE010E9464
:105D5000A7990F94E0250F941D111F928F9388EB44
:105D600091E29F938F93C0EDD4E4DF93CF930F9490
:105D7000F36609900020E9F72197AE01405D544495
:105D800020E060ED74E48AEA99E30F948B310F9080
:105D90000F900F900F900F900F90DF91CF9108957B
:105DA0002115310551F0505861097109F9014083FD
:105DB00051836283738381E0089580E008950097A2
:105DC00019F0FC01848D089580E008954F925F9250
:105DD0006F927F928F929F92AF92BF92EF92FF92BB
:105DE0000F931F93CF93DF931F92CDB7DEB7E114CC
:105DF000F10409F465C0480159012A013B01182F3B
:105E0000C7010E941517143031F484E10E9441D07B
:105E10009B01AC0105C085E10E9441D09B01AC0112
:105E20002115310541055105F9F084189508A6089A
:105E3000B708880C991CAA1CBB1CD501C401880F8B
:105E4000991FAA1FBB1F880F991FAA1FBB1FBC0148
:105E5000CD01680D791D8A1D9B1D0F94AA64822EA9
:105E6000932EA42EB52E0EC088248A940F2EF0EE09
:105E70009F2EF02D0F2EF5EFAF2EF02D0F2EF5E00B
:105E8000BF2EF02D082D192D2A2D3B2D4BE0BE01E4
:105E90006F5F7F4FC7010F940F39F701019000200A
:105EA000E9F73197EE19FF09D7011996EC93199785
:105EB00081E01B968C93682D792D8A2D9B2D04C033
:105EC00060E070E080E090E00F90DF91CF911F9153
:105ED0000F91FF90EF90BF90AF909F908F907F9029
:105EE0006F905F904F9008952F923F924F925F92E4
:105EF0006F927F928F929F92AF92BF92CF92DF92DA
:105F0000EF92FF920F931F93CF93DF93CDB7DEB73E
:105F10002A97CDBFDEBFC5016115710509F402C125
:105F20004115510509F400C1E114F10409F4FEC062
:105F3000802E912EA22EB32E25EB82169104A10461
:105F4000B10438F00F2EF4EB8F2E912CA12CB12C34
:105F5000F02D8B839C83CD82DE82EF82F88649838D
:105F60005A838B01FB01E453FD4F80819181A28113
:105F7000B381892B8A2B8B2B81F53497808191817A
:105F8000A281B38180324EE49407A105B1052CF1C2
:105F9000349680839183A283B383BF93AF939F93FF
:105FA0008F9383ED91E29F938F9380ED94E49F9381
:105FB0008F930F94F366E0EDF4E401900020E9F78D
:105FC0003197AF01405D544420E060ED74E48AEA0B
:105FD00099E30F948B31CDBFDEBFD801CD90DD901A
:105FE000ED90FC90B0E8DB1AE108F108F801C082FE
:105FF000D182E282F38281E08093D132F2E08F1687
:106000009104A104B10408F46FC0F80161ED72E3DA
:1060100021E0821A20EC920A880C991C880C991CA9
:106020001801280C391C4601570100E010E09801C6
:1060300069877A8744815581668177812A013B018E
:1060400080E8581A61087108448255826682778216
:106050004191519161917191441A550A660A770AEA
:10606000141415041604170434F481E0A985BA85C4
:1060700011968C9304C0A985BA8511961C92A985A6
:10608000BA8511965C901197CD01019689879A8700
:106090009C91591691F0D801AA0FBB1FAA0FBB1FE4
:1060A00089819A81A80FB91F4D935D936D937C935D
:1060B00013970F5F1F4F2F4F3F4F408151816281D8
:1060C0007381C416D506E606F70614F46A017B014F
:1060D000481559056A057B0514F44A015B01E21570
:1060E000F30509F0A7CF05C04601570100E010E015
:1060F0009801AF81B8850D931D932D933C93139711
:10610000ED81FE81309721F080829182A282B3825C
:10611000EB81FC81309761F0C082D182E282F38210
:1061200081E007C080E005C080E003C080E001C0DE
:1061300081E02A96CDBFDEBFDF91CF911F910F91F5
:10614000FF90EF90DF90CF90BF90AF909F908F9097
:106150007F906F905F904F903F902F9008958F9217
:106160009F92AF92BF92CF92DF92EF92FF920F93E6
:106170001F93FC01892BA1F16115710599F1008133
:1061800011812281338184819581A681B78108178D
:1061900019072A073B0744F5C084D184E284F384BD
:1061A000C816D906EA06FB060CF584849584A684F5
:1061B000B784C814D904EA04FB04D4F488159905FB
:1061C000AA05BB05BCF40C151D052E053F0524F4DE
:1061D00081E0FB0180830FC0FB01108281E00BC0D6
:1061E00080E009C080E007C080E005C080E003C017
:1061F00080E001C080E01F910F91FF90EF90DF9051
:10620000CF90BF90AF909F908F9008953F924F9204
:106210005F926F927F928F929F92AF92BF92CF9236
:10622000DF92EF92FF920F931F93CF93DF9300972C
:1062300009F448C02115310509F446C04430510520
:106240006105710508F442C06A017B01E4E0CE1AE1
:10625000D108E108F108E1F159018C01912C312CB0
:10626000812C412C512C3201E501C90DD11DBE01FB
:10627000C201880F991F880F991F800F911F6FDF30
:10628000882379F08881882311F0839401C03394A6
:1062900083E0480E511C611C711C9394E2E0E915E7
:1062A00050F08FEF481A580A680A780A4C145D04B7
:1062B0006E047F04C8F2882069F081E0332059F031
:1062C00080E009C080E007C080E005C080E003C036
:1062D00081E001C081E0DF91CF911F910F91FF908C
:1062E000EF90DF90CF90BF90AF909F908F907F9076
:1062F0006F905F904F903F9008952F923F924F92F2
:106300005F926F927F928F929F92AF92BF92CF9245
:10631000DF92EF92FF920F931F93CF93DF93CDB74E
:10632000DEB76B97CDBFDEBF782ED92E662E798B68
:1063300019821A821B821C821D821E821F8218866D
:1063400019861A861B861C861D861E861F86188A3D
:1063500082E00E9465D06B3008F4BBC00F94662DBC
:10636000882309F4CEC00F94552D8091133D8230BF
:1063700009F0B1C083EB90E40F94985CACC08F8AB5
:10638000988E530162010F2EFAEFEF2EFFE2FF2EDF
:10639000F02D04EB10E020E030E041E050E3B401E8
:1063A000832DA2DD882331F14091FA2F5091FB2FEC
:1063B0006091FC2F7091FD2F2EEF3FE281E090E382
:1063C00025DF882361F08091FE2F90E0A0E0B0E00F
:1063D000EF89F88D80839183A283B38314C08EEFFD
:1063E00090E0A0E0B0E0EF89F88D80839183A283F4
:1063F000B38309C08FEF90E0A0E0B0E0F4018083A8
:106400009183A283B3833394F0E38F1AFDEF9F0A45
:1064100084E0480E511C94E0690E711CA6E03A120B
:10642000AECF298C3A8C6B8C862C99886894552435
:1064300052F80F2EF5E44F2EF02D0F2EF2E5DF2E41
:10644000F02D0F2EFCE4CF2EF02DAB88BC886D888C
:106450007E88898A9A8AF301019111912191319163
:106460003F01D5014D915D916D917D915D0174016B
:10647000852DACDC65317105810591051CF4F401B5
:1064800042861AC0F10180819181A281B381009777
:10649000A105B10529F4A989BA891A96CC920CC034
:1064A0000197A105B10521F4E989FA89D28604C0D2
:1064B000A989BA891A964C925394BCE08B0E911C10
:1064C000E0E32E1AEDEF3E0AF6E05F12C2CF81E064
:1064D00018C080E016C0272C3D2CCE0101968B8B76
:1064E0009C8BDE011996AD8BBE8B2C01872C9D2CCD
:1064F0006894772472F8298E3A8E372C6B8E3D0182
:106500003ECF6B96CDBFDEBFDF91CF911F910F9134
:10651000FF90EF90DF90CF90BF90AF909F908F90C3
:106520007F906F905F904F903F902F9008951F93B2
:10653000CF93DF93009709F4FCC0EC01888184308D
:1065400089F128F4813069F08230E9F0F2C08930B5
:1065500009F4B1C08A3009F4C5C0883009F0E9C037
:106560001EC08B81813009F0E4C08C81813009F03C
:10657000E0C00F944E29CE010E94E62962E0CE01D0
:106580000E94AC14D6C080914A49813029F463E05E
:10659000CE010E94AC14CDC00E94CB1BCAC00E9489
:1065A0000651C7C0CE010E94C92189818111C1C095
:1065B00082E00E9465D06B3040F46BE479E38FECAD
:1065C0009CE30E940918182F10C00F94662D882391
:1065D000E1F06BE479E38FEC9CE30E940918182F3B
:1065E0006FED7CE388E89EE488DE113071F482E090
:1065F0000E9465D0162F8FEC9CE30E947A10612FC9
:1066000083E790E40E949C1207C08BE499E30E9408
:106610004717882309F47FC04FED5CE36BE479E30F
:10662000CE0168D978C00F940017882309F47EC082
:106630000F94CC2A63EB70E4CE010E941D250F94C9
:10664000EF1674C08981811174C0CE010E9491211E
:10665000882341F00F94CC2A63EB70E4CE010E94B2
:106660001D2567C01AAA81E08BAB63C08AA9882365
:1066700009F45FC0898181115CC0CE010E945F2155
:10668000882341F00F94CC2A63EB70E4CE010E9482
:106690001D254FC01AAA4DC00F940017882309F476
:1066A00048C00F94CC2A63EB70E4CE010E941D25F4
:1066B0000F94EF163EC0CE010E94C9216BE479E32E
:1066C0008FEC9CE30F94461B813031F08BE499E30F
:1066D0000F949B1B882369F16BE479E3CE010F943F
:1066E000C41E27C0CE010E94C921CE010E9481B4E0
:1066F0004AE953E46BE479E38FEC9CE30E9431B305
:10670000CE010E9492AD8831A1F46AE973E4CE0112
:106710000E9415B40EC0FE01E95CFD4F80818130FE
:1067200009F481CF823009F0B7CFA0CF8AA98111B7
:1067300089CFDF91CF911F910895CF930E945FD8A9
:10674000C82F88E10E9465D0C61741F061E080E063
:106750000F941D1361E081E00F941D13CF910895F4
:10676000CF930E945FD8C82F88E10E9465D0C617DA
:1067700049F061E080E00F941D1361E081E00F9427
:106780001D1308C060E080E00F941D1360E081E0FD
:106790000F941D13CF910895CF93DF93EC01809157
:1067A000493F882319F0EAEAF9E302C0E1EBFAE392
:1067B000209729F18BE7888388E689839CE29A8376
:1067C00082E68B839C838CE68D838DE78E831F828C
:1067D00021E047E050E0BE01CF010F948B310E94D1
:1067E00074C8873061F48091493F811108C021E06D
:1067F00047E050E0BE018AEA99E30F948B31DF91C4
:10680000CF9108958091143D0895CF92DF92FF9229
:106810000F931F93CF93DF931F921F92CDB7DEB7D5
:106820009FEF980F923008F045C09091143D992346
:1068300009F443C0813019F00CE61FE302C001EBFC
:106840001AE3F82E81E6898384E78A8321E042E017
:1068500050E0BE016F5F7F4FC8010F948B310F94E2
:10686000F6290F940D2A643F714081059105C8F304
:10687000C8010E94C6A60F94F6290F940D2A643F02
:10688000714081059105C8F38F2D0E94B1D86C012C
:106890008F2D0E94B1D8FC0101900020E9F73197BB
:1068A000AF01481B590B41F0B601C8010E9436A741
:1068B00091E003C090E001C090E0892F0F900F900D
:1068C000DF91CF911F910F91FF90DF90CF900895AE
:1068D000009791F0FC01E15AFD4F108275961082ED
:1068E000749780599D4FDC0111921192119211926F
:1068F0001D92E817F907C1F708950F931F93CF93DF
:10690000DF931F92CDB7DEB7009709F4CAC08C01A0
:1069100081E0D8018C9311961C92119712961C92CB
:10692000129713961C92139714961C92149715960F
:106930001C921597169682E1E0E2F4E201900D9226
:106940008A95E1F7C80148960E948CD5F801808DA0
:106950008783818D8087828D8187838D8287CE0119
:1069600001960E94ADD589818C3438F4D8015C96AB
:106970001C925C975D961C9211C08C3431F482E0BD
:10698000F801848F81E0858F09C08D3439F482E06D
:10699000D8015C968C935C975D961C9280E00E9477
:1069A00041D0673EB3E07B0781059105BCF49F931E
:1069B0008F937F936F938EEE91E29F938F93C80195
:1069C000C6969F938F930F94F366F80186A9808BE8
:1069D00087A9818B80AD828BCDBFDEBFD8015E964B
:1069E0001C925E975F961C925F97D2961C92D297EC
:1069F000D3961C92F801EA5CFD4F1082319610820A
:106A000031961082319681E0808331961082118216
:106A100012821382349681E090E0A0E0B0E080839F
:106A20009183A283B383349610823196D8018C91DE
:106A30008083E751F24086E0DF011D928A95E9F7F5
:106A4000E85EFD4F108211823296108211823296DA
:106A50001082118232961082118232961082319603
:106A600010823296108231961082319610823196C1
:106A700010823196108231961082319610821182E6
:106A800012821382349610823196108231961082CF
:106A900031961082319688E690E180839183C80117
:106AA00017DF0F90DF91CF911F910F910895EF9213
:106AB000FF920F931F93CF93DF93009709F43FC08A
:106AC000FC01DC01A15ABD4F1C9255961C92EC01B1
:106AD000C05ADD4F84E190E0A0E0B0E08883998364
:106AE000AA83BB8360961882289788839983AA8398
:106AF000BB83DF01AE58BD4F1C92E0A4F1A402A5F8
:106B000013A5D801C7014496A11DB11D2497888300
:106B10009983AA83BB832D961882259788839983AE
:106B2000AA83BB83ED58FD4F108222E830E040E09D
:106B300050E062E870E080E090E00F94BE2DDF91BD
:106B4000CF911F910F91FF90EF900895EF92FF92D8
:106B50000F931F93CF93DF93CDB7DEB72797CDBFAA
:106B6000DEBF7C01FB0184818D8385818E838681DC
:106B70008F8380819181A281B38189839A83AB8342
:106B8000BC83870180EAE81688E0F80629F460E112
:106B900083E00F94F64314C080EBE81688E0F80613
:106BA00029F460E283E00F94F64313C080EAE8160C
:106BB00089E0F80629F460E184E00F94F64312C0FE
:106BC000003B89E0180729F460E284E00F94F64363
:106BD00012C0003A8AE0180729F460E185E00F94BA
:106BE000F64310C0003B8AE0180729F460E285E014
:106BF0000F94F64307C0003A1B4021F460E186E0A1
:106C00000F94F643BE016F5F7F4FC7010E9464710E
:106C10002796CDBFDEBFDF91CF911F910F91FF90DF
:106C2000EF900895DC01892BE1F0E62FE695E695DB
:106C3000E69580E2E89FF0011124FA5F8085677095
:106C400021E030E002C0220F331F6A95E2F72823CB
:106C500081E009F480E08C9311968C931197129641
:106C60001C920895CF93DF93009709F4A5C06D326D
:106C700009F0A4C03091A80621E0432F407235FFEF
:106C800020E0FC0120833181231709F499C0EC0135
:106C9000442309F46BC0311169C00F948F2500970C
:106CA000F9F40E944E2A811119C086E0E4EFF1E266
:106CB000A0EDB4E401900D928A95E1F7E0EDF4E4E3
:106CC00001900020E9F73197AF01405D544421E085
:106CD00060ED74E48AEA99E30F948B311A8268C0FC
:106CE000803D974008F50E944E2A811119C086E028
:106CF000EAEFF1E2A0EDB4E401900D928A95E1F79C
:106D0000E0EDF4E401900020E9F73197AF01405D38
:106D1000544421E060ED74E48AEA99E30F948B31E6
:106D20000F94A3251A8244C081E08A830F94A3257F
:106D30000E944E2A81113CC086E0E0E0F2E2A0ED24
:106D4000B4E401900D928A95E1F7E0EDF4E401904E
:106D50000020E9F73197AF01405D544421E060ED38
:106D600074E48AEA99E30F948B3122C01A8281E09D
:106D700090E00F94B6250E944E2A811119C086E03A
:106D8000E6E0F2E2A0EDB4E401900D928A95E1F71D
:106D9000E0EDF4E401900020E9F73197AF01405DA8
:106DA000544421E060ED74E48AEA99E30F948B3156
:106DB000888189838A8105C080E003C080E001C0AA
:106DC00080E0DF91CF9108958EEB98E40C94CFE5AD
:106DD00008950E944E2A811117C062E575E48AEA7F
:106DE00099E30F9437318091D445813029F542E5FC
:106DF00055E464E575E48AEA99E30E94E1CD82E511
:106E000095E40D942831089562E575E48AEA99E3E2
:106E10000E9415A48091D445813071F427EF3CE3A2
:106E200042E555E464E575E48AEA99E30E9406A424
:106E300082E595E40D94283108950E949A94882360
:106E400041F0E0DC811105C084E292E40C94DA2484
:106E500008950E944E2A81112EC062E472E481EBF3
:106E60009AE30E9415A48091C442813021F50E94CA
:106E70004E2A811112C062E48091AA399091AB39F7
:106E80000E944970409142425091434221E064E4A3
:106E900072E48AEA99E30F948B3127EF3CE342E4F2
:106EA00052E464E472E481EB9AE30E9406A482E473
:106EB00092E40D9428310895CF92DF92EF92FF92E1
:106EC0000F931F93CF93DF930E944E2A882319F0CC
:106ED0000AEA19E302C001EB1AE383E392E40E9499
:106EE00041A6882349F08EDC811106C063E372E479
:106EF000C8010E94C0248BC28091414281508230DF
:106F000008F057C10E94C3A6811104C07BDC88230E
:106F100009F414C36EEE70E48CE69FE30E94B8A5FA
:106F200080911F42813009F072C2E090EE40F090F3
:106F3000EF4082E0E816F10408F400C3809141427A
:106F4000813039F48091F3408F7D8C3409F0CBC0CF
:106F50000AC08091F340843209F0C5C08091F440AA
:106F6000833509F0C0C00E944E2A811156C087E0C7
:106F7000ECE0F2E2A0EDB4E401900D928A95E1F725
:106F8000E0EDF4E401900020E9F73197AF01405DB6
:106F9000544420E060ED74E48AEA99E30F948B3165
:106FA0001092F0401092F140E114F104A1F080E061
:106FB00090E0CEEED0E4FC01E251FF4B65818AEA1D
:106FC00099E30F9417328A819B8101968A839B8370
:106FD0008E159F0580F30F94DE2A1F928F9383E115
:106FE00092E29F938F93C0EDD4E4DF93CF930F94FD
:106FF000F36609900020E9F72197AE01405D544403
:1070000021E060ED74E48AEA99E30F948B310F90EC
:107010000F900F900F900F900F900F94DE2A8823FF
:1070200071F181E00E940890813069F48EEE90E465
:107030000E940EA68EEE90E40E9420A60F94BB2A1A
:107040000E94B4A802C00E9415A9E5E8F3E480817B
:1070500090E0DC01AB57BC4B25853685880F991F26
:10706000FC01EB57FC4B418152811F960C9161E072
:1070700087EF9CE30E9400250F94E52B93C0E092DC
:107080002242F09223420F94DE2A682FC8010E9408
:10709000E6920E944E2A811185C00F94DE2A1F922B
:1070A0008F93809141421F928F9389E192E29F9347
:1070B0008F93C0EDD4E4DF93CF930F94F3660990E0
:1070C0000020E9F72197AE01405D544421E060EDD6
:1070D00074E48AEA99E30F948B31EDB7FEB73896E2
:1070E000EDBFFEBF5FC00E944E2A811157C0809144
:1070F0004142823049F48091F340843229F48091F6
:10710000F440873409F44AC086E0E7E3F2E2A0EDF8
:10711000B4E401900D928A95E1F7E0EDF4E401907A
:107120000020E9F73197AF01405D544420E060ED65
:1071300074E48AEA99E30F948B31EEEEF0E4128264
:10714000138280819181892BA9F080E090E0EF018A
:10715000FC01E251FF4B65818AEA99E30F941732F3
:107160008A819B8101968A839B832881398182173A
:10717000930770F3E0EDF4E480E290E08083918384
:1071800001900020E9F73197AF01405D544421E0C0
:1071900060ED74E48AEA99E30F948B318EEE90E40B
:1071A0000E9420A68EEE90E40E940EA60F94BB2AA9
:1071B0002EC10F9411266B017C016EEE70E48CE6FB
:1071C0009FE30E943CA580911F42813039F0F5E693
:1071D000CF16D104E104F10408F419C10F94282654
:1071E00080911F42813079F48EEE90E40E9491A646
:1071F000882321F0E0902142F12C40C0E090EE4045
:10720000F090EF403BC00F2EFEEEEF2EF0E4FF2E8D
:10721000F02DF70181818F9380818F938DE392E22E
:107220009F938F93C0EDD4E4DF93CF930F94F366D5
:1072300009900020E9F72197AE01405D544421E018
:1072400060ED74E48AEA99E30F948B311092214245
:107250000F900F900F900F900F900F90F70180817B
:1072600091818739910530F086E990E08093EE4076
:107270009093EF40E090EE40F090EF400E944E2A55
:1072800081115DC0FF92EF928CE592E29F938F9304
:10729000C0EDD4E4DF93CF930F94F3660990002000
:1072A000E9F72197AE01405D544420E060ED74E4BD
:1072B0008AEA99E30F948B311092F0401092F140DA
:1072C0000F900F900F900F900F900F90E114F1041A
:1072D000A1F080E090E0CEEED0E4FC01E251FF4B63
:1072E00065818AEA99E30F9417328A819B8101961E
:1072F0008A839B838E159F0580F30F94DE2A1F924D
:107300008F9383E192E29F938F93C0EDD4E4DF9358
:10731000CF930F94F36609900020E9F72197AE010F
:10732000405D544421E060ED74E48AEA99E30F94EF
:107330008B310F900F900F900F900F900F900F9434
:10734000DE2A882371F181E00E940890813069F47F
:107350008EEE90E40E940EA68EEE90E40E9420A68F
:107360000F94BB2A0E94B4A802C00E9415A9E5E8A8
:10737000F3E4808190E0DC01AB57BC4B258536857A
:10738000880F991FFC01EB57FC4B418152811F96DE
:107390000C9161E087EF9CE30E9400250F94E52BA0
:1073A00030C0E0922242F09223420F94DE2A682FEE
:1073B000C8010E94E6920E944E2A811122C00F94B9
:1073C000DE2A1F928F9389E692E29F938F93C0EDFE
:1073D000D4E4DF93CF930F94F36609900020E9F78C
:1073E0002197AE01405D544421E060ED74E48AEAE7
:1073F00099E30F948B310F900F900F900F900F9097
:107400000F908EEE90E40E940EA60F94BB2A0F946C
:107410005A26693C71058105910508F48FC00F94C7
:1074200071260E944E2A81114AC08AE0EDE7F2E2FD
:10743000A0EDB4E401900D928A95E1F7E0EDF4E45B
:1074400001900020E9F73197AF01405D544420E0FE
:1074500060ED74E48AEA99E30F948B31EEEEF0E488
:107460001282138280819181892BA9F080E090E0C3
:10747000EF01FC01E251FF4B65818AEA99E30F9429
:1074800017328A819B8101968A839B832881398167
:107490008217930770F3E0EDF4E480E290E08083DC
:1074A000918301900020E9F73197AF01405D54448A
:1074B00021E060ED74E48AEA99E30F948B3183EF65
:1074C00090E40E949FA78823A9F1809141428111F5
:1074D0000BC0E9E4F3E481E3808382E3818383E307
:1074E000828384E3838314C0813041F4E9E4F3E4CC
:1074F00080E380838183828383830AC0E9E4F3E4A9
:1075000081E3808382E3818383E3828384E38383D3
:1075100021E044E050E069E473E48CE69FE30F94DB
:107520008B3121E044E050E069E473E48AEA99E3B6
:107530000F948B318EEE90E40E940EA6DF91CF91D6
:107540001F910F91FF90EF90DF90CF9008958F9251
:107550009F92AF92BF92CF92DF92EF920F931F93C1
:10756000CF93DF93EC0180E00E9441D04B015C019E
:10757000209709F45CC11F8EFE01E05BFD4F108275
:10758000CE010E94A11F882309F451C16E0186E338
:10759000C80ED11CBE01615E7F4FC6010F94BC09AD
:1075A0008E8F81111FC00E944E2A811119C08BE15C
:1075B000E7E8F2E2A0EDB4E401900D928A95E1F7DC
:1075C000E0EDF4E401900020E9F73197AF01405D70
:1075D000544421E060ED74E48AEA99E30F948B311E
:1075E00081E08F8F6CE777E4C6010F94290FFE01CD
:1075F000E15BFD4F80838CE797E40E9429D78823C5
:10760000A1F181E0FE01E05BFD4F80838CE797E410
:107610000E94C6D60E944E2A811127C0FE01E05B5F
:10762000FD4F80811F928F93319780811F928F939E
:1076300082EA92E29F938F9300ED14E41F930F93DD
:107640000F94F366F80101900020E9F73197AF013C
:10765000405D544421E0B8018AEA99E30F948B31EC
:10766000ADB7BEB71896ADBFBEBF8F8D813039F0B4
:10767000FE01E05BFD4F8081813009F05CC00E941B
:107680004E2A811119C08CE1E5EBF2E2A0EDB4E4E1
:1076900001900D928A95E1F7E0EDF4E4019000206D
:1076A000E9F73197AF01405D544421E060ED74E4A7
:1076B0008AEA99E30F948B316894EE24E2F801EDA5
:1076C00012E2A5019401BE01685E7F4FCE010696CD
:1076D0000E948E598D8340E050E0BA01CE010E9495
:1076E0008F2E8D81882309F4A2C082E00E9465D08C
:1076F000062F8BE00E9465D021E0611120E0BE01E1
:107700006C5C7F4F43EB50E4C6010E949152CE0166
:107710000E94F61B9E01265A3D4FAE01475A5D4F0F
:10772000BE016C5A7D4FCE018D5A9D4F0E94162D81
:107730000F94F4177CC08E010A5F1F4FB80183EBD2
:1077400090E40E9466588D83811139C0A50194018F
:10775000BE01685E7F4FC8010E94C8558D8340E01E
:1077600050E0BA01CE010E948F2E8D81882309F44A
:107770005EC082E00E9465D0062F8BE00E9465D03B
:1077800021E0611120E0BE016C5C7F4F43EB50E4CF
:10779000C6010E949152CE010E94F61B9E01265AFC
:1077A0003D4FAE01475A5D4FBE016C5A7D4FCE0131
:1077B0008D5A9D4F0E94162D0F94F41738C08E01DC
:1077C0000B5A1D4F0F2EF3EBAF2EF0E4BF2EF02D12
:1077D000F5016285738520E032E0A601C5010E94B3
:1077E000F82D015011096E01FDEACF1AFDEFDF0AF5
:1077F000D5011A966D917C911B979801A601C50140
:107800000E942A2DFE01E75AFD4FD6018C918083FC
:10781000C65ADD4FF80180818883D5011A964D91B3
:107820005D916D917C911D97C5010F94EA5CDF918C
:10783000CF911F910F91EF90DF90CF90BF90AF90BD
:107840009F908F9008956DE288E499E30BDA882386
:1078500009F467C080918533882309F446C00E94EB
:10786000B16384E0809326060F94CC248CE797E4E0
:107870000E9480E487EF9CE36ADE8091473F882383
:10788000F1F00E9444E2813019F0823069F017C0B3
:107890008091463F882329F08CE797E40E94E2E13B
:1078A0000EC00E94B5E10BC08091463F882329F0AD
:1078B0008CE797E40E9464E302C00E942FE31092D9
:1078C00085330F94E52B87EF9CE30E949922811169
:1078D0000F944E2987EF9CE30E94E62960913A3F7E
:1078E00087EF9CE30E94AC141CC00F94E52B0F940F
:1078F0002C2966E087EF9CE30E94AC1461E08DEFD9
:107900009CE30E9434580E94B3550F94B83A0E94E9
:10791000876381E08093853384E0809325060F940C
:10792000CC2480918533882331F00E940562811137
:10793000FCCF8091853308954F925F926F927F9232
:107940008F929F92AF92BF92CF92DF92EF92FF926F
:107950001F93CF93DF93CDB7DEB72797CDBFDEBFA1
:107960007C0110924B4910E00F2E812CFBE49F2EDE
:10797000A12CB12CF02D0F2EF0EDCF2EF4E4DF2E44
:10798000F02D0F2EF0E84F2EF5E25F2E612C712CBA
:10799000F02D111120C080E096E9A0E0B0E0F701E1
:1079A00080839183A283B3838AE0E6EDF2E2D6017D
:1079B00001900D928A95E1F7F60101900020E9F718
:1079C0003197AF01405D544421E0B6018AEA99E362
:1079D0000F948B315CC0113001F580EC92E1A0E096
:1079E000B0E0F70180839183A283B38389E0E0EE66
:1079F000F2E2D60101900D928A95E1F7F60101902D
:107A00000020E9F73197AF01405D544421E0B60111
:107A10008AEA99E30F948B313AC01230E9F4D70126
:107A20004D925D926D927C92139789E0E9EEF2E2BD
:107A3000D60101900D928A95E1F7F60101900020A0
:107A4000E9F73197AF01405D544421E0B6018AEA7D
:107A500099E30F948B311BC0F70180829182A2823F
:107A6000B38289E0E2EFF2E2D60101900D928A95AD
:107A7000E1F7F60101900020E9F73197AF01405D91
:107A8000544421E0B6018AEA99E30F948B31D7017F
:107A900014968C9114978D8315968C9115978E83DF
:107AA00016968C9116978F838D919D910D90BC9118
:107AB000A02D89839A83AB83BC8360E185E00F941A
:107AC000F643BE016F5F7F4F80EA9AE00E946471C7
:107AD0000F94582B08C08EEB98E40E94CFE58130BC
:107AE00041F00E94871B0F946B2B803A9F4098F3C4
:107AF0007AC011111DC08CE0EBEFF2E2A0EDB4E40E
:107B000001900D928A95E1F7E0EDF4E401900020F8
:107B1000E9F73197AF01405D544421E060ED74E432
:107B20008AEA99E30F948B3182E080934B4978C0C5
:107B30001130E9F48BE0E7E0F3E2A0EDB4E401906A
:107B40000D928A95E1F7E0EDF4E401900020E9F769
:107B50003197AF01405D544421E060ED74E48AEA5E
:107B600099E30F948B3181E080934B4959C01230D7
:107B7000E9F48BE0E2E1F3E2A0EDB4E401900D92D0
:107B80008A95E1F7E0EDF4E401900020E9F7319700
:107B9000AF01405D544421E060ED74E48AEA99E36A
:107BA0000F948B3183E080934B493AC08BE0EDE139
:107BB000F3E2A0EDB4E401900D928A95E1F7E0EDD7
:107BC000F4E401900020E9F73197AF01405D54449F
:107BD00021E060ED74E48AEA99E30F948B3184E04C
:107BE00080934B491DC01F5F143009F0D2CE89E04D
:107BF000E8E2F3E2A0EDB4E401900D928A95E1F79A
:107C0000E0EDF4E401900020E9F73197AF01405D29
:107C1000544421E060ED74E48AEA99E30F948B31D7
:107C20002796CDBFDEBFDF91CF911F91FF90EF90E0
:107C3000DF90CF90BF90AF909F908F907F906F908C
:107C40005F904F900895CF92DF92EF92FF920F9343
:107C50001F93CF9387EF9CE30E94BF14883009F4F1
:107C6000D6C087EF9CE30E94BF14863009F4CFC0D2
:107C70008091543F9091553F8E349C4008F4BEC093
:107C80000E9441D88111B4C0C2C00F94262C81112A
:107C90001FC00F94292C0E944E2A811119C088E11F
:107CA000E1E3F3E2A0EDB4E401900D928A95E1F7EF
:107CB000E0EDF4E401900020E9F73197AF01405D79
:107CC000544421E060ED74E48AEA99E30F948B3127
:107CD0000F94122C811129C09AC08CE1E9E4F3E2DF
:107CE000A0EDB4E401900D928A95E1F7E0EDF4E4A3
:107CF00001900020E9F73197AF01405D544421E045
:107D000060ED74E48AEA99E30F948B310F94AA240E
:107D1000C0E00F949924882331F00F94AA24CF5FF8
:107D2000CA30B9F702C0CA30A0F30F942C290E94C0
:107D3000B3550E944E2A811119C08EE0E7E5F3E2A7
:107D4000A0EDB4E401900D928A95E1F7E0EDF4E442
:107D500001900020E9F73197AF01405D544421E0E4
:107D600060ED74E48AEA99E30F948B310F94AA24AE
:107D700001E010E0C0E00F2EFDE0CF2EF1E2DF2E9B
:107D8000F02D0F2EF0EDEF2EF4E4FF2EF02D0F94DA
:107D90009924882341F10F94AA24CF5F0E944E2A90
:107DA00081111CC01F930F93DF92CF92FF92EF922D
:107DB0000F94F366F70101900020E9F73197AF01C6
:107DC000405D544421E0B7018AEA99E30F948B3176
:107DD0000F900F900F900F900F900F900F5F1F4F0D
:107DE000C33019F0D4CFC33090F20F945D100FC0A0
:107DF0000F941C2C882309F46BCF47CF89E493E4BC
:107E00000E94CC330E944E2A811180CF66CFCF9141
:107E10001F910F91FF90EF90DF90CF900895F8940D
:107E20000E94B9660F94A1430F947C130F94DD1345
:107E300060E080E00F9475140F94B83A0E94CFA4CC
:107E40000F94F9120E947EED41E060EA78E081EB48
:107E50009AE30F94ED3165E170E280EA98E00E94C8
:107E6000A635E0EAF8E083818F7C8061838382E439
:107E700092E40F94283161E084E292E40E9431A6FA
:107E800041E060EA7BE08CE69FE30F94ED316EE029
:107E900070E280EA9BE00E94A635E0EAFBE0838185
:107EA0008F7C806183838EEE90E40E940EA68EEE1E
:107EB00090E40E9420A661E083E392E40E9431A650
:107EC000109241421092484385EC92E40F9428317D
:107ED00041E060EA7AE088EC9BE30F94ED3167E0E3
:107EE00070E280EA9AE00E94A635E0EAFAE0838137
:107EF0008F7C8061838341E060EA79E08AEA99E3DC
:107F00000F94ED3160E070E280EA99E00E94A635BE
:107F1000E0EAF9E083818F7C8061838382E595E4E8
:107F20000F9428310F9434240F94A3260F945828CB
:107F30000F94F42A0F94C9260F94C42C0F940C119B
:107F40000F947F160E94D70FC0E060E08C2F0F9433
:107F50001D13CF5FC830C9F787E08093A2007894E3
:107F6000E0E2F6E082E0868384E086830E94FDCF33
:107F7000811116C00E9403D10E942DD10E947DD58F
:107F80000E941AD70E9412D80E9459D881E00E94FC
:107F900006D982E00E9406D981E08093453F27C040
:107FA0000E94F0D4882309F181E08093453F0E942C
:107FB0004E2A81111CC08DE1E5E6F3E2A0EDB4E4A8
:107FC00001900D928A95E1F7E0EDF4E40190002034
:107FD000E9F73197AF01405D544421E060ED74E46E
:107FE0008AEA99E30F948B3102C01092453F0E94B8
:107FF000A6D60F94F4170E94D0D481E00F940A28DB
:108000006DE288E499E30E9412360E94C7A86FEEE1
:1080100075E48EEB98E40E9443DE8EEB98E40E94B8
:1080200025D987EF9CE30E947D3480E00F94F815FA
:108030008CE797E40E9480E40F942D1587EF9CE372
:1080400086DA81E00E9477C880E00E9471C880E0F3
:108050000E947AC880E00E947DC80E9421170E9479
:108060009D330E94D3A48EEB98E40E9425D987E02B
:1080700090E262DC0E9444E2813029F48091463F24
:108080000E9412E825C00E9444E2823091F481E00F
:108090000E9447E28091463F882329F08CE797E4CD
:1080A0000E9464E302C00E942FE381E00E94F9E293
:1080B0000FC00E9444E2833029F480ED94E40E94D2
:1080C00029E406C00E9444E2843011F40E9450E882
:1080D00084E0809326060E948AED81E00E940534A8
:1080E00082E00E94053487EF9CE30E94E6298AEA39
:1080F00099E30E94B5B90E9413100F94A62D02E8CF
:1081000013E2C0EDD4E40E94E4366FEE75E48EEB2A
:1081100098E40E944C1687EF9CE30E94DD1587EFE0
:108120009CE30E94751587EF9CE30E94992E87EFD0
:108130009CE30E9497320E94E93685DB0E941D373E
:108140000E945C3787EF9CE30E94911B0E94B7ED71
:108150000E9474C8833031F50E94BA1F882311F140
:108160000E944E2A81111EC00F9409291F928F93DD
:108170001F930F93DF93CF930F94F366FE0101904B
:108180000020E9F73197AF01405D544421E0BE0182
:108190008AEA99E30F948B310F900F900F900F9014
:1081A0000F900F9084E59FE30E942D2465E873E40F
:1081B00087EF9CE30E94CB2565E873E487EF9CE39F
:1081C0000E941F260F9403173EDD0FB607FC9BCFBE
:1081D00080E00E94607C0E94747CFFCFEF92FF924F
:1081E0000F931F93CF93DF93009749F161157105AA
:1081F00041F14115510539F18A017B01EC010F94E0
:108200007A66F80180839183892B89F0D70120E079
:1082100030E0FE01E20FF31FE491ED932F5F3F4F3B
:10822000F801808191812817390798F302C020E076
:1082300030E0F701E20FF31F108281E005C080E01B
:1082400003C080E001C080E0DF91CF911F910F91CA
:10825000FF90EF9008950F931F93CF93DF930097B4
:10826000C9F061157105C1F041155105B9F0EA0178
:108270008B01FC0165917491C8010F947366F8013C
:1082800001900020E9F73197E01BF10BE883F983B7
:1082900081E005C080E003C080E001C080E0DF91A4
:1082A000CF911F910F9108957F928F929F92AF92DD
:1082B000BF92CF92DF92EF92FF920F931F93CF93D3
:1082C000DF931F921F92CDB7DEB7009709F49BC0D2
:1082D0006115710509F497C0D42E7B018C01AE01A4
:1082E0004F5F5F4FBC018DEE94E178DF882309F486
:1082F0008AC089819A815C012FEFA21AB20AF80123
:10830000E80FF91F20E22083B8016A0D7B1DAE0142
:108310004F5F5F4F86ED94E161DF882309F473C0FE
:1083200089819A81A80EB91EF801EA0DFB1D8DE026
:10833000808382E0A80EB11C8AE08183B8016A0DB7
:108340007B1DAE014F5F5F4F8FEB94E147DF8823CA
:1083500009F459C0A981BA81AA0EBB1E48018A0C32
:108360009B1C0F2EFDE07F2EF02DF40170820F2E4E
:10837000FAE0CF2EF02DC182C5010296800F911F29
:108380000E9423D0F401748ED5015E96C58EDD2047
:1083900059F1A00FB11F8AE0EAE8F3E201900D92D3
:1083A0008A95E1F7F7E2AF0EB11C0E9450D5BC01EF
:1083B000C8018A0D9B1D0F94D5660E9450D5FC0103
:1083C00001900020E9F73197E81BF90BE131F10545
:1083D00018F4E983FA8304C080E190E089839A83EA
:1083E000A981BA81AA0DBB1DF801EA0FFB1F8DE020
:1083F000808312968AE08183F801EA0FFB1F1082C6
:10840000F701A083B1830F900F90DF91CF911F915F
:108410000F91FF90EF90DF90CF90BF90AF909F9023
:108420008F907F900895CF92DF92EF92FF920F93FB
:108430001F93CF93DF931F921F92CDB7DEB76115C5
:10844000710591F14115510579F1009769F17A01B2
:108450006B018C0119821A82AE014F5F5F4F89E177
:1084600093E1BCDE882301F1C80106969F938F93A8
:1084700084E993E29F938F9389819A818C0D9D1D4E
:108480009F938F930F94F366F60101900020E9F714
:108490003197EC19FD09D701ED93FC930F900F90E4
:1084A0000F900F900F900F900F900F90DF91CF9142
:1084B0001F910F91FF90EF90DF90CF900895BF92A2
:1084C000CF92DF92EF92FF920F931F93CF93DF93A0
:1084D0001F921F92CDB7DEB7009709F482C06115D5
:1084E000710509F47EC06B018C0119821A82DB01CF
:1084F0001D921C92AE014F5F5F4FBC018DE093E176
:108500006DDE882309F46DC0E8E2F4E587858F937A
:1085100086858F9385858F9384858F9380E59BE2F5
:108520009F938F9389819A81800F911F9F938F933F
:108530000F94F366F80101900020E9F73197E01BF2
:10854000F10BE983FA83CDBFDEBFB12C0F2EF9E921
:10855000EF2EF3E2FF2EF02D2DC0EB2DF0E0EE0F0D
:10856000FF1FEE0FFF1FE85DFB4ADF015A961396CF
:108570008C9113978F9312968C9112978F931196DB
:108580008C918F93828D8F93FF92EF9289819A8144
:10859000800F911F9F938F930F94F366F8010190C2
:1085A0000020E9F73197E01BF10BE983FA83B394DC
:1085B000CDBFDEBF0F942D2CB81678F2E981FA8179
:1085C000E00FF11F8DE09AE0808391831282F80121
:1085D00001900020E9F73197E01BF10BD601ED93F4
:1085E000FC930F900F90DF91CF911F910F91FF900F
:1085F000EF90DF90CF90BF900895BF92CF92DF921F
:10860000EF92FF920F931F93CF93DF9300D01F92AF
:10861000CDB7DEB719821A821B821C82009709F43B
:10862000CDC06115710509F4C9C0022FB42E6B01CC
:108630007C011FEF120F123108F0B5C0AE014F5F81
:108640005F4FBC0185E293E1C9DD882309F4B6C020
:108650001A3079F5BB2069F069817A816E0D7F1D32
:10866000AE014D5F5F4F86EB99E0F5DD81110EC0E5
:10867000A5C069817A816E0D7F1DAE014D5F5F4F90
:1086800082E999E0E8DD882309F498C069817A815C
:108690008B819C81680F791F69837A836E0D7F1DA2
:1086A000AE014D5F5F4F88E19BE098DD811171C0A5
:1086B00085C084EF800F873008F046C0BB2089F06A
:1086C00069817A816E0D7F1D812F90E0880F991F3F
:1086D000AE014D5F5F4F8C55964FBDDD811112C0CD
:1086E0006DC069817A816E0D7F1D812F90E0880FAA
:1086F000991FAE014D5F5F4F8058964FACDD8823C8
:1087000009F45CC069817A818B819C81680F791F33
:1087100069837A8322EF200F223058F46E0D7F1D7B
:10872000AE014D5F5F4F84E999E095DD811131C065
:1087300045C06E0D7F1DAE014D5F5F4F83E09BE036
:108740004DDD811126C03AC0BB2091F069817A814C
:108750006E0D7F1D212F30E0C901880F991FAE01DA
:108760004D5F5F4F8C55964F76DD811112C026C04C
:1087700069817A816E0D7F1D212F30E0C901880F3C
:10878000991FAE014D5F5F4F8058964F64DD88237F
:10879000A9F029813A818B819C81820F931FF60178
:1087A000808391830BC0AE014F5F5F4FBC0185E2B8
:1087B00093E114DD882311F010E0C6CF2496CDBFDD
:1087C000DEBFDF91CF911F910F91FF90EF90DF906F
:1087D000CF90BF90089589E10E9465D081E062301A
:1087E00009F080E00895CF92DF92EF92FF921F93FD
:1087F000CF93DF9300D01F92CDB7DEB719821A82D4
:108800001B821C82009709F453C06115710509F49D
:108810004FC0142F6B017C01AE014F5F5F4FBC0155
:1088200085E293E1DBDC882309F442C0173089F04C
:108830001930E1F0113039F569817A816E0D7F1DB3
:10884000AE014D5F5F4F82EA9AE0C8DC811127C01C
:108850002FC069817A816E0D7F1DAE014D5F5F4F24
:1088600081E49AE0BBDC81111AC022C069817A815F
:108870006E0D7F1DAE014D5F5F4F80EE99E0AEDC67
:1088800081110DC015C069817A816E0D7F1DAE0109
:108890004D5F5F4F82EA9AE0A1DC882349F029818D
:1088A0003A818B819C81820F931FF6018083918393
:1088B0002496CDBFDEBFDF91CF911F91FF90EF9047
:1088C000DF90CF900895EF92FF920F931F93CF9375
:1088D000DF931F921F92CDB7DEB719821A820097DD
:1088E000B1F16115710599F17B018C0187E10E945D
:1088F00065D0613051F4AE014F5F5F4FB8018BE23C
:1089000094E16CDC811116C022C061110AC0AE0175
:108910004F5F5F4FB8018EEA93E160DC81110AC0BE
:1089200016C0AE014F5F5F4FB80181E393E156DCA3
:10893000882369F089819A81F801E80FF91F2DE0F9
:1089400020832AE021830296F701808391830F9090
:108950000F90DF91CF911F910F91FF90EF900895AD
:10896000EF92FF920F931F93CF93DF931F921F926B
:10897000CDB7DEB7009709F47EC04115510509F463
:108980007CC0F22E8A01E62EAE014F5F5F4FB80128
:1089900062DC811102C019821A8283E0E81629F193
:1089A0008E1538F091E0E91659F082E0E81699F05A
:1089B0003AC094E0E91619F185E0E81651F133C0A8
:1089C000ECE7F7E401900020E9F73197EC57F74422
:1089D0006CE777E42BC0E3E9F7E401900020E9F7C6
:1089E000E459F74463E977E421C0EAEAF7E4019047
:1089F0000020E9F7EB5AF7446AEA77E417C0E1ECA4
:108A0000F7E401900020E9F7E25CF74461EC77E4D9
:108A10000DC0E8EDF7E401900020E9F7E95DF744C7
:108A200068ED77E403C06CE777E4E0E0EF3008F04E
:108A3000EEE0CB018E0F911DFC01108289819A819D
:108A4000800F911F0F94D566F80101900020E9F77F
:108A50003197E01BF10BFF2091F0C8018E0F911DA3
:108A6000FC018CE29DE0808391838AE090E0828328
:108A7000938381E005C080E003C080E001C081E015
:108A80000F900F90DF91CF911F910F91FF90EF907A
:108A900008958F929F92AF92BF92CF92DF92EF9202
:108AA000FF920F931F93CF93DF931F921F92CDB727
:108AB000DEB73091463F311104C0FB0110821182B4
:108AC00036C00097A1F1672B91F14115510579F15D
:108AD000022F4A016C010F2EFBEBEF2EFAE1FF2E65
:108AE000F02D11E0202FA601612FC70139DF882367
:108AF000A9F0F60101900020E9F731975F01AC1869
:108B0000BD089E012F5F3F4FA501B601C4010F9420
:108B1000EA5A89819A81A816B90631F41F5FF2E0FA
:108B2000EF0EF11C1630F1F6C4010F94985C0F9013
:108B30000F90DF91CF911F910F91FF90EF90DF90F9
:108B4000CF90BF90AF909F908F9008958F929F92FB
:108B5000AF92BF92DF92EF92FF920F931F93CF934A
:108B6000DF93CDB7DEB72597CDBFDEBF009709F401
:108B700021C54115510509F41FC5D22E7A01162FC2
:108B8000AE014F5F5F4FB70166DB811102C01982F2
:108B90001A82163109F06DC00F9474054B015C0107
:108BA000672B682B692BE1F486E10E9465D020E1F8
:108BB0003EE040E050E00F94AA645F934F933F93F0
:108BC0002F9384EA93E29F938F9389819A818E0DEC
:108BD0009F1D9F938F930F94F366CDBFDEBFD3C4C9
:108BE00086E10E9465D0992324F586E10E9465D034
:108BF00020E13EE040E050E00F94AA64CA01B901D0
:108C00000F940837BF92AF929F928F929F938F934A
:108C10007F936F938FE993E29F938F9389819A81DA
:108C20008E0D9F1D9F938F930F94F366CDBFDEBF74
:108C3000AAC486E10E9465D0BF92AF929F928F92A4
:108C400020E13EE040E050E00F94AA645F934F9330
:108C50003F932F9380EA93E29F938F9389819A8128
:108C60008E0D9F1D9F938F930F94F366CDBFDEBF34
:108C70008AC4123060F4812F0E94CAD029813A81BF
:108C8000BC01C701820F931F0F94D5667CC41630B8
:108C900081F486E00E9465D08B019C0189819A81D4
:108CA0004BE0BE016B5F7F4F8E0D9F1D0F946137B0
:108CB0006AC4153081F485E00E9465D08B019C0167
:108CC00089819A814BE0BE016B5F7F4F8E0D9F1DA6
:108CD0000F94AD3858C4123009F06EC082E00E9483
:108CE00065D0633171058105910524F061E070E084
:108CF00080E090E0013009F049C029813A812E0DD1
:108D00003F1DDC01CB010197A109B109880F991F13
:108D1000AE014D5F5F4FB9018D58974F9CDA81309E
:108D2000F9F4F70101900020E9F73197EE19FF09F6
:108D3000E983FA8382E00E9465D09F938F937F93AB
:108D40006F9389EA93E29F938F9389819A818E0D25
:108D50009F1D9F938F930F94F366CDBFDEBF13C407
:108D600082E00E9465D09F938F937F936F938AEAEE
:108D700093E29F938F9389819A818E0D9F1D9F937C
:108D80008F930F94F366CDBFDEBFFDC382E00E94D8
:108D900065D09F938F937F936F9381E59BE29F9321
:108DA0008F9389819A818E0D9F1D9F938F930F942E
:108DB000F366CDBFDEBFE7C3173109F086C087E198
:108DC0000E9465D04B015C01011113C0BF92AF92AC
:108DD0009F926F9381E59BE29F938F9389819A8104
:108DE0008E0D9F1D9F938F930F94F366CDBFDEBFB3
:108DF000CAC391E089169104A104B10439F082E05C
:108E000088169104A104B10409F140C069817A81F6
:108E10006E0D7F1DAE014D5F5F4F88E098E0DED99B
:108E20008111B1C31F921F921F9281E08F9381E540
:108E30009BE29F938F9389819A818E0D9F1D9F93B3
:108E40008F930F94F366CDBFDEBF9DC369817A8196
:108E50006E0D7F1DAE014D5F5F4F83E098E0BED980
:108E6000811191C31F921F921F9282E08F9381E51F
:108E70009BE29F938F9389819A818E0D9F1D9F9373
:108E80008F930F94F366CDBFDEBF7DC369817A8176
:108E90006E0D7F1DAE014D5F5F4F8CE098E09ED957
:108EA000811171C3BF92AF929F928F9281E59BE235
:108EB0009F938F9389819A818E0D9F1D9F938F938E
:108EC0000F94F366CDBFDEBF5EC31B3049F08DEE5D
:108ED000810F823028F0812F8D7F883109F05CC0AE
:108EE000812F0E9465D04B015C01011113C0BF921C
:108EF000AF929F926F9381E59BE29F938F938981BD
:108F00009A818E0D9F1D9F938F930F94F366CDBF13
:108F1000DEBF39C3672B682B692BF9F469817A812D
:108F20006E0D7F1DAE014D5F5F4F8FE698E056D905
:108F3000811129C31F921F921F921F9281E59BE20C
:108F40009F938F9389819A818E0D9F1D9F938F93FD
:108F50000F94F366CDBFDEBF16C369817A816E0DB3
:108F60007F1DAE014D5F5F4F8CE698E037D98111D0
:108F70000AC3BF92AF929F928F9281E59BE29F932B
:108F80008F9389819A818E0D9F1D9F938F930F944C
:108F9000F366CDBFDEBFF7C2173009F05CC087E0D3
:108FA0000E9465D04B015C01011113C0BF92AF92CA
:108FB0009F926F9381E59BE29F938F9389819A8122
:108FC0008E0D9F1D9F938F930F94F366CDBFDEBFD1
:108FD000DAC2672B682B692BF9F469817A816E0DEF
:108FE0007F1DAE014D5F5F4F88E698E0F7D8811195
:108FF000CAC21F921F921F921F9281E59BE29F930C
:109000008F9389819A818E0D9F1D9F938F930F94CB
:10901000F366CDBFDEBFB7C269817A816E0D7F1D59
:10902000AE014D5F5F4F84E698E0D8D88111ABC2A6
:10903000BF92AF929F928F9281E59BE29F938F9315
:1090400089819A818E0D9F1D9F938F930F94F36654
:10905000CDBFDEBF98C2143009F05CC084E00E942E
:1090600065D04B015C01011113C0BF92AF929F927A
:109070006F9381E59BE29F938F9389819A818E0DF7
:109080009F1D9F938F930F94F366CDBFDEBF7BC26E
:10909000672B682B692BF9F469817A816E0D7F1D2E
:1090A000AE014D5F5F4F8DE598E098D881116BC29E
:1090B0001F921F921F921F9281E59BE29F938F93B5
:1090C00089819A818E0D9F1D9F938F930F94F366D4
:1090D000CDBFDEBF58C269817A816E0D7F1DAE01A2
:1090E0004D5F5F4F84E598E079D881114CC2BF9203
:1090F000AF929F928F9281E59BE29F938F9389819C
:109100009A818E0D9F1D9F938F930F94F366CDBF11
:10911000DEBF39C2133009F0ADC083E00E9465D0D4
:109120004B015C01011113C0BF92AF929F926F93EC
:1091300081E59BE29F938F9389819A818E0D9F1D7C
:109140009F938F930F94F366CDBFDEBF1CC291E057
:1091500089169104A104B10461F182E0881691049A
:10916000A104B10409F445C081149104A104B1041F
:1091700009F060C069817A816E0D7F1DAE014D5F7F
:109180005F4F88E498E02AD88111FDC11F921F9299
:109190001F921F9281E59BE29F938F9389819A8111
:1091A0008E0D9F1D9F938F930F94F366CDBFDEBFEF
:1091B000EAC169817A816E0D7F1DAE014D5F5F4FFF
:1091C0008FE398E00BD88111DEC11F921F921F928E
:1091D00081E08F9381E59BE29F938F9389819A81B0
:1091E0008E0D9F1D9F938F930F94F366CDBFDEBFAF
:1091F000CAC169817A816E0D7F1DAE014D5F5F4FDF
:109200008AE398E00E94EE408111BDC11F921F9237
:109210001F9282E08F9381E59BE29F938F938981D8
:109220009A818E0D9F1D9F938F930F94F366CDBFF0
:10923000DEBFA9C169817A816E0D7F1DAE014D5FD0
:109240005F4F88E498E00E94EE4081119CC1BF927C
:10925000AF929F928F9281E59BE29F938F9389813A
:109260009A818E0D9F1D9F938F930F94F366CDBFB0
:10927000DEBF89C1193109F0AFC089E10E9465D014
:109280004B015C01011113C0BF92AF929F926F938B
:1092900081E59BE29F938F9389819A818E0D9F1D1B
:1092A0009F938F930F94F366CDBFDEBF6CC191E0A7
:1092B00089169104A104B10469F182E08816910431
:1092C000A104B10409F447C081149104A104B104BC
:1092D00009F062C069817A816E0D7F1DAE014D5F1C
:1092E0005F4F86E398E00E94EE4081114CC11F92CF
:1092F0001F921F921F9281E59BE29F938F9389811A
:109300009A818E0D9F1D9F938F930F94F366CDBF0F
:10931000DEBF39C169817A816E0D7F1DAE014D5F5F
:109320005F4F80E398E00E94EE4081112CC11F92B4
:109330001F921F9281E08F9381E59BE29F938F9311
:1093400089819A818E0D9F1D9F938F930F94F36651
:10935000CDBFDEBF18C169817A816E0D7F1DAE0160
:109360004D5F5F4F88E298E00E94EE4081110BC193
:109370001F921F921F9282E08F9381E59BE29F9341
:109380008F9389819A818E0D9F1D9F938F930F9448
:10939000F366CDBFDEBFF7C069817A816E0D7F1D98
:1093A000AE014D5F5F4F86E398E00E94EE40811171
:1093B000EAC0BF92AF929F928F9281E59BE29F930A
:1093C0008F9389819A818E0D9F1D9F938F930F9408
:1093D000F366CDBFDEBFD7C0123109F05EC082E1B7
:1093E0000E9465D04B015C01011113C0BF92AF9286
:1093F0009F926F9381E59BE29F938F9389819A81DE
:109400008E0D9F1D9F938F930F94F366CDBFDEBF8C
:10941000BAC0672B682B692B01F569817A816E0DC3
:109420007F1DAE014D5F5F4F87E198E00E94EE40E7
:109430008111A9C01F921F921F921F9281E59BE28A
:109440009F938F9389819A818E0D9F1D9F938F93F8
:109450000F94F366CDBFDEBF96C069817A816E0D31
:109460007F1DAE014D5F5F4F8FE098E00E94EE40A0
:10947000811189C0BF92AF929F928F9281E59BE24A
:109480009F938F9389819A818E0D9F1D9F938F93B8
:109490000F94F366CDBFDEBF76C0153109F05EC014
:1094A00085E10E9465D04B015C01011113C0BF92A0
:1094B000AF929F926F9381E59BE29F938F938981F7
:1094C0009A818E0D9F1D9F938F930F94F366CDBF4E
:1094D000DEBF59C0672B682B692B01F569817A8142
:1094E0006E0D7F1DAE014D5F5F4F83E298E00E94DD
:1094F000EE40811148C01F921F921F921F9281E57A
:109500009BE29F938F9389819A818E0D9F1D9F93DC
:109510008F930F94F366CDBFDEBF35C069817A812A
:109520006E0D7F1DAE014D5F5F4F8EE198E00E9492
:10953000EE40811128C0BF92AF929F928F9281E539
:109540009BE29F938F9389819A818E0D9F1D9F939C
:109550008F930F94F366CDBFDEBF15C0812F0E949D
:1095600065D09F938F937F936F9381E59BE29F9349
:109570008F9389819A818E0D9F1D9F938F930F9456
:10958000F366CDBFDEBFF70101900020E9F7319708
:10959000EE19FF09DD2091F0C7018E0F911DFC012E
:1095A0008CE29DE0808391838AE090E082839383C4
:1095B00081E005C080E003C080E001C081E0259625
:1095C000CDBFDEBFDF91CF911F910F91FF90EF9044
:1095D000DF90BF90AF909F908F9008956F927F9291
:1095E0008F929F92AF92BF92CF92DF92EF92FF92B3
:1095F0000F931F93CF93DF931F921F92CDB7DEB7C8
:109600000097B1F1672BA1F14115510589F1802E29
:10961000922E3A016C010F2EFAE6EF2EFCE1FF2E9E
:10962000F02D10E0082D292DA601612FC7018EDA3B
:109630008823A9F0F60101900020E9F731975F0136
:10964000AC18BD089E012F5F3F4FA501B601C301B5
:109650000F94EA5A89819A81A816B90631F41F5FDE
:1096600082E0E80EF11C1C31E9F6C3010F94985C0E
:109670000F900F90DF91CF911F910F91FF90EF907E
:10968000DF90CF90BF90AF909F908F907F906F9022
:1096900008958F929F92AF92BF92DF92EF92FF92C6
:1096A0000F931F93CF93DF931F921F92CDB7DEB717
:1096B000009709F48FC06115710509F48BC04B0147
:1096C0007C010E9450D59F938F9380EB93E29F93F0
:1096D0008F93FF92EF920F94F366F70101900020B1
:1096E000E9F73197AF014E195F094231510510F08A
:1096F00041E150E09E012F5F3F4FB701C4010F943D
:10970000EA5A0F900F900F900F900F900F90D12C5E
:109710000F2EFBE0AF2EFAE2BF2EF02D8D2D0E9412
:1097200041D09F938F937F936F93BF92AF92FF929D
:10973000EF920F94F366F70101900020E9F731975B
:109740008F010E191F099E012F5F3F4FA801B7011E
:10975000C4010F94EA5ACDBFDEBF89819A810817F0
:10976000190731F4D39496E1D912D8CF11E001C092
:1097700011E00F2EF0EBAF2EF3E2BF2EF02D812F74
:109780000E94B1D89F938F93BF92AF92FF92EF92B6
:109790000F94F366F70101900020E9F73197AF01CC
:1097A0004E195F094231510510F041E150E09E0130
:1097B0002F5F3F4FB701C4010F94EA5A1F5F0F900C
:1097C0000F900F900F900F900F901330C1F6C401BF
:1097D0000F94985C0F900F90DF91CF911F910F9194
:1097E000FF90EF90DF90BF90AF909F908F90089583
:1097F0002F923F924F925F926F927F928F929F92A1
:10980000AF92BF92CF92DF92EF92FF920F931F938E
:10981000CF93DF93CDB7DEB7E197CDBFDEBF91E049
:109820009BA76115710509F4EAC34115510509F4B7
:10983000E8C38A017B0189AB0F94E52B29A921306C
:1098400089F4A80166E873E3CE010B960E94D9560D
:10985000182F86E08BA70F94A2186DA77EA78FA75D
:1098600098AB1AC0A80166E873E3CE010B960E947C
:109870004E57182F0F94A2186DA77EA78FA798ABED
:1098800082E00F941B17862FAE01445D5F4FBE012F
:10989000655D7F4F0E940E22112309F4B4C341E09D
:1098A000BE01675F7F4FC7010E94544149855A85B9
:1098B000CA01A0E0B0E089839A83AB83BC839E0198
:1098C000275F3F4FB701CE010B960F94EA5ACE01A6
:1098D0000B960F94985CBE01655F7F4FC701D9DE80
:1098E0000DE0D7010C931AE011961C939E01275F9F
:1098F0003F4F42E050E0B701CE010B960F94EA5A79
:10990000CE010B960F94985CE6E8F3E3018B128B83
:109910009E01275F3F4F43E150E0BF01CE010B9610
:109920000F94EA5ACE010B960F94985CB9A9B11125
:109930006EC30F94F7180F94E01869C301E021E09B
:10994000A701612FC60102D9882381F0F701019098
:109950000020E9F73197AF014E195F099E01275F9B
:109960003F4FB701CE010B960F94EA5AE2E0CE0EBC
:10997000D11C1F5F133011F70F2EFCE7CF2EFCE137
:10998000DF2EF02D19E001E021E0A701612FC601D3
:10999000DDD8882381F0F70101900020E9F73197A5
:1099A000AF014E195F099E01275F3F4FB701CE01FE
:1099B0000B960F94EA5AF2E0CF0ED11C1F5F1B30BA
:1099C00011F70F2EF2E18F2E912CA12CB12CF02D3E
:1099D00028E182169104A104B10451F401E021E0D0
:1099E000A70169E18CE99CE1B1D881110EC030C0BA
:1099F00001E021E0A701682DC401880F991F865955
:109A0000934EA4D88823C1F007C00F2EF9E18F2E02
:109A1000912CA12CB12CF02DF70101900020E9F739
:109A20003197AF014E195F099E01275F3F4FB70184
:109A3000CE010B960F94EA5A33E0830E911CA11CC1
:109A4000B11C4AE184169104A104B10408F4C0CF0A
:109A5000CE010B960F94985C89E00E9465D06F311F
:109A6000710581059105C0F4DC01CB01072E7CE076
:109A7000880F991FAA1FBB1F7A95D1F7702D898374
:109A80009A83AB83BC8380E090E1A0E0B0E08D835B
:109A90009E83AF83B88717C0DC01CB01072E79E026
:109AA000880F991FAA1FBB1F7A95D1F7702D898344
:109AB0009A83AB83BC8380E092E0A0E0B0E08D832A
:109AC0009E83AF83B8878DA59EA5AFA5B8A9811544
:109AD000904EA140B10589F489E00E9465D06E31B5
:109AE00071058105910549F080E090E1A0E0B0E0CA
:109AF0008D839E83AF83B88741C089819A81AB8172
:109B0000BC812DA53EA54FA558A9281739074A079E
:109B10005B07A1F1AE01475F5F4FB70184ED99E0AC
:109B20000E94EE40813081F4F70101900020E9F7B6
:109B30003197AF014E195F099E01275F3F4FB70173
:109B4000CE010B960F94EA5ACE010B960F94985CB7
:109B5000CE010B960F94DF5C39A9311156C20F94D8
:109B60006E1987EF9CE30E94992281110F944E2970
:109B700087EF9CE30E94E62980E051C2AE01475F77
:109B80005F4FB70188EC99E00E94EE40813081F48C
:109B9000F70101900020E9F73197AF014E195F09F5
:109BA0009E01275F3F4FB701CE010B960F94EA5AF3
:109BB00048A94F935FA55F938EA58F939DA59F9313
:109BC00088858F938F818F938E818F938D818F93D3
:109BD00084EB93E29F938F93FF92EF920F94F3663F
:109BE000F70101900020E9F73197AF014E195F09A5
:109BF0009E01275F3F4FB701CE010B960F94EA5AA3
:109C000088E290E089879A8768E2C7010E94EFB8EE
:109C1000482F50E060E070E049835A836B837C8377
:109C2000682F70E0C7010F94F138CDBFDEBF8823E5
:109C3000C9F049815A819E01275F3F4FB701CE018C
:109C40000B960F94EA5A8DE0F70180838AE08183B6
:109C50009E01275F3F4F42E050E0B701CE010B96D7
:109C60000F94EA5ABE016F5F7F4FC7010E946344A1
:109C700049815A819E01275F3F4FB701CE010B9664
:109C80000F94EA5A6BE370E0C7010E9442B8A0E06B
:109C9000B0E089839A83AB83BC830E944E2A8111F2
:109CA0000EC0F70101900020E9F73197AF014E197E
:109CB0005F0920E0B7018AEA99E30F948B3149816B
:109CC0005A816B817C814115510561057105C1F097
:109CD0009E01275F3F4FB701CE010B960F94EA5AC2
:109CE0008DE0D7018C938AE011968C939E01275FBB
:109CF0003F4F42E050E0B701CE010B960F94EA5A75
:109D0000CE010B960F94985C0E946D5B19821A82AB
:109D10001B821C822DA53EA54FA558A9232B242BC1
:109D2000252B09F433C180E090E0DC010F2EFDEE1D
:109D30002F2EF3E23F2EF02D0F2EFFEB8F2EF3E2AE
:109D40009F2EF02D880F991FAA1FBB1FBC01CD01AC
:109D50007E5F8F4F9F4F0E94755B0E94005E811156
:109D6000FCCF80E091E0E6ECF3E4DF019C011D9282
:109D700021503040E1F76F010F2EF6ECAF2EF4E4E6
:109D8000BF2EF02D8F010E9403B8D8018D939D93B3
:109D90008D01AA16BB06B9F70E94405C0F94B83A31
:109DA000CE010B960F94985C412C512C3201F60198
:109DB000619171916F01AE014B5F5F4F8BA50E9466
:109DC000EA14882309F496C088858F938F818F9336
:109DD0008E818F938D818F9389819A81AB81BC8194
:109DE000840D951DA61DB71DBF93AF939F938F93B1
:109DF0009F928F92FF92EF920F94F366F70101907A
:109E00000020E9F73197AF014E195F099E01275FE6
:109E10003F4FB701CE010B960F94EA5A182FCDBFD2
:109E2000DEBF882309F48CC00E944E2A811126C00F
:109E300089819A81AB81BC81840D951DA61DB71DBA
:109E4000BF93AF939F938F931F921F9349EC53E25D
:109E50005F934F93FF92EF920F94F366F701019097
:109E60000020E9F73197AF014E195F0920E0B701F3
:109E70008AEA99E30F948B31CDBFDEBFF7010190E1
:109E80000020E9F73197AF014E195F099E01275F66
:109E90003F4FB701CE010B960F94EA5A182F0E943C
:109EA0004E2A81114DC089819A81AB81BC81840D7C
:109EB000951DA61DB71DBF93AF939F938F931F92C0
:109EC0001F93EAEDF3E2FF93EF93FF92EF920F946B
:109ED000F366F70101900020E9F73197AF014E19C1
:109EE0005F0920E0B7018AEA99E30F948B31CDBF77
:109EF000DEBF26C00E944E2A811122C089819A812C
:109F0000AB81BC81840D951DA61DB71DBF93AF937A
:109F10009F938F933F922F92FF92EF920F94F3664D
:109F2000F70101900020E9F73197AF014E195F0961
:109F300020E0B7018AEA99E30F948B31CDBFDEBFF1
:109F40009FEF491A590A690A790AA0E84A1651048A
:109F50006104710409F02BCFCE010B960F94985C2D
:109F600089819A81AB81BC8180589F4FAF4FBF4F91
:109F700089839A83AB83BC832DA53EA54FA558A9A1
:109F800082179307A407B50708F4DCCECE010B9621
:109F90000F94985CCE010B960F94DF5C1092973370
:109FA00086E893E30E942D5839A931110DC00F9412
:109FB0006E1987EF9CE30E94992281110F944E291C
:109FC00087EF9CE30E94E62903EB10E4D801129688
:109FD0006D917C9113978D919C910F941458D0D5CD
:109FE0006DEF7CE3C8010E946658F80142855385F5
:109FF00064857585C8010F94EA5C81E010C080E03B
:10A000000EC080E00CC080E00AC080E008C00F2EC7
:10A01000FAE6CF2EFCE1DF2EF02D10E08FCCE1969A
:10A02000CDBFDEBFDF91CF911F910F91FF90EF90D9
:10A03000DF90CF90BF90AF909F908F907F906F9068
:10A040005F904F903F902F900895CF92DF92EF92C4
:10A05000FF920F931F93CF93DF931F921F92CDB761
:10A06000DEB7009709F457C06115710509F453C0B4
:10A070007B018C01AE014F5F5F4FBC018DEE94E11F
:10A080000E94EE40882309F446C089819A816C01C0
:10A090002FEFC21AD20AF801E80FF91F20E220833D
:10A0A000B8016C0D7D1DAE014F5F5F4F86ED94E1F1
:10A0B0000E94EE40882379F189819A81C80ED91EC9
:10A0C000F801EC0DFD1D8DE0808382E0C80ED11CEF
:10A0D0008AE08183B8016C0D7D1DAE014F5F5F4F3B
:10A0E00088EA94E10E94EE408823A9F089819A8150
:10A0F000C80ED91EF801EC0DFD1D8DE0808322E015
:10A10000C20ED11C8AE08183F801EC0DFD1D108286
:10A11000F701C082D1820F900F90DF91CF911F91F4
:10A120000F91FF90EF90DF90CF900895EF92FF9204
:10A130000F931F93CF93DF93CDB7DEB7A297CDBF19
:10A14000DEBF009709F451C06115710509F44FC0D5
:10A150007B018C0160E0CE01039615D7882309F4BA
:10A160004BC0B701C80171DFF701408151819E01E9
:10A170002F5F3F4FB801CE0103960F94EA5ACE01EC
:10A1800003960F94985CF7012081318189819A812F
:10A190002817390771F5BE016D5F7F4FC80179DA65
:10A1A000A701B80182EA9CE10E94EE40813099F457
:10A1B000F701408151819E012F5F3F4FB801CE01D1
:10A1C00003960F94EA5AF7012081318189819A819F
:10A1D0002817390781F4CE0103960F94DF5C81E0E4
:10A1E00012D70F94E52B81E007C080E005C080E026
:10A1F00003C080E001C080E0A296CDBFDEBFDF914A
:10A20000CF911F910F91FF90EF9008950F931F939F
:10A21000CF93DF931F921F92CDB7DEB70F94E52B3C
:10A220008091393F823009F462C028F4882359F0C4
:10A23000813081F1D6C0843009F485C008F464C04F
:10A240008A30E1F0CEC060E083E990E47FD58111EF
:10A2500007C060913A3F87EF9CE30E94AC14C9C0ED
:10A260000F943411811104C081E08093393FC1C043
:10A270008AE08093393F0F94F629BBC00F940D2AD2
:10A280006C3D75408105910508F4B3C081E0809371
:10A29000393FAFC040E06BE27DE38DE29DE30E9479
:10A2A000544107EF1CE3F80144A955A99E012F5F13
:10A2B0003F4F6DE27DE383E990E40F94EA5A83E92E
:10A2C00090E40F94985CF80124A935A989819A81BA
:10A2D0002817390741F01092393F60913A3FC80181
:10A2E0000E94AC1486C082E08093393F82C000E0B7
:10A2F00021E043E950E46BE27DE38DE29DE36ED91A
:10A3000083E08093393F75C04BE25DE36DE27DE30E
:10A3100082EA9CE10E94EE40813069F440912B3D3D
:10A3200050912C3D9E012F5F3F4F6DE27DE383E90D
:10A3300090E40F94EA5A83E990E40F94DF5C84E0A0
:10A340008093393F56C00E9444E2882381F10F94E4
:10A35000402B8823C9F00E94BA1F882309F449C002
:10A3600087EF9CE30E94992281110F944E2987EF79
:10A370009CE30E94E6291092393F60913A3F87EFB3
:10A380009CE30E94AC1435C087EF9CE30E949922A5
:10A3900081110F944E2987EF9CE30E94E6291092C9
:10A3A000393F61E087EF9CE30E94AC1422C00F9418
:10A3B0008829672B682B692BE1F487EF9CE30E94C7
:10A3C000992281110F944E2987EF9CE30E94E62980
:10A3D0001092393F60913A3F87EF9CE30E94AC14A2
:10A3E00008C01092393F60913A3F87EF9CE30E948A
:10A3F000AC140F900F90DF91CF911F910F910895A2
:10A400009F92AF92BF92CF92DF92EF92FF920F9303
:10A410001F93CF93DF9300D0CDB7DEB7009709F439
:10A4200071C06115710509F46DC0A42E6B017C012A
:10A430008EE0E8EFF3E2D70101900D928A95E1F703
:10A44000F70101900020E9F73197EE19FF09E98340
:10A45000AF0155279E012E5F3F4FB701C6010F94F4
:10A46000EA5AB12C0F2EFCE29F2EF02D8B2D0E946C
:10A47000C0D78B019C0148E0BE016F5F7F4FC701D1
:10A480000F940F3982E08B1550F08981F701E80FA6
:10A49000F11D90828F5FF701E80FF11D1082F70127
:10A4A00001900020E9F73197EE19FF09E983AF0128
:10A4B00055279E012E5F3F4FB701C6010F94EA5A00
:10A4C000898190E02A813B818217930721F4B3941C
:10A4D000E4E0BE12CBCFAA2081F08DE0F7018083AB
:10A4E0008AE0818382E089839E012E5F3F4F42E0B4
:10A4F00050E0B701C6010F94EA5AC6010F94985C68
:10A500000F94E52B2396CDBFDEBFDF91CF911F9136
:10A510000F91FF90EF90DF90CF90BF90AF909F9002
:10A5200008959F92AF92BF92CF92DF92EF92FF92E7
:10A530000F931F93CF93DF931F921F92CDB7DEB778
:10A54000009709F4E1C06115710509F4DFC04115F8
:10A55000510509F4DDC0902E122F5A016B017C01C8
:10A560000F94E52B41E0B601C7010E945441F6016A
:10A57000408151819E012F5F3F4FB701C5010F946C
:10A58000EA5AC5010F94985CF601208131818981D6
:10A590009A812817390709F0BDC08DE0E6E0F4E2A2
:10A5A000D70101900D928A95E1F7F7010190002003
:10A5B000E9F73197AF014E195F0955279E012F5FCB
:10A5C0003F4FB701C5010F94EA5AC5010F94985C3B
:10A5D000B501C7015ED88DE0F70180838AE08183F1
:10A5E0009E012F5F3F4F42E050E0B701C5010F943D
:10A5F000EA5AC5010F94985C41E0B501C70100DF3C
:10A60000A601B70187EF9CE30E941342F601408147
:10A6100051819E012F5F3F4FB701C5010F94EA5A48
:10A62000C5010F94985CF6012081318189819A815E
:10A630002817390709F070C0B601C7010E945F42B0
:10A64000F601408151819E012F5F3F4FB701C50147
:10A650000F94EA5AC5010F94985CF601208131816C
:10A6600089819A812817390709F058C001E021E053
:10A67000A501B601C7010E94EE4A21E0A501B6017D
:10A68000C7010E9449450E94EB43882331F0492DC0
:10A69000B601C7010E94F34306C0292D412FB60120
:10A6A000C7010E94FD42F601408151819E012F5F4A
:10A6B0003F4FB701C5010F94EA5AC5010F94985C4A
:10A6C000F6012081318189819A812817390741F566
:10A6D000B601C7010E946344F601408151819E0189
:10A6E0002F5F3F4FB701C5010F94EA5AC5010F9480
:10A6F000985C81E0F6014081518129813A814217BD
:10A70000530779F080E00DC080E00BC080E009C005
:10A7100080E007C080E005C080E003C080E001C0A9
:10A7200080E00F900F90DF91CF911F910F91FF90DC
:10A73000EF90DF90CF90BF90AF909F9008952F92B1
:10A740003F924F925F926F927F928F929F92AF92C1
:10A75000BF92CF92DF92EF92FF920F931F93CF930E
:10A76000DF93CDB7DEB7A897CDBFDEBF411551054A
:10A7700009F4D7C12115310509F4D5C16115710559
:10A7800009F4D3C1280169011A017B0188A70F943C
:10A79000E52BA60166E873E3CE010796A7D68823CA
:10A7A00009F4C5C141E0BE016B5F7F4FC1010E944A
:10A7B00054414D815E819E012B5F3F4FB101CE011F
:10A7C00007960F94EA5ACE0107960F94985CBE0143
:10A7D000695F7F4FC1010E94494B1DE0F101108369
:10A7E0000AE001839E012B5F3F4F42E050E0B10140
:10A7F000CE0107960F94EA5ACE0107960F94985C03
:10A80000E6E8F3E3118B028B9E012B5F3F4F43E1A0
:10A8100050E0BF01CE0107960F94EA5ACE01079689
:10A820000F94985C0F2EFAE6CF2EFCE1DF2EF02D70
:10A8300010E001E021E0A101612FC6010E94A645C0
:10A84000882381F0F10101900020E9F73197AF01F1
:10A85000421953099E012B5F3F4FB101CE0107966C
:10A860000F94EA5AF2E0CF0ED11C1F5F133009F7A4
:10A870000F2EFCE7CF2EFCE1DF2EF02D19E001E0DA
:10A8800021E0A101612FC6010E94A645882381F025
:10A89000F10101900020E9F73197AF014219530906
:10A8A0009E012B5F3F4FB101CE0107960F94EA5AEC
:10A8B00022E0C20ED11C1F5F1B3009F70F2EF2E100
:10A8C0008F2E912CA12CB12CF02D88E188169104AB
:10A8D000A104B10491F401E021E0A10169E18CE956
:10A8E0009CE10E94A645811116C00F2EFCE18F2E1F
:10A8F000912CA12CB12CF02D31C001E021E0A1015F
:10A90000682DC401880F991F8659934E0E94A64551
:10A910008823C1F007C00F2EF9E18F2E912CA12CB6
:10A92000B12CF02DF10101900020E9F73197AF0132
:10A93000421953099E012B5F3F4FB101CE0107968B
:10A940000F94EA5A93E0890E911CA11CB11CEAE114
:10A950008E169104A104B10408F4B7CF1F92F8A594
:10A96000FF9383E194E29F938F933F922F920F94F2
:10A97000F366F10101900020E9F73197AF01421928
:10A9800053099E012B5F3F4FB101CE0107960F94F3
:10A99000EA5ACE0107960F94985C612C712C0F90A7
:10A9A0000F900F900F900F900F904114510461047D
:10A9B000710409F4A7C0870175016401812C912CF1
:10A9C0005401F80141915191619171918F019E0162
:10A9D0002F5F3F4F88A50E94D02E882309F482C0A4
:10A9E0008C818F938B818F938A818F9389818F93B1
:10A9F000BF92AF929F928F928FEB93E29F938F9330
:10AA00003F922F920F94F366F10101900020E9F735
:10AA10003197AF01421953099E012B5F3F4FB1019E
:10AA2000CE0107960F94EA5A8FA3CDBFDEBF9FA138
:10AA3000992309F457C00E944E2A81111FC0FF922A
:10AA4000EF92DF92CF921F92EFA1EF9389EC93E206
:10AA50009F938F933F922F920F94F366F101019091
:10AA60000020E9F73197AF014219530920E0B10105
:10AA70008AEA99E30F948B31CDBFDEBFF1010190DB
:10AA80000020E9F73197AF01421953099E012B5F6E
:10AA90003F4FB101CE0107960F94EA5A8FA30E944F
:10AAA0004E2A81111FC0FF92EF92DF92CF921F9228
:10AAB0009FA19F93EAEDF3E2FF93EF933F922F92D2
:10AAC0000F94F366F10101900020E9F73197AF018F
:10AAD0004219530920E0B1018AEA99E30F948B31BE
:10AAE000CDBFDEBF9FEF891A990AA90AB90AEFEF15
:10AAF000CE1ADE0AEE0AFE0A84149504A604B704F0
:10AB000008F45FCFCE0107960F94985CCE010796AC
:10AB10000F94DF5C1092973386E893E39ED281E036
:10AB200007C080E005C080E003C080E001C080E095
:10AB3000A896CDBFDEBFDF91CF911F910F91FF90FF
:10AB4000EF90DF90CF90BF90AF909F908F907F90CD
:10AB50006F905F904F903F902F900895089580914F
:10AB60009B330895089510929B3380919A338823E4
:10AB700031F010929A3383EB90E40D94DF5C0895EA
:10AB800083EB90E40D94DF5C089580919A330895EF
:10AB9000CF92DF92EF92FF921F93CF93DF93CDB7C7
:10ABA000DEB76897CDBFDEBF6C017B0184E1EEE1CB
:10ABB000F4E2DE01159601900D928A95E1F7DA0133
:10ABC000C9010196A11DB11D883E23E09207A10590
:10ABD000B1050CF460C01F921F921F9281E08F9309
:10ABE0008EEE91E29F938F93CE0101969F938F9368
:10ABF0000F94F3668981898B8A818A8B8B818B8BF9
:10AC000080E38D838AE38E83CDBFDEBFE114F10440
:10AC100059F0D701FE0138969E01245F3F4F8D9178
:10AC20008193E217F307D9F710E346E0BE016B5FAB
:10AC30007F4F83EB90E40F944C5899EF980F92302C
:10AC4000C8F48B89893399F48A89893361F48989B5
:10AC5000893321F410929A3380E03CC08F5F898B56
:10AC60001A8B1B8BE2CF1B8B8F5F8A8BDECF8F5FA4
:10AC70008B8BDBCF882321F010929A3380E02AC09F
:10AC800081E080939A33BE01695F7F4FC6010F94C4
:10AC9000D56681E01FC0BF93AF939F938F938EEED5
:10ACA00091E29F938F93CE0101969F938F930F9480
:10ACB000F3668981898B8A818A8B8B818B8B80E378
:10ACC0008D838AE38E83CDBFDEBFE114F10409F0EA
:10ACD000A0CFAACF6896CDBFDEBFDF91CF911F91E5
:10ACE000FF90EF90DF90CF90089580E00F947B115C
:10ACF000882361F08250823030F580919B33882325
:10AD000011F110929B3310929A33089580919B33E6
:10AD1000811119C081E080939B338EE292E0ECE9CF
:10AD2000F3E3DF019C011D9221503040E1F7BF01A8
:10AD300080E00F942E588B3019F410929A330895B6
:10AD400081E080939A3308958AE00895CF93DF934A
:10AD5000CDB7DEB76097CDBFDEBF009719F120E316
:10AD600029832AE32A832BE0E2E3F4E2DE0113964F
:10AD700001900D922A95E1F7613041F441E0BE0166
:10AD80006F5F7F4F0F944C58982F07C04AE0BE0169
:10AD90006F5F7F4F0F944C58982F81E0992319F0E3
:10ADA00080E001C080E06096CDBFDEBFDF91CF9133
:10ADB0000895DF92EF92FF920F931F93CF93DF934B
:10ADC000CDB7DEB76497CDBFDEBF8C0184E1EDE384
:10ADD000F4E2DE01119601900D928A95E1F70115DA
:10ADE000110509F449C06115710509F447C080E3F4
:10ADF00089838AE38A834115510559F0DA01FE01FE
:10AE000034969E01285F3F4F9D919193E217F3077F
:10AE1000D9F77B010F2EF0E3DF2EF02D46E0BE01C7
:10AE20006F5F7F4FC8010F944C5899EF980F923085
:10AE3000A8F49F85993379F48E85893341F48D8503
:10AE40008933F1F08F5F8D87DE86DF86E7CFDF867F
:10AE50008F5F8E87E3CF9F5F9F87E0CF811112C006
:10AE600081E1FE013396D70101900D928A95E1F7B9
:10AE7000F701118A81E007C080E005C080E003C0CF
:10AE800080E001C080E06496CDBFDEBFDF91CF914E
:10AE90001F910F91FF90EF90DF900895DF92EF9256
:10AEA000FF920F931F93CF93DF93CDB7DEB76497D5
:10AEB000CDBFDEBF8C0184E1E1E5F4E2DE01119655
:10AEC00001900D928A95E1F70115110509F449C029
:10AED0006115710509F447C080E389838AE38A8399
:10AEE0004115510559F0DA01FE0134969E01285FA3
:10AEF0003F4F9D919193E217F307D9F77B010F2EF6
:10AF0000F0E3DF2EF02D46E0BE016F5F7F4FC801FA
:10AF10000F944C5899EF980F9230A8F49F8599336D
:10AF200079F48E85893341F48D858933F1F08F5F13
:10AF30008D87DE86DF86E7CFDF868F5F8E87E3CF64
:10AF40009F5F9F87E0CF811112C081E1FE013396A0
:10AF5000D70101900D928A95E1F7F701118A81E0FE
:10AF600007C080E005C080E003C080E001C080E051
:10AF70006496CDBFDEBFDF91CF911F910F91FF90FF
:10AF8000EF90DF9008950F931F93CF93DF93CDB78A
:10AF9000DEB76097CDBFDEBF009761F18C0180E323
:10AFA00089838AE38A838BE0E5E6F4E2DE01139687
:10AFB00001900D928A95E1F7613049F441E0BE01BC
:10AFC0006F5F7F4FC8010F944C58982F0EC041E01F
:10AFD00060E0CE0103960F94BC5E4AE0BE016F5F55
:10AFE0007F4FC8010F944C58982F81E0992319F096
:10AFF00080E001C080E06096CDBFDEBFDF91CF91E1
:10B000001F910F910895CF93DF93CDB7DEB760976F
:10B01000CDBFDEBF9BE0E5E6F4E2DE0111960190D4
:10B020000D929A95E1F7813041F441E061E0CE0163
:10B0300001960F94BC5E982F07C041E060E0CE01FE
:10B0400001960F94BC5E982F81E0911180E060968C
:10B05000CDBFDEBFDF91CF910895009721F041E091
:10B0600061E00D94BC5E08951F93CF93DF93CDB73D
:10B07000DEB76497CDBFDEBF009701F1162FBC018C
:10B0800080E389838AE38A83CE0103960F94D56691
:10B09000113041F441E061E0CE0101960F94BC5EB5
:10B0A000982F07C041E060E0CE0101960F94BC5E8E
:10B0B000982F81E0992319F080E001C080E0649628
:10B0C000CDBFDEBFDF91CF911F910895EF92FF9228
:10B0D0000F931F93CF93DF93CDB7DEB76497CDBFA8
:10B0E000DEBF6115710589F1009789F18B017C0143
:10B0F00080E389838AE38A83CE0103960F94D56621
:10B1000043E0BE016F5F7F4FC7010F944C588730FB
:10B1100069F460E0C801A8DF982F8823D9F043E0E4
:10B12000BE016F5F7F4FC7010F944C58811111C052
:10B13000F7014285538564857585C7010F94EA5CE4
:10B1400091E0882339F090E005C090E003C090E0E2
:10B1500001C090E0892F6496CDBFDEBFDF91CF9113
:10B160001F910F91FF90EF900895CF93DF93CDB78C
:10B17000DEB76097CDBFDEBF0097C1F020E3298323
:10B180002AE32A832AE0E0E7F4E2DE011396019045
:10B190000D922A95E1F741E0BE016F5F7F4F0F945A
:10B1A0004C5891E0882319F090E001C090E0892F7D
:10B1B0006096CDBFDEBFDF91CF9108953F924F9251
:10B1C0005F926F927F928F929F92AF92BF92CF9237
:10B1D000DF92EF92FF920F931F93CF93DF93CDB740
:10B1E000DEB76197CDBFDEBF6115710509F470C090
:10B1F000009709F46FC04115510509F46DC03FEF88
:10B20000320F383008F06AC0322E7A018C01FB010F
:10B21000138A41E00F944C58811162C0F8014285B5
:10B22000538564857585483EF3E05F0761057105C8
:10B2300008F458C0413B84E058076105710508F0E7
:10B2400053C0C32CD12C5601E6E0AE0EB11C250133
:10B250000B2C000C66087708441955096609770914
:10B26000C8010F94EA5C811141C0A50160E070E063
:10B27000CE0103960F94CE669E012F5F3F4FA5012E
:10B28000BE016D5F7F4FC8010F949E59C8010F9496
:10B29000DF5CFE01EC0DFD1D12868E010D5F1F4F60
:10B2A000812C912C5401A601B801C7010F94B866F6
:10B2B000892BF1F0FFEF8F1A9F0AAF0ABF0A0F5FC9
:10B2C0001F4F481459046A047B0468F780E011C0DA
:10B2D00080E00FC080E00DC080E00BC080E009C0BE
:10B2E00080E007C081E005C080E003C080E001C0CD
:10B2F00081E06196CDBFDEBFDF91CF911F910F91AD
:10B30000FF90EF90DF90CF90BF90AF909F908F9085
:10B310007F906F905F904F903F9008954F925F9213
:10B320006F927F92AF92BF92CF92DF92EF92FF9295
:10B330000F931F93CF93DF93CDB7DEB76897CDBF41
:10B34000DEBF680114E1EEE1F4E2DE011596019042
:10B350000D921A95E1F7009709F491C0C114D10438
:10B3600009F48FC0EFEFEE0DE83008F08CC08601D5
:10B3700029013A015B016C01283E83E03807410551
:10B3800051050CF482C01F921F921F9281E08F938F
:10B390008EEE91E29F938F93CE0101969F938F93B0
:10B3A0000F94F3668981898B8A818A8B8B818B8B41
:10B3B00080E38D838AE38E83CDBFDEBFA114B10409
:10B3C00059F0D501FE0138969E01245F3F4F8D91C3
:10B3D0008193E217F307D9F70F2EF0E3FF2EF02D3C
:10B3E00046E0BE016B5F7F4F83EB90E40F944C58B7
:10B3F00099EF980F923090F52E2DA801BE016B5F4A
:10B400007F4F83EB90E4DADE882379F060E0C601B9
:10B410002BDE882351F04AE0BE016B5F7F4F83EB48
:10B4200090E40F944C588823F9F09B89993399F450
:10B430008A89893361F48989893321F410929A3396
:10B4400080E042C08F5F898BFA8AFB8AC9CFFB8A72
:10B450008F5F8A8BC5CF9F5F9B8BC2CF882321F0E4
:10B4600010929A3380E030C081E080939A33BE011D
:10B47000695F7F4FC6010F94D56681E025C080E0EB
:10B4800023C080E021C080E01FC07F926F925F9256
:10B490002F938EEE91E29F938F93CE0101969F930F
:10B4A0008F930F94F3668981898B8A818A8B8B8134
:10B4B0008B8B80E38D838AE38E83CDBFDEBFA114A7
:10B4C000B10409F07ECF88CF6896CDBFDEBFDF9193
:10B4D000CF911F910F91FF90EF90DF90CF90BF9091
:10B4E000AF907F906F905F904F900895DF92EF92B2
:10B4F000FF920F931F93CF93DF93CDB7DEB764977F
:10B50000CDBFDEBF8C0184E1EAE7F4E2DE011196F3
:10B5100001900D928A95E1F70115110509F449C0D2
:10B520006115710509F447C080E389838AE38A8342
:10B530004115510559F0DA01FE0134969E01285F4C
:10B540003F4F9D919193E217F307D9F77B010F2E9F
:10B55000F0E3DF2EF02D46E0BE016F5F7F4FC801A4
:10B560000F944C5899EF980F9230A8F49F85993317
:10B5700079F48E85893341F48D858933F1F08F5FBD
:10B580008D87DE86DF86E7CFDF868F5F8E87E3CF0E
:10B590009F5F9F87E0CF811112C081E1FE0133964A
:10B5A000D70101900D928A95E1F7F701118A81E0A8
:10B5B00007C080E005C080E003C080E001C080E0FB
:10B5C0006496CDBFDEBFDF91CF911F910F91FF90A9
:10B5D000EF90DF9008958091CA35089508950895F9
:10B5E00081E08093CA3508951092CA350895CF92AC
:10B5F000DF92EF92FF920F931F936623B9F08111B0
:10B600001DC0C12CD12C760100E010E62AEE30E0FE
:10B6100040E06CE170E280EB98E00F94AC446CE1A8
:10B6200070E280EB98E00F94F64408C0811106C0E8
:10B630006CE170E280EB98E00F940C451F910F9144
:10B64000FF90EF90DF90CF900895CF93DF931F92FC
:10B650001F92CDB7DEB78091CB359091CC35A091BC
:10B66000CD35B091CE35072E75E1B695A795979556
:10B6700087957A95D1F7702D61E0B9DF87ED8A83E0
:10B6800041E050E0BE016E5F7F4F80EB98E00F9489
:10B69000C74441E050E0BE016F5F7F4F80EB98E010
:10B6A0000F94DE4489818823A4F78091CB35909153
:10B6B000CC35A091CD35B091CE35072E75E1B6953C
:10B6C000A795979587957A95D1F7702D60E08FDFD4
:10B6D0000F900F90DF91CF91089580EB98E00F9439
:10B6E00075441092CF3581E008951F93CF93DF9377
:10B6F000CDB7DEB72C97CDBFDEBF6115710520E257
:10B700008207910508F0A1C0DC01CB018093CB3505
:10B710009093CC35A093CD35B093CE358091CF3575
:10B72000811193DF1092CF358091CB359091CC353C
:10B73000A091CD35B091CE35072E75E1B695A79580
:10B74000979587957A95D1F7702D61E050DF82ED5E
:10B750008C8741E050E0BE01645F7F4F80EB98E052
:10B760000F94C7448091CB359091CC35A091CD35C5
:10B77000B091CE35AC01BD01032E39E076956795C9
:10B78000579547953A95D1F7302D032E3AE0440F5F
:10B79000551F661F771F3A95D1F7302D9170AA2754
:10B7A000BB27842B952BA62BB72B89839A83AB833E
:10B7B000BC838B818D8341E050E0BE016B5F7F4F86
:10B7C00080EB98E00F94C7448A818E8341E050E07B
:10B7D000BE016A5F7F4F80EB98E00F94C744898178
:10B7E0008F8341E050E0BE01695F7F4F80EB98E0BE
:10B7F0000F94C74415E5188741E050E0BE01685F2B
:10B800007F4F80EB98E00F94C744198741E050E0E8
:10B81000BE01675F7F4F80EB98E00F94C7441A87A3
:10B8200041E050E0BE01665F7F4F80EB98E00F94EF
:10B83000C7441B8741E050E0BE01655F7F4F80EB4E
:10B8400098E00F94C74481E001C080E02C96CDBF02
:10B85000DEBFDF91CF911F910895052E59E0660F4D
:10B86000771F881F991F5A95D1F7502D61157105C3
:10B8700020E28207910510F438CF089580E0089502
:10B880008091CB359091CC35A091CD35B091CE350E
:10B890000097A105B10569F00197A109B109072E2B
:10B8A00075E1B695A795979587957A95D1F7702DFF
:10B8B00001C080E060E09BDE1092CF350895CF9309
:10B8C000DF93CDB7DEB72897CDBFDEBF6115710519
:10B8D00020E28207910508F078C0DC01CB0180935B
:10B8E000CB359093CC35A093CD35B093CE358091A8
:10B8F000CF358111AADE1092CF358091CB35909152
:10B90000CC35A091CD35B091CE35072E75E1B695E9
:10B91000A795979587957A95D1F7702D61E067DEA9
:10B9200082E8888741E050E0BE01685F7F4F80EB8E
:10B9300098E00F94C7448091CB359091CC35A0917D
:10B94000CD35B091CE35AC01BD01032E39E07695F1
:10B950006795579547953A95D1F7302D032E3AE0E4
:10B96000440F551F661F771F3A95D1F7302D917000
:10B97000AA27BB27842B952BA62BB72B89839A83C9
:10B98000AB83BC838B818D8341E050E0BE016B5F54
:10B990007F4F80EB98E00F94C7448A818E8341E00B
:10B9A00050E0BE016A5F7F4F80EB98E00F94C74480
:10B9B00089818F8341E050E0BE01695F7F4F80EB5A
:10B9C00098E00F94C74481E001C080E02896CDBF85
:10B9D000DEBFDF91CF910895CF93DF931F92CDB754
:10B9E000DEB78091CB359091CC35A091CD35B0911B
:10B9F000CE35AC01BD01517066277727452B462B0C
:10BA0000472B31F1198241E050E0BE016F5F7F4F5B
:10BA100080EB98E00F94C7448091CB359091CC3562
:10BA2000A091CD35B091CE350196A11DB11D809369
:10BA3000CB359093CC35A093CD35B093CE35AC01BA
:10BA4000BD01517066277727452B462B472BD1F632
:10BA50000097A105B10569F00197A109B109072E69
:10BA600075E1B695A795979587957A95D1F7702D3D
:10BA700001C080E060E0BBDD81E08093CF350F90B6
:10BA8000DF91CF9108950F931F93CF93DF931F9270
:10BA9000CDB7DEB78091CF358823B1F01092CF3586
:10BAA0008091CB359091CC35A091CD35B091CE35EC
:10BAB000BC01CD01052E59E0969587957795679540
:10BAC0005A95D1F7502DC9DE41E050E0BE016F5FBD
:10BAD0007F4F80EB98E00F94DE448091CB359091BE
:10BAE000CC35A091CD35B091CE35AC01BD014F5FC5
:10BAF0005F4F6F4F7F4F4093CB355093CC35609362
:10BB0000CD357093CE358A019B01117022273327E2
:10BB1000012B022B032BA1F4452B462B472B51F075
:10BB2000072E75E1B695A795979587957A95D1F7E4
:10BB3000702D01C080E060E05ADD81E08093CF3558
:10BB400089810F90DF91CF911F910F9108950F93ED
:10BB50001F93CF93DF931F92CDB7DEB7182F80913D
:10BB6000CF35882349F06091CB357091CC358091E9
:10BB7000CD359091CE35A3DE198341E050E0BE0172
:10BB80006F5F7F4F80EB98E00F94C7448091CB3577
:10BB90009091CC35A091CD35B091CE35AC01BD01A1
:10BBA0004F5F5F4F6F4F7F4F4093CB355093CC35F6
:10BBB0006093CD357093CE358A019B011170222799
:10BBC0003327012B022B032BA1F4452B462B472BAC
:10BBD00051F0072E75E1B695A795979587957A95BB
:10BBE000D1F7702D01C080E060E001DD81E080933D
:10BBF000CF3581E00F90DF91CF911F910F91089584
:10BC0000CF93DF931F921F92CDB7DEB78091CF35D0
:10BC1000882309F440C08091CB359091CC35A09118
:10BC2000CD35B091CE35072E75E1B695A795979590
:10BC300087957A95D1F7702D61E0D9DC87ED8A83FD
:10BC400041E050E0BE016E5F7F4F80EB98E00F94C3
:10BC5000C74441E050E0BE016F5F7F4F80EB98E04A
:10BC60000F94DE448091CB359091CC35A091CD35A9
:10BC7000B091CE35072E75E1B695A7959795879526
:10BC80007A95D1F7702D60E0B2DC89818095881FAC
:10BC90008827881F01C080E00F900F90DF91CF911F
:10BCA0000895CF93DF93EC01803C28E0920729F4BC
:10BCB00068E083E00F94F64310C0803C29E09207CF
:10BCC00029F468E084E00F94F64307C0803C9A4072
:10BCD00021F468E085E00F94F643888180618883D1
:10BCE000DF91CF910895EF92FF920F931F93CF931F
:10BCF0007C01C42FB901A80100E010E62AEE30E073
:10BD00000E94A768882344F0F7018081CC0FCC0FF4
:10BD1000CC70837FC82BC083CF911F910F91FF9070
:10BD2000EF90089580E0089591E0811101C090E0C6
:10BD30009093D34081E08093442008950F931F9304
:10BD400002E710E62FE130E040E156E361E082E0F7
:10BD50000E942A79811105C06EE97EE582E00E9489
:10BD60007A7A1F910F910895CF93DF931092F33554
:10BD70001092F4350F942245811104C010920C36B4
:10BD8000D0E012C0815080930C362ADCD82F882353
:10BD900059F0C0E060E08C2F0F943845CF5F809160
:10BDA0000C368C17B8F7CADF8D2FDF91CF9108952D
:10BDB000C5CF08950F931F9308ED1EE52DE030E0E9
:10BDC00048E450E260E081E80E942A79811105C0D0
:10BDD0006AED7EE581E80E947A7A1F910F910895BD
:10BDE0008091F435882341F082E00E94537A60EF1D
:10BDF0007EE582E00C947A7A08958091F435882368
:10BE000041F081E80E94537A6DEF7EE581E80C9461
:10BE10007A7A08958091502090915120A0915220DB
:10BE2000B0915320892B8A2B8B2B59F080911C3693
:10BE3000882324F481E80E94537A03C082E00E94A0
:10BE4000537A8091143690911536A0911636B091A0
:10BE5000173680934C2090934D20A0934E20B093A2
:10BE60004F20A8CF0895E8EFF5E382E1DF011D92AE
:10BE70008A95E9F780EF80838AE087830895DF92CF
:10BE8000EF92FF920F931F93CF93DF93D82EC62F7D
:10BE9000D72F122F032FF42EE52EE5DF81E08093BC
:10BEA0005420E8EFF5E3D282E382F482058316831F
:10BEB000D487C587DF91CF911F910F91FF90EF90AD
:10BEC000DF90089520E030E0A90160E074E285E0B1
:10BED000D6CF08950F931F9320911C3642276CF004
:10BEE00000915020109151202091522030915320E8
:10BEF000061717072807390720F4E4DF8BDF80E0F7
:10BF000001C081E01F910F91089520E030E0A90168
:10BF100060E070E084E0B3CF08950F931F93262F65
:10BF200030E003EB1FE5AC0161E081E80E942A7973
:10BF3000811102C0EADF6EDF1F910F91089520E0AA
:10BF400030E0A90160E078E286E099CF089520E032
:10BF500030E0A90160E07AE382E091CF089583DFC9
:10BF6000109254200895CF93DF93811111C0EB01FB
:10BF7000F6DFE8E4F0E280859185A285B3858C1B2D
:10BF80009D0BA109B10980879187A287B38742DF02
:10BF9000DF91CF9108951F93CF93DF93D82F84E142
:10BFA000E8EDF5E3DF011D928A95E9F7DD2331F035
:10BFB00090912736E0EEF5E318E005C09091233626
:10BFC000ECEDF5E314E0809121368F738C3111F0A4
:10BFD0008F3339F48CE180838AE0818385E0838329
:10BFE000145FC12F911708F4C92F8C2F90E0A0E0A7
:10BFF000B0E040E8BC01CD016DDF882309F18091FC
:10C000001D360F943F45811102C020E001C020E899
:10C01000DD2361F0E8EDF5E3812F90E002979827AA
:10C020008927982780839183238306C0E8EDF5E371
:10C030008FEF810F808322836C2F88ED95E36DDF76
:10C04000DF91CF911F910895CF93C82F81110FC019
:10C0500080911D360F943F45882349F020E030E061
:10C06000A90160E077E287E00ADFD4DE39C0AEEEF6
:10C07000B5E3E0E1F6E3818913968C931397828907
:10C0800012968C931297838911968C9311978489B9
:10C090008C93ACEEB5E3868911968C9311978789C2
:10C0A0008C936091EC357091ED35CB01A0E0B0E060
:10C0B000BC01CD01052E59E0660F771F881F991F1F
:10C0C0005A95D1F7502DC11102C040E001C040E89F
:10C0D00001DF882329F0C093F23581E08093F335A6
:10C0E000CF9108950F931F93CF93DF93811132C1A6
:10C0F0006F31710569F48091103690911136A091DD
:10C100001236B091133685359345A244B34431F0CD
:10C1100081E08093F43564DE70DE1CC1E0E1F6E37B
:10C1200095859F70958780910C36891718F4CADE23
:10C1300071DE10C1E0E1F6E34085518562857385CB
:10C14000409350205093512060935220709353207D
:10C15000478550E04B35510508F0EEC0FA018827BD
:10C16000E958FE4F8F4F0D94C664C0912336C331FA
:10C1700008F0C2E18C2F90E0A0E0B0E040E8BC0104
:10C18000CD01A8DE882309F4E5C06C2F88EF95E384
:10C19000C4DEE0C0C0912336C53208F0C4E28C2F63
:10C1A00090E0A0E0B0E040E8BC01CD0193DE882340
:10C1B00009F4D0C080912036837021F4D0912136CB
:10C1C000DD2319F07FDE26DEC5C080911D360F9479
:10C1D00046458111D0E800E210E2F801D183809158
:10C1E0001D360F944D4520E1FC013196A0E3B0E2ED
:10C1F00001900D922A95E1F7F8018089882309F4CE
:10C20000A4C0823209F4A3C0E1E3F0E281E091919D
:10C21000992309F49DC0923209F49AC08F5F80314E
:10C22000B1F708C0E82FF0E0E05EFF4D908B8F5F24
:10C230008031C1F76C2F80E290E26FDE8BC080E02E
:10C24000AADE88C081E0A7DE85C0892F0F9424452F
:10C25000823039F0833019F0811105C006C06FDEDD
:10C2600005C075DE03C051DE01C079DED3DD72C0CA
:10C2700040E868E070E080E090E02CDE882309F47C
:10C2800069C060ED75E380911D360F942B458230B7
:10C2900041F0833019F0811107C009C050DEBADDCA
:10C2A00059C055DEB7DD56C030DEB4DD53C0E0ED19
:10C2B000F5E380E090E0A2E0B0E084839583A6837C
:10C2C000B78380819181A281B3815A2F4B2F60E087
:10C2D00070E0982789279827A0E0B0E0DC01992733
:10C2E0008827842B952BA62BB72B80839183A28341
:10C2F000B38368E0CF0111DE2DC08091233681FF2A
:10C3000006C08095682F6170892F0F94384527DE0D
:10C3100081DD20C080912336811102C020DE01C062
:10C32000D1DD78DD17C01BDE75DD14C081E08CDE49
:10C3300011C080E089DE0EC020E030E0A90160E09D
:10C3400070E285E09CDD66DD05C080E001C080E034
:10C3500090E268CFDF91CF911F910F9108951092D5
:10C36000F33542C908958091DC408823F4F4807647
:10C370008032D9F58091DD408E3FC9F58091E24051
:10C380009091E3400197A9F58091DE409091DF40C4
:10C39000892B89F5ECEDF0E48CE096E380879187BA
:10C3A00081E090E08287938708958076803229F536
:10C3B0008091DD408F3F19F58091E2409091E340FC
:10C3C000892BF9F48091DE409091DF40892BD9F4DC
:10C3D0001092F4351092F33582E00E94E87981E8FA
:10C3E0000E94E879ABDC81E0089580E0089580E068
:10C3F000089580E0089580E0089580E0089580E049
:10C40000089580E0089580E00895CF93C091F335BA
:10C41000CC23A9F11092F3358091F235882389F06D
:10C420002091EC353091ED354091EE355091EF355E
:10C430006091F0357091F13580911D360F9455451E
:10C4400010C02091EC353091ED354091EE35509192
:10C45000EF356091F0357091F13580911D360F9474
:10C460007945823041F0833021F0811106C077DDBB
:10C4700005C065DD03C06BDD01C047DDCBDC8C2F63
:10C48000CF910895EF92FF920F931F93CF93DF9375
:10C49000982F80914420882309F448C010924420AA
:10C4A0002115310511F0890102C004E91EE5911141
:10C4B00002C082E001C081E8E9017A01AB01970185
:10C4C00060E00E942A79811104C091E09093442099
:10C4D0002DC0CD2BD9F4809144208823E1F38091A5
:10C4E000D340811122C0E8E4F0E280859185A285E5
:10C4F000B3858E199F09A109B10980879187A28709
:10C50000B3879091D34081E0892710C0E8E4F0E23E
:10C5100040855185628573854E195F0961097109EE
:10C52000408751876287738701C080E0DF91CF9198
:10C530001F910F91FF90EF900895E0913536F091A3
:10C5400036360190F081E02D228133812E0F3F1F7E
:10C55000FC014081E40FF11DE217F307A0F4818193
:10C560008430A1F0861306C014C081818430A1F00C
:10C570008617A9F08081E80FF11DE217F307A8F3F1
:10C5800080E090E0089580E090E0089580E090E001
:10C5900008958E2F9F2F089580E090E008958E2FAC
:10C5A0009F2F08958091DE408F770C9445780895F1
:10C5B00090913736992381F1E0913536F0913636F6
:10C5C0000190F081E02D9481891740F5E093333696
:10C5D000F0933436228133812E0F3F1FE217F30789
:10C5E000F8F49181943061F49281891309C09381A8
:10C5F000961306C0E0933336F093343681E0089505
:10C600009081E90FF11DE217F30758F3E0933336F9
:10C61000F093343680E0089580E0089580E0089536
:10C6200080E00895EF92FF921F93CF93DF93C82F7E
:10C6300060E0BEDF182F882381F1A0913536B091DC
:10C640003636EC2FF0E0EE0FFF1F12968D919C9185
:10C650001397E80FF91FE080F180D7011696ED914E
:10C66000FC9117971995682F8C2FA2DF182F88231C
:10C67000A1F0C0913336D091343665E0CE015DDF54
:10C68000EC01892B21F08A810E94377AF6CFD701FD
:10C690001296ED91FC9113971995812FDF91CF910F
:10C6A0001F91FF90EF9008951F93CF93DF93182F62
:10C6B0007FDF882341F1C0913336D091343665E075
:10C6C000CE013BDFEC01892B49F04C815D816B8110
:10C6D0008A810E9452788111F2CF15C0A09135361F
:10C6E000B0913636E12FF0E0EE0FFF1F12968D91DC
:10C6F0009C911397E80FF91F0190F081E02D0190B4
:10C70000F081E02D1995DF91CF911F9108950C9440
:10C71000DD770895CF93809137368823C1F0E0917B
:10C720003536F09136360190F081E02D84818823F2
:10C7300071F0C0E08C2F76DFCF5FE0913536F0915D
:10C7400036360190F081E02D8481C81798F310925D
:10C75000373681E090E08093383690933936CF9128
:10C7600008950E94A977D6CF0895CF938091373648
:10C77000882349F1A0913536B0913636ED91FC9180
:10C78000119784818823F9F0C0E0EC2FF0E0EE0FE0
:10C79000FF1F12968D919C911397E80FF91F01903E
:10C7A000F081E02D0084F185E02D309709F0199596
:10C7B000CF5FA0913536B0913636ED91FC9111974F
:10C7C0008481C81710F3CF9108950F931F93CF93CF
:10C7D000DF93ECEDF0E41286138614861586168638
:10C7E0001786808188230CF060C22091E24030914E
:10C7F000E3402115310509F05DC24FC28F7109F088
:10C8000097C09091DD40963081F0983009F485C052
:10C8100091118EC02230310509F0FBC162E070E059
:10C8200088E396E30E944B784EC28091DE4090915F
:10C83000DF40292F33272230310589F0233031059D
:10C8400079F12130310509F0A6C1809162209091E3
:10C850006320DC016C9170E00E944B784FC0E09146
:10C860006220F09163202189821708F0D2C19927B4
:10C87000880F991F880F991FE0916420F09165201F
:10C88000E80FF91F80819181FC01628173810E9410
:10C890004B78E091E440F091E54082E081832EC046
:10C8A00099278130910599F058F08230910509F46B
:10C8B00006C2039709F078C13CE0EEE8F4E20AC052
:10C8C00064E070E088EC90E20E944B7817C0EEEBD9
:10C8D000F0E239E0A2EAB0E220E0819190E08D93AD
:10C8E0009D932F5F2317C8F3632F660F6E5F6093CE
:10C8F000A02070E080EA90E20E944B78ECEDF0E43A
:10C9000086819781228533858217930708F0DBC1E2
:10C910008093E6409093E740D6C12130310509F07D
:10C9200078C161E070E087E396E30E944B78CBC169
:10C930008130E9F59091DD409A30C9F5213031051B
:10C9400009F037C180913736882309F432C1C0918C
:10C95000E040D091E1400091353610913636D80153
:10C96000ED91FC918481C81708F023C160E08C2F01
:10C970001FDE882309F418C1CE019927880F991F5B
:10C98000D8011296ED91FC911397E80FF91F0190D1
:10C99000F081E02D86819781FC01199580933236D4
:10C9A00061E070E082E396E30E944B788CC18230B4
:10C9B00009F0FAC08091DD408111EFC022303105CD
:10C9C00009F027C18091E0400E94DA7890E08093DE
:10C9D00030369093313662E070E080E396E30E9457
:10C9E0004B7871C18F7109F084C09091DD40933014
:10C9F00009F4D5C018F49130A1F07BC0953019F03E
:10CA0000993039F176C08091E2409091E340892BD2
:10CA100009F0FFC082ED92E68093E8409093E940F0
:10CA200052C18091E2409091E340892B09F0F1C01E
:10CA30008091DE409091DF40019709F0EAC080913B
:10CA40003836909139368D7F8093383690933936C9
:10CA50003AC18091E2409091E340892B09F0D9C01E
:10CA60000E944878882309F49FC02091DE403091CD
:10CA7000DF403327E0916220F0916320818990E0CC
:10CA80008217930708F490C045DE8091DE409091B4
:10CA9000DF4080933736882309F415C199278150E8
:10CAA000904C880F991F880F991FE0916420F09196
:10CAB0006520E80FF91FE0933536F0933636019084
:10CAC000F081E02D8481882309F4FDC0C0E060E09E
:10CAD0008C2FEADD882309F467C0CF5FE0913536FB
:10CAE000F09136360190F081E02D8481C81778F3FB
:10CAF000EAC08130E9F49091DD409B30C9F4809127
:10CB0000E2409091E340892B09F053C08091373681
:10CB1000882309F44EC0ECEDF0E4C481D2818C2F5F
:10CB200081DD882309F440C06D2F8C2FBDDD3AC014
:10CB30008230D1F58091DD40813019F08330A1F051
:10CB400030C08091E2409091E340892B09F061C0B0
:10CB50008091DE409091DF40892B09F05AC080918E
:10CB6000E0400E94F5781EC08091E2409091E34041
:10CB7000892B09F04EC08091DE409091DF40892BD7
:10CB800009F047C0CCEDD0E48C810E94E8798C811B
:10CB90000E94537A07C080E005C080E003C080E0B7
:10CBA00001C080E0811190C08091DC408F718130A4
:10CBB00081F580913736882309F471C00091E040F7
:10CBC0001091E140C0913536D0913636E881F98137
:10CBD0008481081708F065C060E0802FE9DC8823B5
:10CBE000C1F0F801FF27CF01880F991FEA81FB816F
:10CBF000E80FF91FC081D181EE81FF811995682F5F
:10CC0000802FD6DC882329F0EC81FD8119958111D4
:10CC10005BC08091DC408F71823009F044C080910C
:10CC200037368823B1F1A0913536B0913636ED9183
:10CC3000FC9111978481882371F1C0E0EC2FF0E022
:10CC4000EE0FFF1F12968D919C911397E80FF91F1D
:10CC500000811181D8011696ED91FC9117971995D5
:10CC6000682F8C2FA5DC882379F1D8011496ED91DB
:10CC7000FC9115971995811127C0CF5FA09135368A
:10CC8000B0913636ED91FC9111979481C917B0F2AD
:10CC90001BC080E019C080E017C080E015C080E0B4
:10CCA00013C080E011C080E00FC0982F907609F08B
:10CCB0007BCF98CE982F907609F076CF9FCD33E03A
:10CCC000EAEBF0E207CE81E0DF91CF911F910F9167
:10CCD00008958038910558F1672B21F4873C910520
:10CCE00071F41CC08F3F910509F0F8F49C01220FEC
:10CCF000331FF901E55AF84D808191810895EDE5E2
:10CD0000F8E221E030E0419151918417950741F01C
:10CD10002F5F3F4F20383105B1F702C020E030E0EF
:10CD200020583F4FC9019927089580E090E0089569
:10CD30008136910589F0EDE7F6E240E050E04F5F83
:10CD40005F4F219131912115310591F02817390755
:10CD5000B1F7892B19F40AC040E050E0440F551F89
:10CD6000FA01E556FB4D80819181089580E090E0C5
:10CD7000089543E050E060E880E096E00F944E4470
:10CD800043E050E064E080E296E00F944E4443E0DC
:10CD900050E062E080E296E00F944E4440E058E1BB
:10CDA00060E280EA96E00F944E4441E050E062E099
:10CDB00080EA96E00F944E4443E050E060E180E862
:10CDC00096E00F944E4443E050E060E180E496E04A
:10CDD0000F944E4441E050E061E080E496E00F940F
:10CDE0004E4441E050E062E080E496E00F944E440F
:10CDF00041E050E060E280E696E00F944E4441E06E
:10CE000050E062E080E096E00F944E4443E050E052
:10CE100062E080E696E00F944E4440E050E061E02E
:10CE200080EA96E00F944E4440E050E061E080E0FC
:10CE300096E00F944E4440E050E068E080E096E0D9
:10CE40000F944E4441E050E060E480E096E00F949F
:10CE50004E4440E058E161E080E896E00F944E4493
:10CE600040E050E061E080E096E00F944E4440E006
:10CE700050E060E280E096E00F944E4440E050E0E5
:10CE800064E080E096E00F944E4440E050E061E0C2
:10CE900080EA96E00F944E4443E050E060E880E47E
:10CEA00096E00F944E4443E050E060E280E496E068
:10CEB0000F944E4440E050E060E480E496E00F942C
:10CEC0004E4441E050E060E880E896E00F944E4424
:10CED00041E050E060E280E896E00F944E4440E08C
:10CEE00050E060E480E896E00F944E4443E050E068
:10CEF00068E080E496E00F944E4440E050E064E047
:10CF000080E496E00F944E4443E050E068E080E611
:10CF100096E00F944E4440E050E064E080E696E0F6
:10CF20000F944E4443E050E068E080E896E00F94B0
:10CF30004E4440E050E064E080E896E00F944E44B8
:10CF400043E050E068E080EA96E00F944E4440E011
:10CF500050E064E080EA96E00F944E4440E058E1EF
:10CF600060E480EA96E00F944E4440E058E160E1CE
:10CF700080E696E00F944E4440E058E161E080E2A4
:10CF800096E00F944E4443E050E060E880E496E081
:10CF90000F944E4443E050E060E280E496E00F944A
:10CFA0004E4440E050E060E480E496E00F944E444C
:10CFB00043E050E060E880EA96E00F944E4443E09E
:10CFC00050E060E880E496E00F944E4443E050E087
:10CFD00060E280E496E00F944E4440E050E060E46C
:10CFE00080E496E00F944E4443E050E068E080E235
:10CFF00096E00F944E4441E050E062E080E896E015
:10D000000F944E4440E050E061E080E696E00F94DB
:10D010004E4440E050E060E180E096E00D944E44E4
:10D0200008951F920F920FB60F9211240BB60F9214
:10D030008F939F93EF93FF93E4EDF0E480819181D0
:10D04000019680839183FF91EF919F918F910F9033
:10D050000BBE0F900FBE0F901F9018951F920F924E
:10D060000FB60F9211240BB60F92CF92DF92EF9270
:10D07000FF920F931F932F933F934F935F936F9361
:10D080007F938F939F93AF93BF93EF93FF93E4EDC1
:10D09000F0E4808191812281338182179307F0F13E
:10D0A00021E020930204E091DA40F091DB403097D8
:10D0B000A9F16091080470910904A0E0B0E0DC01DE
:10D0C00099278827AB0160E070E08C019D01042B5B
:10D0D000152B262B372BC901B801A4EDB0E412960D
:10D0E0000D911C91139720E030E098011127002743
:10D0F0001496CD90DC901597E12CF12C0C291D296C
:10D100002E293F29061717072807390730F0C901CC
:10D11000B8016F5F7F4F8F4F9F4F1995FF91EF9130
:10D12000BF91AF919F918F917F916F915F914F913F
:10D130003F912F911F910F91FF90EF90DF90CF9033
:10D140000F900BBE0F900FBE0F901F901895CF92AF
:10D15000DF92EF92FF920F931F93CF93DF93EC0137
:10D160006A017B01DB01CA010197A109B109BC0178
:10D17000CD01600F711F821F931FA70196010F94AD
:10D1800088642138310541055105F8F4213460F4F3
:10D19000213260F4213160F4293060F4253060F4EC
:10D1A000233060F490E80BC093E009C092E007C020
:10D1B00092E805C091E003C091E801C090E0888149
:10D1C0008C77892B888381E001C08FEFDF91CF912D
:10D1D0001F910F91FF90EF90DF90CF9008951F92D5
:10D1E0000F920FB60F9211240BB60F922F933F930D
:10D1F0004F935F936F937F938F939F93AF93BF935F
:10D20000EF93FF93E0918036F0918136309709F0EB
:10D210001995FF91EF91BF91AF919F918F917F9160
:10D220006F915F914F913F912F910F900BBE0F9097
:10D230000FBE0F901F9018951F920F920FB60F926E
:10D2400011240BB60F922F933F934F935F936F93DD
:10D250007F938F939F93AF93BF93EF93FF93E0914F
:10D260007E36F0917F36309709F01995FF91EF9156
:10D27000BF91AF919F918F917F916F915F914F91EE
:10D280003F912F910F900BBE0F900FBE0F901F90EC
:10D2900018951F920F920FB60F9211240BB60F9292
:10D2A0002F933F934F935F936F937F938F939F93AE
:10D2B000AF93BF93EF93FF93E0917C36F0917D366F
:10D2C000309709F01995FF91EF91BF91AF919F9120
:10D2D0008F917F916F915F914F913F912F910F901F
:10D2E0000BBE0F900FBE0F901F9018951F920F92BC
:10D2F0000FB60F9211240BB60F922F933F934F93BB
:10D300005F936F937F938F939F93AF93BF93EF93AD
:10D31000FF93E0917A36F0917B36309709F01995BA
:10D32000FF91EF91BF91AF919F918F917F916F91FD
:10D330005F914F913F912F910F900BBE0F900FBEB9
:10D340000F901F9018951F920F920FB60F921124F5
:10D350000BB60F922F933F934F935F936F937F93EF
:10D360008F939F93AF93BF93EF93FF93E0917836A2
:10D37000F0917936309709F01995FF91EF91BF91AF
:10D38000AF919F918F917F916F915F914F913F915D
:10D390002F910F900BBE0F900FBE0F901F901895FE
:10D3A0001F920F920FB60F9211240BB60F922F936C
:10D3B0003F934F935F936F937F938F939F93AF931D
:10D3C000BF93EF93FF93E0917636F09177363097E5
:10D3D00009F01995FF91EF91BF91AF919F918F91B6
:10D3E0007F916F915F914F913F912F910F900BBE65
:10D3F0000F900FBE0F901F9018951F920F920FB6AF
:10D400000F9211240BB60F922F933F934F935F937C
:10D410006F937F938F939F93AF93BF93EF93FF93FC
:10D42000E0917436F0917536309709F01995FF91B7
:10D43000EF91BF91AF919F918F917F916F915F918C
:10D440004F913F912F910F900BBE0F900FBE0F90F9
:10D450001F9018951F920F920FB60F9211240BB6C2
:10D460000F922F933F934F935F936F937F938F937D
:10D470009F93AF93BF93EF93FF93E0917236F09138
:10D480007336309709F01995FF91EF91BF91AF91E5
:10D490009F918F917F916F915F914F913F912F91CC
:10D4A0000F900BBE0F900FBE0F901F9018951F92FC
:10D4B0000F920FB60F9211240BB60F922F933F933A
:10D4C0004F935F936F937F938F939F93AF93BF938C
:10D4D000EF93FF93E0917036F0917136309709F039
:10D4E0001995FF91EF91BF91AF919F918F917F918E
:10D4F0006F915F914F913F912F910F900BBE0F90C5
:10D500000FBE0F901F9018951F920F920FB60F929B
:10D5100011240BB60F922F933F934F935F936F930A
:10D520007F938F939F93AF93BF93EF93FF93E0917C
:10D530006E36F0916F36309709F01995FF91EF91A3
:10D54000BF91AF919F918F917F916F915F914F911B
:10D550003F912F910F900BBE0F900FBE0F901F9019
:10D5600018951F920F920FB60F9211240BB60F92BF
:10D570002F933F934F935F936F937F938F939F93DB
:10D58000AF93BF93EF93FF93E0916C36F0916D36BC
:10D59000309709F01995FF91EF91BF91AF919F914D
:10D5A0008F917F916F915F914F913F912F910F904C
:10D5B0000BBE0F900FBE0F901F9018951F920F92E9
:10D5C0000FB60F9211240BB60F922F933F934F93E8
:10D5D0005F936F937F938F939F93AF93BF93EF93DB
:10D5E000FF93E0916A36F0916B36309709F0199508
:10D5F000FF91EF91BF91AF919F918F917F916F912B
:10D600005F914F913F912F910F900BBE0F900FBEE6
:10D610000F901F9018951F920F920FB60F92112422
:10D620000BB60F922F933F934F935F936F937F931C
:10D630008F939F93AF93BF93EF93FF93E0916836DF
:10D64000F0916936309709F01995FF91EF91BF91EC
:10D65000AF919F918F917F916F915F914F913F918A
:10D660002F910F900BBE0F900FBE0F901F9018952B
:10D670001F920F920FB60F9211240BB60F922F9399
:10D680003F934F935F936F937F938F939F93AF934A
:10D69000BF93EF93FF93E0916636F0916736309732
:10D6A00009F01995FF91EF91BF91AF919F918F91E3
:10D6B0007F916F915F914F913F912F910F900BBE92
:10D6C0000F900FBE0F901F9018951F920F920FB6DC
:10D6D0000F9211240BB60F922F933F934F935F93AA
:10D6E0006F937F938F939F93AF93BF93EF93FF932A
:10D6F000E0916436F0916536309709F01995FF9105
:10D70000EF91BF91AF919F918F917F916F915F91B9
:10D710004F913F912F910F900BBE0F900FBE0F9026
:10D720001F9018951F920F920FB60F9211240BB6EF
:10D730000F922F933F934F935F936F937F938F93AA
:10D740009F93AF93BF93EF93FF93E0916236F09175
:10D750006336309709F01995FF91EF91BF91AF9122
:10D760009F918F917F916F915F914F913F912F91F9
:10D770000F900BBE0F900FBE0F901F9018951F9229
:10D780000F920FB60F9211240BB60F922F933F9367
:10D790004F935F936F937F938F939F93AF93BF93B9
:10D7A000EF93FF93E0916036F0916136309709F086
:10D7B0001995FF91EF91BF91AF919F918F917F91BB
:10D7C0006F915F914F913F912F910F900BBE0F90F2
:10D7D0000FBE0F901F9018951F920F920FB60F92C9
:10D7E00011240BB60F922F933F934F935F936F9338
:10D7F0007F938F939F93AF93BF93EF93FF93E091AA
:10D800005E36F0915F36309709F01995FF91EF91F0
:10D81000BF91AF919F918F917F916F915F914F9148
:10D820003F912F910F900BBE0F900FBE0F901F9046
:10D8300018951F920F920FB60F9211240BB60F92EC
:10D840002F933F934F935F936F937F938F939F9308
:10D85000AF93BF93EF93FF93E0915C36F0915D3609
:10D86000309709F01995FF91EF91BF91AF919F917A
:10D870008F917F916F915F914F913F912F910F9079
:10D880000BBE0F900FBE0F901F9018951F920F9216
:10D890000FB60F9211240BB60F922F933F934F9315
:10D8A0005F936F937F938F939F93AF93BF93EF9308
:10D8B000FF93E0915A36F0915B36309709F0199555
:10D8C000FF91EF91BF91AF919F918F917F916F9158
:10D8D0005F914F913F912F910F900BBE0F900FBE14
:10D8E0000F901F9018951F920F920FB60F92112450
:10D8F0000BB60F922F933F934F935F936F937F934A
:10D900008F939F93AF93BF93EF93FF93E09158361C
:10D91000F0915936309709F01995FF91EF91BF9129
:10D92000AF919F918F917F916F915F914F913F91B7
:10D930002F910F900BBE0F900FBE0F901F90189558
:10D940001F920F920FB60F9211240BB60F922F93C6
:10D950003F934F935F936F937F938F939F93AF9377
:10D96000BF93EF93FF93E0915636F091573630977F
:10D9700009F01995FF91EF91BF91AF919F918F9110
:10D980007F916F915F914F913F912F910F900BBEBF
:10D990000F900FBE0F901F9018951F920F920FB609
:10D9A0000F9211240BB60F922F933F934F935F93D7
:10D9B0006F937F938F939F93AF93BF93EF93FF9357
:10D9C000E0915436F0915536309709F01995FF9152
:10D9D000EF91BF91AF919F918F917F916F915F91E7
:10D9E0004F913F912F910F900BBE0F900FBE0F9054
:10D9F0001F9018951F920F920FB60F9211240BB61D
:10DA00000F922F933F934F935F936F937F938F93D7
:10DA10009F93AF93BF93EF93FF93E0915236F091B2
:10DA20005336309709F01995FF91EF91BF91AF915F
:10DA30009F918F917F916F915F914F913F912F9126
:10DA40000F900BBE0F900FBE0F901F9018951F9256
:10DA50000F920FB60F9211240BB60F922F933F9394
:10DA60004F935F936F937F938F939F93AF93BF93E6
:10DA7000EF93FF93E0915036F0915136309709F0D3
:10DA80001995FF91EF91BF91AF919F918F917F91E8
:10DA90006F915F914F913F912F910F900BBE0F901F
:10DAA0000FBE0F901F9018951F920F920FB60F92F6
:10DAB00011240BB60F922F933F934F935F936F9365
:10DAC0007F938F939F93AF93BF93EF93FF93E091D7
:10DAD0004E36F0914F36309709F01995FF91EF913E
:10DAE000BF91AF919F918F917F916F915F914F9176
:10DAF0003F912F910F900BBE0F900FBE0F901F9074
:10DB000018951F920F920FB60F9211240BB60F9219
:10DB10002F933F934F935F936F937F938F939F9335
:10DB2000AF93BF93EF93FF93E0914C36F0914D3656
:10DB3000309709F01995FF91EF91BF91AF919F91A7
:10DB40008F917F916F915F914F913F912F910F90A6
:10DB50000BBE0F900FBE0F901F9018951F920F9243
:10DB60000FB60F9211240BB60F922F933F934F9342
:10DB70005F936F937F938F939F93AF93BF93EF9335
:10DB8000FF93E0914A36F0914B36309709F01995A2
:10DB9000FF91EF91BF91AF919F918F917F916F9185
:10DBA0005F914F913F912F910F900BBE0F900FBE41
:10DBB0000F901F9018951F920F920FB60F9211247D
:10DBC0000BB60F922F933F934F935F936F937F9377
:10DBD0008F939F93AF93BF93EF93FF93E09148365A
:10DBE000F0914936309709F01995FF91EF91BF9167
:10DBF000AF919F918F917F916F915F914F913F91E5
:10DC00002F910F900BBE0F900FBE0F901F90189585
:10DC10001F920F920FB60F9211240BB60F922F93F3
:10DC20003F934F935F936F937F938F939F93AF93A4
:10DC3000BF93EF93FF93E0914636F09147363097CC
:10DC400009F01995FF91EF91BF91AF919F918F913D
:10DC50007F916F915F914F913F912F910F900BBEEC
:10DC60000F900FBE0F901F9018951F920F920FB636
:10DC70000F9211240BB60F922F933F934F935F9304
:10DC80006F937F938F939F93AF93BF93EF93FF9384
:10DC9000E0914436F0914536309709F01995FF919F
:10DCA000EF91BF91AF919F918F917F916F915F9114
:10DCB0004F913F912F910F900BBE0F900FBE0F9081
:10DCC0001F9018951F920F920FB60F9211240BB64A
:10DCD0000F922F933F934F935F936F937F938F9305
:10DCE0009F93AF93BF93EF93FF93E0914236F091F0
:10DCF0004336309709F01995FF91EF91BF91AF919D
:10DD00009F918F917F916F915F914F913F912F9153
:10DD10000F900BBE0F900FBE0F901F9018951F9283
:10DD20000F920FB60F9211240BB60F922F933F93C1
:10DD30004F935F936F937F938F939F93AF93BF9313
:10DD4000EF93FF93E0914036F0914136309709F020
:10DD50001995FF91EF91BF91AF919F918F917F9115
:10DD60006F915F914F913F912F910F900BBE0F904C
:10DD70000FBE0F901F9018951F920F920FB60F9223
:10DD800011240BB60F922F933F934F935F936F9392
:10DD90007F938F939F93AF93BF93EF93FF93E09104
:10DDA0003E36F0913F36309709F01995FF91EF918B
:10DDB000BF91AF919F918F917F916F915F914F91A3
:10DDC0003F912F910F900BBE0F900FBE0F901F90A1
:10DDD00018951F920F920FB60F9211240BB60F9247
:10DDE0002F933F934F935F936F937F938F939F9363
:10DDF000AF93BF93EF93FF93E0913C36F0913D36A4
:10DE0000309709F01995FF91EF91BF91AF919F91D4
:10DE10008F917F916F915F914F913F912F910F90D3
:10DE20000BBE0F900FBE0F901F9018951F920F9270
:10DE30000FB60F9211240BB60F922F933F934F936F
:10DE40005F936F937F938F939F93AF93BF93EF9362
:10DE5000FF93E0913A36F0913B36309709F01995EF
:10DE6000FF91EF91BF91AF919F918F917F916F91B2
:10DE70005F914F913F912F910F900BBE0F900FBE6E
:10DE80000F901F901895CF93CFB7F894282F392F64
:10DE9000211588E0380749F461E083E00F94F643E8
:10DEA00064E083E00F94F6434FC0203488E03807E5
:10DEB00049F462E083E00F94F64364E083E00F945A
:10DEC000F64342C0211589E0380749F461E084E057
:10DED0000F94F64364E084E00F94F64335C0203499
:10DEE00089E0380749F462E084E00F94F64364E087
:10DEF00084E00F94F64328C021158AE0380749F4DE
:10DF000061E085E00F94F64364E085E00F94F6430A
:10DF10001BC020348AE0380749F462E085E00F94A2
:10DF2000F64364E085E00F94F6430EC021153B40B4
:10DF300049F461E086E00F94F64364E086E00F94D4
:10DF4000F64302C0CFBF01C0CFBFCF910895CF939A
:10DF5000CFB7F894282F392F211588E0380749F4D6
:10DF600061E083E00F94024464E083E00F94024494
:10DF70004FC0203488E0380749F462E083E00F9412
:10DF8000024464E083E00F94024442C0211589E01A
:10DF9000380749F461E084E00F94024464E084E0CF
:10DFA0000F94024435C0203489E0380749F462E018
:10DFB00084E00F94024464E084E00F94024428C09B
:10DFC00021158AE0380749F461E085E00F940244A6
:10DFD00064E085E00F9402441BC020348AE03807D7
:10DFE00049F462E085E00F94024464E085E00F9418
:10DFF00002440EC021153B4049F461E086E00F94D5
:10E00000024464E086E00F94024402C0CFBF01C026
:10E01000CFBFCF910895811528E0920729F460932E
:10E020008036709381360895803428E0920729F471
:10E0300060937436709375360895811529E09207C0
:10E0400029F460936C3670936D360895803429E01E
:10E05000920729F4609360367093613608958115B4
:10E060002AE0920729F46093583670935936089540
:10E0700080342AE0920729F460934C3670934D3631
:10E08000089581159B4021F4609344367093453682
:10E090000895FC01918195FFFDCF608380E090E0C1
:10E0A00008954F925F926F927F928F929F92AF925C
:10E0B000BF92EF92FF920F931F93CF937C014A017F
:10E0C0005B0128013901FC01848182FF16C0D9015E
:10E0D000C801689412F8B695A795979587951694F8
:10E0E000D1F7B901A801032E36E1769567955795CA
:10E0F00047953A95D1F7302D15C0D901C8016894DC
:10E1000013F8B695A795979587951694D1F7B90109
:10E11000A801032E37E176956795579547953A956F
:10E12000D1F7302D88159905AA05BB0508F4A6C0BE
:10E1300084169506A606B70608F4A2C0F7018481E6
:10E1400082FD04C0880C991CAA1CBB1CC301B2012F
:10E15000A50194010F9488642F3F310541055105B5
:10E1600008F490C08FEF90E0A0E0B0E0C9EF05C0E8
:10E17000281739074A075B0758F0880F991FAA1F0D
:10E18000BB1FCD3F0CF48160CF5FC73089F74FC014
:10E19000CC230CF04CC0D501C401880F991FAA1FD5
:10E1A000BB1F880F991FAA1FBB1F880F991FAA1F8B
:10E1B000BB1F481A590A6A0A7B0ACE3FF4F48DEF56
:10E1C0009FEF8C1B9109C7FD939504C0440C551C0F
:10E1D000661C771C8A95D2F7D501C401B695A79520
:10E1E00097958795BC01CD01640D751D861D971D02
:10E1F000A50194010F94886437C083E08C0FA501BA
:10E20000940104C0220F331F441F551F8A95D2F773
:10E21000DA01C901B695A79597958795BC01CD01FF
:10E22000640D751D861D971D0F9488641DC083E0C5
:10E230008C0FA501940104C0220F331F441F551FEA
:10E240008A95D2F7DA01C901B695A7959795879572
:10E25000BC01CD01640D751D861D971D0F9488644A
:10E260002150310941095109832F8F70C295C07F18
:10E27000C82BF701C783268381E018C080E016C051
:10E2800080E014C0D501C401880F991FAA1FBB1FCD
:10E29000880F991FAA1FBB1F880F991FAA1FBB1F9A
:10E2A000481A590A6A0A7B0AC9EF89CFCF911F9190
:10E2B0000F91FF90EF90BF90AF909F908F907F90C5
:10E2C0006F905F904F9008950F931F93CF93DF93BC
:10E2D000EC018B01009709F41EC1803C910529F4E3
:10E2E00060E180E00F94F64316C1C11584E0D807C1
:10E2F00029F464E080E00F94F6430DC1C038E1E0FA
:10E30000DE0729F462E080E00F94F64304C1C115F2
:10E31000F1E0DF0729F461E080E00F94F643FBC0F1
:10E32000C03883E0D80729F461E081E00F94F64318
:10E33000F2C0C039E3E0DE0729F461E082E00F9427
:10E34000F643E9C0C115F2E0DF0729F462E081E09D
:10E350000F94F643E0C0C03482E0D80729F462E0AD
:10E3600082E00F94F643D7C0C032E3E0DE0729F421
:10E3700064E082E00F94F643CEC0C115F8E0DF07F9
:10E3800029F461E083E00F94F643C5C0C11589E02C
:10E39000D80729F461E084E00F94F643BCC0C115AE
:10E3A000EAE0DE0729F461E085E00F94F643B3C0AC
:10E3B000C115FBE0DF0729F461E086E00F94F64326
:10E3C000AAC0C03488E0D80729F462E083E00F9443
:10E3D000F643A1C0C034E9E0DE0729F462E084E03E
:10E3E0000F94F64398C0C034FAE0DF0729F462E0E6
:10E3F00085E00F94F6438FC0C03988E0D80729F430
:10E4000064E083E00F94F64386C0C039E9E0DE079C
:10E4100029F464E084E00F94F6437DC0C039FAE04B
:10E42000DF0729F464E085E00F94F64374C0C03937
:10E430008BE0D80729F464E086E00F94F6436BC0C4
:10E44000C03CE8E0DE0729F468E083E00F94F6437F
:10E4500062C0C03CF9E0DF0729F468E084E00F9473
:10E46000F64359C0C03C8AE0D80729F468E085E04B
:10E470000F94F64350C0C03AE8E0DE0729F460E1AB
:10E4800083E00F94F64347C0C03AF9E0DF0729F470
:10E4900060E184E00F94F6433EC0C03A8AE0D807BA
:10E4A00029F460E185E00F94F64335C0C03AEBE013
:10E4B000DE0729F460E186E00F94F6432CC0C03BF0
:10E4C000F8E0DF0729F460E283E00F94F64323C00D
:10E4D000C03B89E0D80729F460E284E00F94F6435A
:10E4E0001AC0C03BEAE0DE0729F460E285E00F9441
:10E4F000F64311C0C038F4E0DF0729F460E483E09C
:10E500000F94F64308C0C03A84E0D80721F460E4D1
:10E5100085E00F94F6438D818F738D83F80195818B
:10E520008481892B9681911198E0892B8D83F80144
:10E53000408151816281738100E010E62AEE30E073
:10E54000CE01AFDD9C8198609C839C8190619C830F
:10E55000DF91CF911F910F910895CF92DF92EF92AB
:10E56000FF920F931F93CF93DF93EC01D901C80162
:10E57000B695A79597958795481759076A077B071A
:10E5800078F46A017B01CC0CDD1CEE1CFF1CC90178
:10E59000B801A70196010F9488642150310902C087
:10E5A00020E030E0832F8F708F832E83DF91CF9117
:10E5B0001F910F91FF90EF90DF90CF900895EF9211
:10E5C000FF920F931F93CF93DF93EC017B01009792
:10E5D00009F4B9C1803C910529F460E180E00F9411
:10E5E000F643B1C18115944029F464E080E00F94B2
:10E5F000F643A9C1C03881E0D80729F462E080E081
:10E600000F94F643A0C1C115E1E0DE0729F461E0F3
:10E6100080E00F94F64397C1C038F3E0DF0729F498
:10E6200061E081E00F94F6438EC1C03933E0D30737
:10E6300029F461E082E00F94F64385C1C11582E0C0
:10E64000D80729F462E081E00F94F6437CC1C0341E
:10E65000E2E0DE0729F462E082E00F94F64373C142
:10E66000C032F3E0DF0729F464E082E00F94F64360
:10E670006AC1C11538E0D30729F461E083E00F9443
:10E68000F64361C1C11589E0D80729F461E084E04F
:10E690000F94F64358C1C115EAE0DE0729F461E0A2
:10E6A00085E00F94F6434FC1C115FBE0DF0729F465
:10E6B00061E086E00F94F64346C1C03438E0D307EA
:10E6C00029F462E083E00F94F6433DC1C03489E051
:10E6D000D80729F462E084E00F94F64334C1C034D3
:10E6E000EAE0DE0729F462E085E00F94F6432BC1EF
:10E6F000C039F8E0DF0729F464E083E00F94F643C3
:10E7000022C1C03939E0D30729F464E084E00F94D2
:10E71000F64319C1C0398AE0D80729F464E085E0DE
:10E720000F94F64310C1C039EBE0DE0729F464E032
:10E7300086E00F94F64307C1C03CF8E0DF0729F4F8
:10E7400068E083E00F94F643FEC0C03C39E0D30795
:10E7500029F468E084E00F94F643F5C0C03C8AE0F9
:10E76000D80729F468E085E00F94F643ECC0C03A7E
:10E77000E8E0DE0769F460E183E00F94F643E0EA45
:10E78000F8E084818F7E8483F7012481225053C076
:10E79000C03AF9E0DF0729F460E184E00F94F64322
:10E7A000D2C0C03A3AE0D30729F460E185E00F9483
:10E7B000F643C9C0C03A8BE0D80729F460E186E08F
:10E7C0000F94F643C0C0C03BE8E0DE0729F460E2E6
:10E7D00083E00F94F643B7C0C03BF9E0DF0729F4AC
:10E7E00060E284E00F94F643AEC0C03B3AE0D3074A
:10E7F00029F460E285E00F94F643A5C0C03884E0B8
:10E80000D80729F460E483E00F94F6439CC0C03A33
:10E81000E4E0DE0729F460E485E00F94F64393C05A
:10E820008C818F7E8C83FB0124812250CE01C03AE3
:10E83000F8E0DF0731F480914E0684FD8CC011E1D1
:10E840008BC0803B38E0930779F0803AE9E09E077F
:10E8500031F430916E0634FD82C019E110C0803B66
:10E86000F9E09F0789F001C015E1803A3AE093078B
:10E8700031F480918E0684FD74C011E212C0803B99
:10E88000EAE09E0759F001C01DE1803A9B4049F43F
:10E890008091AE0684FD04C019E203C015E201C0F8
:10E8A0001DE2E12FE695E695E69530E2E39FF00163
:10E8B0001124FA5F177081E090E0012E02C0880FEA
:10E8C000991F0A94E2F78183223010F040E001C0E2
:10E8D00040E4DF015096A10FB11D3FB7F8942C9191
:10E8E00027702C939C91942B9C933FBF85838D81A3
:10E8F000806C8D83F70184818D7F813021F48D813F
:10E9000082608D8303C08D818D7F8D83F70185812A
:10E91000882321F08D8184608D8303C08D818B7F5E
:10E920008D83F701408151816281738100E010E69F
:10E930002AEE30E0CE0111DE8C8188608C838C81E0
:10E9400080618C8310C08C818F7E8C83F701248141
:10E950002250CE0176CF15E180EA98E080CF1DE10C
:10E960008ECF15E29ECFDF91CF911F910F91FF9037
:10E97000EF9008950F93E8ECF4E080818F7D808321
:10E9800080818F7D8083E0E8F7E302E005931092B9
:10E9900082371092833700E2069300E40693E8E79B
:10E9A000F7E300E2069300E40693ECEDF0E414864E
:10E9B0001586168617861286138610926B370F916E
:10E9C00008950F9385E080936B37E1E8F7E304E067
:10E9D0000593E9E7F7E304E005930F9108950F939A
:10E9E00083E080936B371092823710928337E0E890
:10E9F000F7E302E006930F910895E091E840F0916B
:10EA0000E940309709F0199508950F93CF93DF935C
:10EA100080916B37833019F4F0DFACDF5EC08091FA
:10EA2000673790916837C091E640D091E740C81BA6
:10EA3000D90B71F52091693730916A37820F931F96
:10EA40008093693790936A372091E2403091E34098
:10EA50008217930721F080918236882341F084E069
:10EA600080936B37E8E7F7E302E0069336C0E09166
:10EA7000EA40F091EB40309799F01995882381F0A6
:10EA80001092673710926837C091E640D091E74006
:10EA9000C034D10528F010928236C0E4D0E003C023
:10EAA00081E080938236ECE6F7E3C68BD78B8091CA
:10EAB0006737909168372091E4403091E540280F06
:10EAC000391F208F318FC80FD91FC0936737D0935C
:10EAD0006837E0E8F7E302E00693DF91CF910F910A
:10EAE0000895FC018181E82FE7708E2F90E0FC01F2
:10EAF0003197E730F105D8F48827EE52FE4F8F4F5B
:10EB00000D94C66480E190E0089580E290E008955D
:10EB100080E490E0089580E890E0089580E091E03E
:10EB2000089580E092E008958FEF93E0089588E0E3
:10EB300090E00895282F2F7030E0220F331F082E09
:10EB4000000C990B8827990F881F9927820F931F14
:10EB500002979C01220F331F220F331F220F331FF6
:10EB6000820F931F8D5F984C08950F93CF938091E0
:10EB7000CC0480FF63C081E08093CC04E8E7F7E336
:10EB800000E80693E0E8F7E300E806938093CA0400
:10EB9000E8E7F7E300E1069380916B37882329F0DB
:10EBA0008350823008F429DFE5DE80917A37909136
:10EBB0007B37089709F044C088E0E7E2F7E3ACED63
:10EBC000B0E401900D928A95E1F7E8ECF4E08081E1
:10EBD000806280838081806280830E94E563C82F89
:10EBE000811103C0EEDEC1E02CC08091DC4088239F
:10EBF0006CF41092693710926A371092673710924E
:10EC0000683782E080936B3700DF1BC08091E24061
:10EC10009091E340892B11F4E2DE13C01092693722
:10EC200010926A37109267371092683781E08093AC
:10EC30006B37E8E7F7E302E0069303C0C0E001C0EA
:10EC4000C1E08C2FCF910F9108958F929F92AF9238
:10EC5000BF92DF92EF92FF920F931F93CF93DF93B8
:10EC6000D82E68DF8C01CD2DCF70D0E0CE01880F7B
:10EC7000991FCD2D0D2C000CDD0BCC27DD0FCC1FEB
:10EC8000DD27C80FD91FCE01880F991F880F991F44
:10EC9000880F991F9C012858384C7901C90121DF40
:10ECA0004C01DD200CF07BC0FE01EE0FFF1FEE0FCC
:10ECB000FF1FEE0FFF1FE459F84C22893389D8015A
:10ECC00015968D919C911697820F931F15968D9393
:10ECD0009C93169713962D913C9114978217930746
:10ECE00009F447C0281B390B2115B4E03B0740F05D
:10ECF0002FEF33E0C901B4010F946164281B390B75
:10ED0000F801808181FF0AC0C901B4010F946164D8
:10ED100041E0892B09F040E0842F01C080E0D80158
:10ED20009C9180FB91F99C93FE01EE0FFF1FEE0F6B
:10ED3000FF1FEE0FFF1FE459F84C128A138A268733
:10ED4000378711962D913C91129715968D919C9134
:10ED50001697820F931FCC0FDD1FCC0FDD1FCC0F3A
:10ED6000DD1FC458D84C88839983F70102E00693CD
:10ED7000E4C0D8018C9181FFCDC08D7F8C93CC0FE6
:10ED8000DD1FCC0FDD1FCC0FDD1FC459D84C1A8AF4
:10ED90001B8A1E861F86F70102E00693CEC0FE0185
:10EDA000EE0FFF1FEE0FFF1FEE0FFF1FE459F84C91
:10EDB000A684B784D8018C9182FF1BC01196ED9177
:10EDC000FC91129715962D913C91169713968D9163
:10EDD0009C911497B4010F946164B0E4DB9EB00180
:10EDE00011246D5B794CAC01CF01820F931F0F94FE
:10EDF000C566F801258136812A0D3B1D25833683A2
:10EE0000838194818217930768F485839683CC0F5E
:10EE1000DD1FCC0FDD1FCC0FDD1FC459D84C8A89F4
:10EE20009B8978C0FE01EE0FFF1FEE0FFF1FEE0F54
:10EE3000FF1FE459F84C42895389A416B50609F01E
:10EE400069C02817390709F465C0AC01421B530B90
:10EE50009A01211554E0350748F02FEF33E0C9013E
:10EE6000B4010F946164281B390B06C0C901B401B9
:10EE70000F946164281B390BFE01EE0FFF1FEE0F8C
:10EE8000FF1FEE0FFF1FE459F84C16861786281552
:10EE9000390500F5D8018C9184608C93B0E4DB9E39
:10EEA000C00111248D5B994CFE01EE0FFF1FEE0F88
:10EEB000FF1FEE0FFF1FE458F84C80839183CC0FA7
:10EEC000DD1FCC0FDD1FCC0FDD1FC459D84C8A8A43
:10EED0009B8A1CC0F8014181528185819681840FF3
:10EEE000951FFE01EE0FFF1FEE0FFF1FEE0FFF1F1E
:10EEF000E458F84C80839183CC0FDD1FCC0FDD1FCD
:10EF0000CC0FDD1FC459D84C2A8B3B8BF70102E094
:10EF1000069313C0D8018C9180FF0FC08E7F8C9315
:10EF20001796ED91FC911897309739F015966D91E1
:10EF30007C9116974D2D80E01995DF91CF911F910F
:10EF40000F91FF90EF90DF90BF90AF909F908F90C8
:10EF50000895CF93CFB7F894E1ECF4E080818E7FF1
:10EF600080831092C00410820F9445441092AC37F5
:10EF7000CFBFCF9108959FB7F89481E08093AC37CD
:10EF8000EAECF4E080E4808380E28083E1ECF4E06A
:10EF9000808181608083A9ECB4E08C9182608C9345
:10EFA000E8ECF4E08081806480838C9181608C93B4
:10EFB0008081806880839FBF0895CF93DF93C0E6F0
:10EFC000D0E0188280E30F940D44E0ECF4E08081FF
:10EFD0008064808381E08883CFB7F894ECE6F7E320
:10EFE0001586158A158E15A215A615AAE3E0F7E376
:10EFF00080818E7F8083ECE0F7E380818E7F808349
:10F00000E5E1F7E380818E7F8083EEE1F7E38081A5
:10F010008E7F80836AE170E082E00F9421628F3FEF
:10F0200019F08093FA0403C08FE18093FA046BE136
:10F0300070E082E00F9421628F3F19F08093FB040F
:10F0400003C08FE18093FB04E0ECF4E080818260F8
:10F05000808380818068808380818061808388E76D
:10F0600097E3868397838081806280838FEF80938C
:10F07000C504E8ECF4E08081816080831092AC37B5
:10F080007ADFCFBFDF91CF9108958093C3040895B5
:10F090008091C3040895ECEDF0E480879187628746
:10F0A00073870895282F2F7030E0220F331F082E0A
:10F0B000000C990B8827990F881F9927820F931F9F
:10F0C000FC01EE0FFF1FEE0FFF1FEE0FFF1FE459B5
:10F0D000F84C2585207C09F069C06370613011F01F
:10F0E00018F404C060EC03C060E801C060E440387C
:10F0F0005105E9F050F440325105A9F04034510572
:10F10000A1F040315105D9F40CC0411522E052075D
:10F1100091F04F3F23E0520781F04115514079F4BF
:10F1200008C021E00DC022E00BC023E009C024E0AC
:10F1300007C025E005C026E003C027E001C020E0AD
:10F14000FC01EE0FFF1FEE0FFF1FEE0FFF1FE45934
:10F15000F84C158636E03487262B2587FC01EE0F08
:10F16000FF1FEE0FFF1FEE0FFF1FE459F84C258520
:10F17000207C203C69F4FC01EE0FFF1FEE0FFF1F07
:10F18000EE0FFF1FE459F84C25852770273081F0DA
:10F19000880F991F880F991F880F991FFC01E45948
:10F1A000F84C85858062858781E0089580E0089528
:10F1B00081E00895E82FEF70F0E0EE0FFF1F082EBA
:10F1C000000C990B8827990F881F9927E80FF91FC2
:10F1D000EE0FFF1FEE0FFF1FEE0FFF1FE459F84C5D
:10F1E000858582FB882780F90895282F2F7030E0CD
:10F1F000A901440F551F282F082E000C330B22277E
:10F20000330F221F3327240F351FF901EE0FFF1F85
:10F21000EE0FFF1FEE0FFF1FE459F84C958592FF8C
:10F2200017C0220F331F220F331F220F331FF90184
:10F23000E459F84C95859B7F95877CDCFC018081A7
:10F2400080FF06C08E7F80830780F085E02D1995B2
:10F2500081E008958F929F92AF92BF92CF92DF92FA
:10F26000EF92FF920F931F93CF93DF93982E862EEA
:10F270006A0179015FDC5C01292DC92DCF70D0E0D6
:10F28000CE01880F991FC92D092C000CDD0BCC274E
:10F29000DD0FCC1FDD27C80FD91FFE01EE0FFF1FAA
:10F2A000EE0FFF1FEE0FFF1FE459F84C8585807CA1
:10F2B00009F47EC0FE01EE0FFF1FEE0FFF1FEE0FE1
:10F2C000FF1FE459F84C8585807C803C61F0FE018D
:10F2D000EE0FFF1FEE0FFF1FEE0FFF1FE459F84C5C
:10F2E000858582FD67C08FB7F894F501908190FF06
:10F2F00003C08FBF80E05FC0F50190819160908373
:10F300008FBFC182D282E382F48215821682078384
:10F310001087811006C091E0E114F10419F090E02B
:10F3200001C091E0F501808190FB81F98B7F8083A2
:10F3300022235CF4CC0FDD1FCC0FDD1FCC0FDD1FB3
:10F34000C459D84C1A8A1B8A2FC0FE01EE0FFF1F2A
:10F35000EE0FFF1FEE0FFF1FE459F84C8585807CF0
:10F36000803CB1F4CE01880F991F880F991F880F38
:10F37000991F8858984CB5DBBC01C7010F94616494
:10F38000892B31F0F50180818E7F808380E013C06E
:10F39000CC0FDD1FCC0FDD1FCC0FDD1FC459D84CA7
:10F3A0001E861F861A8A1B8A892D4FDC81E003C0C6
:10F3B00080E001C080E0DF91CF911F910F91FF901D
:10F3C000EF90DF90CF90BF90AF909F908F90089577
:10F3D000FF920F931F93CF93DF93182FC82FCF70F7
:10F3E000D0E0CE01880F991FC12F012E000CDD0B3C
:10F3F000CC27DD0FCC1FDD27C80FD91F812F9ADB4B
:10F40000DC01FE01EE0FFF1FEE0FFF1FEE0FFF1FCF
:10F41000E858F84C02E005938C9180FF22C08E7F63
:10F420008C931796ED91FC9118973097D1F011239A
:10F430005CF4CC0FDD1FCC0FDD1FCC0FDD1FC459DA
:10F44000D84C6A897B890AC0CC0FDD1FCC0FDD1F29
:10F45000CC0FDD1FC459D84C6E857F85412F81E0CC
:10F460001995DF91CF911F910F91FF900895CF9340
:10F47000C82FAEDFEC2FEF70F0E0EE0FFF1F8C2FE8
:10F48000CC0F990B8827990F881F9927E80FF91F30
:10F49000EE0FFF1FEE0FFF1FEE0FFF1FE459F84C9A
:10F4A0001586CF9108950F93E82FEF70F0E0EE0FDF
:10F4B000FF1F282F082E000C330B2227330F221F8B
:10F4C0003327E20FF31FEE0FFF1FEE0FFF1FEE0FAC
:10F4D000FF1FDF01A459B84C1D969C911D979460A5
:10F4E0001D969C93E858F84C01E0069371DF81E08B
:10F4F0000F9108950F931F93CF93DF938B01C82F24
:10F50000CF70D0E0CC0FDD1F282F082E000C330B5E
:10F510002227330F221F3327C20FD31F0BDBCC0F41
:10F52000DD1FCC0FDD1FCC0FDD1FC459D84C2D853E
:10F5300022FF0AC0FC01208120FD0AC02160208337
:10F540000783108781E005C0F801199581E001C0AB
:10F5500080E0DF91CF911F910F9108951F920F923C
:10F560000FB60F9211240BB60F920F932F933F9368
:10F570004F935F936F937F938F939F93AF93BF93BB
:10F58000EF93FF938091CB04882344F480E8809329
:10F59000CA040E94B5630E94EB5A87C08091CB04D5
:10F5A00082FF20C084E08093CA048091803786FF68
:10F5B0007CC08091CC0481FD78C0D7DA811175C000
:10F5C00080916B37813011F40ADA6FC0843009F012
:10F5D0006CC0E1E8F7E304E00593E9E7F7E304E052
:10F5E000059363C08091CB0481FF5AC082E0809371
:10F5F000CA048091783786FF58C08091CC0481FD81
:10F6000054C0B3DA811151C080916B37823041F41C
:10F6100084E080936B37E8E7F7E302E0069345C0A8
:10F62000833009F042C0E1E8F7E304E00593E9E73D
:10F63000F7E304E0059339C080E18093CA0481E0D8
:10F64000C7DE81E8C5DE0E948A631092C304ECE63F
:10F65000F7E3158696E0948783E48587158A948B73
:10F66000858B87E297E3808B918B84D91EC0809134
:10F67000CB0486FF08C080E48093CA041092AC37A4
:10F680000E94EE5A12C08091CB0485FF0EC080E22A
:10F690008093CA0481E08093AC370E94EF5A05C082
:10F6A0008091CB0484FFE3CFC7CFFF91EF91BF914F
:10F6B000AF919F918F917F916F915F914F913F910A
:10F6C0002F910F910F900BBE0F900FBE0F901F90B8
:10F6D00018951F920F920FB60F9211240BB60F922E
:10F6E0000F931F932F933F934F935F936F937F934A
:10F6F0008F939F93AF93BF93CF93DF93EF93FF933A
:10F700008091CC0481FD03C030DA8111C2C082E057
:10F710008093CC048091C5048195880FE8E7F7E3D6
:10F72000E81BF10920813181285737433695279509
:10F730003695279536952795822F869520FD02C010
:10F7400090E001C090E8890FE82FEF70F0E0EE0F35
:10F75000FF1F282F082E000C330B2227330F221FE8
:10F760003327E20FF31FDF01AA0FBB1FAA0FBB1F36
:10F77000AA0FBB1FA459B84C1C969C9195FF89C039
:10F78000EE0FFF1FEE0FFF1FEE0FFF1FE858F84CA4
:10F7900000E20693811178C080916B37843019F4B0
:10F7A0002CD9E8D876C000917A3710917B378091B8
:10F7B000E6409091E740C0916737D0916837980153
:10F7C0002C0F3D1F8217930718F48C010C1B1D0B87
:10F7D0008091E4409091E540A80167E277E38C0FC7
:10F7E0009D1F0F94C566C00FD11FC0936737D0937C
:10F7F00068370034110569F48091693790916A3750
:10F800008C0F9D1F2091E2403091E34082179307B7
:10F8100080F0ECEDF0E4C287D3870684F785E02D15
:10F82000309729F01995811102C0CBD832C0D7D8B2
:10F8300030C08091E6409091E740C817D907F9F4AD
:10F84000E091EA40F091EB40309711F4BAD821C032
:10F850001995811102C0B5D81CC02091693730912B
:10F860006A378091673790916837820F931F809332
:10F87000693790936A371092673710926837E8E7D4
:10F88000F7E302E0069305C0803811F4BED801C04A
:10F89000DCD9FF91EF91DF91CF91BF91AF919F9113
:10F8A0008F917F916F915F914F913F912F911F9118
:10F8B0000F910F900BBE0F900FBE0F901F901895D9
:10F8C0009091800024E0829FB00111246C739270AB
:10F8D0009160692B80E890E00F94C261E0E8F0E06D
:10F8E000828180FDFDCF0895609180006C7363601C
:10F8F00080E890E00F94C261E0E8F0E0828180FD52
:10F90000FDCF0895CF92DF92EF92FF92CF93DF93D6
:10F91000EC016B01E12CF12C60E070E68AEE90E0E6
:10F92000A70196010F948864CA01B9012FEF3FEF38
:10F9300040E050E00F9488642115310529F481E0FE
:10F940008C8321E030E02DC02230310528F482E0A4
:10F950008C8322E030E025C02430310528F483E098
:10F960008C8324E030E01DC02830310528F484E089
:10F970008C8328E030E015C02034310528F485E080
:10F980008C8320E430E00DC02F3F310509F028F4CE
:10F9900086E08C8320E031E004C087E08C8320E0A7
:10F9A00034E040E050E060E070E68AEE90E00F94D2
:10F9B0008864CA01B901A70196010F9488642D8358
:10F9C0003E832436310518F41C821D821E82DF918D
:10F9D000CF91FF90EF90DF90CF9008950F931F93FA
:10F9E000CF93DF93EC018901862F90E0873091055A
:10F9F00008F08BC0FC018827E752FE4F8F4F0D9413
:10FA0000C66480E098E088839983E0E4F6E0308182
:10FA100081E090E02FEF240F02C0880F991F2A95F4
:10FA2000E2F7832B808371C080E498E08883998318
:10FA3000E0E4F6E0308181E090E023E0240F02C0B2
:10FA4000880F991F2A95E2F7832B80835EC080E0A0
:10FA500099E088839983E0E6F6E0308181E090E0E8
:10FA60002FEF240F02C0880F991F2A95E2F7832BEE
:10FA700080834BC080E499E088839983E0E6F6E0D8
:10FA8000308181E090E023E0240F02C0880F991FAD
:10FA90002A95E2F7832B808338C080E09AE0888340
:10FAA0009983E0E8F6E0308181E090E02FEF240FC9
:10FAB00002C0880F991F2A95E2F7832B808325C007
:10FAC00080E49AE088839983E0E8F6E0308181E081
:10FAD00090E023E0240F02C0880F991F2A95E2F7D7
:10FAE000832B808312C080E09BE088839983E0EAC7
:10FAF000F6E0308181E090E02FEF240F02C0880F04
:10FB0000991F2A95E2F7832B80834A83423061F064
:10FB100018F4413031F010C0433049F0443051F016
:10FB20000BC080E18B8308C080E28B8305C080E43A
:10FB30008B8302C080E88B83888199810E94436F08
:10FB4000E881F9818181887F836081831D821E82A3
:10FB50001C82E881F9818081807F8083B801CE0199
:10FB6000D1DEDF91CF911F910F910895CF93DF9355
:10FB7000EC012D813E81A62FB0E00F94CE6424E6E7
:10FB800030E040E050E00F9488648A81E881F98198
:10FB9000E6FD17C0823061F018F4813031F01BC0EF
:10FBA000833049F0843051F016C020AF31AF13C01C
:10FBB00022AF33AF10C024AF35AF0DC026AF37AF83
:10FBC0000AC0813019F0823021F005C020AF31AF7A
:10FBD00002C022AF33AF8D819E81E881F98186A377
:10FBE00097A38B81E881F981E6FD04C09181892B7F
:10FBF000818304C091818073892B8183E881F9819D
:10FC00008081807F9C81892B8083DF91CF910895B3
:10FC1000CF93DF93EC014115510509F443C0A9E4EA
:10FC2000B3E420E030E0922FF901E45FFA4EE49172
:10FC3000ED932F5F3F4F27303105A9F7FA01DE0121
:10FC4000C9E4D3E480818B8381818C83F901E75BF4
:10FC5000FC4B8CE28083E2E0E90FF0E0E75BFC4BD9
:10FC60006083C4E0C90F9D5FE92FF0E0E75BFC4BC8
:10FC70008DE78083D0E0FE01E75BFC4B108221E042
:10FC8000AE0169E473E4CD010F948B310E944E2ADA
:10FC9000811108C021E0AE0169E473E48AEA99E3C6
:10FCA0000F948B31DF91CF9108954F925F926F92B5
:10FCB0007F928F929F92AF92BF92DF92EF92FF92CC
:10FCC0000F931F93CF93DF931F92CDB7DEB77C01C5
:10FCD0004115510509F466C188E08983A9E4B3E4BC
:10FCE00020E030E0922FF901E45FFA4EE491ED93C9
:10FCF0002F5F3F4F27303105A9F7FA01162FA9E4EE
:10FD0000B3E4808113968C931397818114968C931E
:10FD100002E0090FF901E75BFC4B8CE28083623063
:10FD200088F5862F0F9412188823B1F0812F0F9435
:10FD3000D7179F938F931F921F938BE599E29F9301
:10FD40008F93E02FF0E0E75BFC4BFF93EF930F9472
:10FD5000F366CDBFDEBF08C1812F0E94CAD09F933A
:10FD60008F931F921F938BE599E29F938F93E02FC0
:10FD7000F0E0E75BFC4BFF93EF930F94F366CDBF8E
:10FD8000DEBFF2C0663109F078C086E10F941B1720
:10FD90002B013C010F94A50E4B015C01672B682BD6
:10FDA000692BF1F4C301B20120E13EE040E050E0F4
:10FDB0000F94AA645F934F933F932F931F9286E112
:10FDC0008F9382E699E29F938F93E02FF0E0E75BB9
:10FDD000FC4BFF93EF930F94F366CDBFDEBFC4C01F
:10FDE000802F0E9465D0992334F5C301B20120E130
:10FDF0003EE040E050E00F94AA64CA01B9010F94BC
:10FE00000837BF92AF929F928F929F938F937F9369
:10FE10006F931F9286E18F938AE699E29F938F9367
:10FE2000E02FF0E0E75BFC4BFF93EF930F94F3665A
:10FE3000CDBFDEBF99C0BF92AF929F928F92C30198
:10FE4000B20120E13EE040E050E00F94AA645F93ED
:10FE50004F933F932F931F9286E18F9387E799E209
:10FE60009F938F93E02FF0E0E75BFC4BFF93EF93C2
:10FE70000F94F366CDBFDEBF77C0663071F5E02F1B
:10FE8000F0E0E75BFC4B86E380836894DD24D2F8E6
:10FE9000D90E9D5FE92FF0E0E75BFC4B8CE280839D
:10FEA00086E00F941B178B019C018D2D90E04BE099
:10FEB000BE016F5F7F4F875B9C4B0F946137E98179
:10FEC000ED0DAE2FB0E0A75BBC4B8DE78C93EF5FE1
:10FED000F0E0E75BFC4B108247C0653071F5E02F26
:10FEE000F0E0E75BFC4B85E380836894DD24D2F887
:10FEF000D90E9D5FE92FF0E0E75BFC4B8CE280833D
:10FF000085E00F941B178B019C018D2D90E04BE039
:10FF1000BE016F5F7F4F875B9C4B0F94AD38E981CB
:10FF2000ED0DAE2FB0E0A75BBC4B8DE78C93EF5F80
:10FF3000F0E0E75BFC4B108217C0862F0F941B1775
:10FF40009F938F937F936F931F921F9382E699E203
:10FF50009F938F93802F90E0875B9C4B9F938F9311
:10FF60000F94F366CDBFDEBFE9E4F3E40190002017
:10FF7000E9F73197E954F344E983AF01552721E0CC
:10FF800069E473E4C7010F948B310E944E2A8111FA
:10FF900009C0498150E021E069E473E48AEA99E309
:10FFA0000F948B310F90DF91CF911F910F91FF90A4
:10FFB000EF90DF90BF90AF909F908F907F906F9069
:10FFC0005F904F900895AC016115710571F1E5E105
:10FFD000F5E1A9E4B3E421E533E494919D933196EE
:10FFE000A217B307D1F7FB01CA01A9E4B3E420814A
:10FFF00013962C931397218114962C93149718968B
:020000021000EC
:100000001C92189721E048E050E0BD010F948B311D
:100010000E944E2A811109C021E048E050E069E4C5
:1000200073E48AEA99E30D948B310895EF92FF927D
:100030000F931F93CF93DF938C016115710509F422
:100040007FC04115510509F47BC0E3E0F5E1A9E467
:10005000B3E4C1E5D3E494919D933196AC17BD0709
:10006000D1F7FA017B01C9E4D3E480818B838181DC
:100070008C831F922F9383E899E29F938F9381E55E
:1000800093E49F938F930F94F36609900020E9F710
:100090002197C954D344F70181810F900F900F909D
:1000A0000F900F900F90811115C080811F928F9338
:1000B00080E791E29F938F93DD27C75BDC4BDF9353
:1000C000CF930F94F3660F900F900F900F900F90B7
:1000D0000F9016C01F928F93F70180811F928F930C
:1000E0008DE691E29F938F93DD27C75BDC4BDF9317
:1000F000CF930F94F366EDB7FEB73896EDBFFEBF12
:10010000E9E4F3E401900020E9F73197E954F3447E
:10011000EF01DD2721E0AE0169E473E4C8010F942B
:100120008B310E944E2A81110BC00A5A194341F0AB
:1001300021E0AE0169E473E48AEA99E30F948B311C
:10014000DF91CF911F910F91FF90EF900895CF9382
:10015000DF93EC014115510509F43FC0662361F0BE
:10016000E5E1F5E1A9E4B3E490E024912D939F5FEC
:1001700031969730D1F70BC0ECE0F5E1A9E4B3E498
:1001800090E024912D939F5F31969730D1F7DA015B
:10019000CE01E9E4F3E42C91238311962C9124837E
:1001A0002CE227833CE43087218720E322872DE758
:1001B0002387148621E04CE050E0BF010F948B317F
:1001C0000E944E2A811109C021E04CE050E069E410
:1001D00073E48AEA99E30F948B31DF91CF9108950C
:1001E000EF92FF920F931F93CF93DF9300D01F9254
:1001F000CDB7DEB70097C9F166307105C0F1FC01DB
:1002000020812035B1F521812C32A9F524812C32B1
:10021000A1F57A018C010B5F1F4FAB0145505109CD
:100220009E012F5F3F4FB8018CE20F94383788232F
:1002300049F149815A814B5F5F4F49835A83463068
:100240005105E8F045509E012D5F3F4F60E0C80129
:100250000F94C0358823B1F08B819C818C3191053E
:1002600080F4F701808381E00DC080E00BC080E066
:1002700009C080E007C080E005C080E003C080E0E6
:1002800001C080E02496CDBFDEBFDF91CF911F91EA
:100290000F91FF90EF900895CF92DF92EF92FF922F
:1002A0000F931F93CF93DF93CDB7DEB72C97CDBFBE
:1002B000DEBF009709F431C16630710508F42FC123
:1002C000FC012081203509F02CC121812C3209F05C
:1002D0002AC124812C3209F028C17B018C016C01D8
:1002E000F5E0CF0ED11CAB01455051099E012F5FA7
:1002F0003F4FB6018CE20F943837982F882309F4CA
:1003000023C149815A814B5F5F4F49835A834630ED
:10031000510508F40CC145509E012D5F3F4F60E030
:10032000C6010F94C035982F882309F40DC12B8185
:100330003C812C31310508F0FCC049815A81DA0139
:100340001196AE15BF0508F0F6C02C31310508F046
:10035000F4C0F9018827E052FE4F8F4F0D94C66418
:10036000C8018A0F9B1FFC0160816D3241F4FA01C4
:100370003296EE15FF0508F0E2C040E002C0FD0134
:1003800041E02631310559F46E2D6E1B9E01275F29
:100390003F4FC8018E0F9F1F0F94110512C02630CA
:1003A000310541F46E2D6A1BAE01475F5F4F0F941C
:1003B000DE0707C06E2D6A1BAE01475F5F4F0F94CB
:1003C000FA08882309F4BDC049855A856B857C8568
:1003D0008B810E94B9D5982F882309F4B5C049852F
:1003E0005A856B857C858B810F942E1791E0ACC06C
:1003F0004E2D4A1B9E012B5F3F4F60E0C8018A0FC4
:100400009B1F0F944B36982F882309F49DC04D8174
:100410005E816F81788549875A876B877C878B815E
:100420000E94B9D5982F882309F48EC089859A85B2
:10043000AB85BC858B309105A105B10549F487EFEB
:100440009CE30E94DF2E982F882309F47DC00CC006
:100450000C97A105B10544F087EF9CE30E94DF2EC5
:10046000982F882309F470C049855A856B857C854F
:100470008B810F942E1791E067C04E2D4A1B9E0171
:100480002B5F3F4F60E0C8018A0F9B1F0F944B36D4
:10049000982F882309F458C04D815E816F8178853B
:1004A00049875A876B877C878B810E94B9D5982FA3
:1004B000882349F049855A856B857C858B810F940B
:1004C0002E1791E041C02B813C81A9014C5051096C
:1004D00046305105C8F549855A856B857C85452B85
:1004E000462B472B89F540E050E0BA01822F0F944C
:1004F0002E1791E029C0C7018A1B9B0B899718F51D
:100500006E2D6A1B422FC8018A0F9B1F0F949917EB
:1005100091E0811119C090E017C090E015C090E003
:1005200013C090E011C090E00FC090E00DC090E0CB
:100530000BC090E009C090E007C090E005C090E0DB
:1005400003C090E001C090E0892F2C96CDBFDEBFA4
:10055000DF91CF911F910F91FF90EF90DF90CF909F
:1005600008950F931F93CF93DF931F921F92CDB7E0
:10057000DEB7009741F16630710538F1FC0120814A
:10058000203529F521812C3221F524812C3219F5D1
:100590008C01AB0145505109BC016B5F7F4F9E013F
:1005A0002F5F3F4F8CE20F9438378823B9F0898151
:1005B0009A810596069788F081E0F8019581963436
:1005C00069F080E00BC080E009C080E007C080E0F7
:1005D00005C080E003C080E001C080E00F900F9074
:1005E000DF91CF911F910F910895EF92FF920F939A
:1005F0001F93CF93DF9300D000D0CDB7DEB7009725
:1006000009F453C06630710508F451C0FC01208123
:10061000203509F04EC021812C3209F04CC02481D4
:100620002C3209F04AC07B018C01AB0145505109C5
:10063000BC016B5F7F4F9E012F5F3F4F8CE20F9499
:100640003837882309F442C089819A819C012B5F45
:100650003F4F29833A832630310588F1F8012581FF
:10066000263479F506968E159F0568F54E2D481BA4
:100670009E012D5F3F4F60E0800F911F0F944B361E
:10068000882321F16B817C818D819E818B019C016E
:100690000150110921093109073E13402105310597
:1006A000A0F40E944ED181E011C080E00FC080E034
:1006B0000DC080E00BC080E009C080E007C080E092
:1006C00005C080E003C080E001C080E02696CDBF79
:1006D000DEBFDF91CF911F910F91FF90EF900895B2
:1006E0000F931F93CF93DF93EC016115710509F40C
:1006F00044C0A9E4B3E420E030E0922FF901E45FC4
:10070000FA4EE491ED932F5F3F4F27303105A9F763
:10071000FB01A9E4B3E4808113968C931397818144
:1007200014968C931497F901E75BFC4B8CE2808361
:100730009E5FE92FF0E0E75BFC4B86E49DE780835A
:1007400091831282FD0101900020E9F73197E9546D
:10075000F3448F01112721E0A801BD01CE010F94C0
:100760008B310E944E2A811108C021E0A80169E462
:1007700073E48AEA99E30F948B31DF91CF911F9153
:100780000F910895FC01892B61F06530710558F0D7
:100790008081803551F481E091819C3239F080E094
:1007A000089580E0089580E0089580E0089500971E
:1007B00099F06330710590F0FC012081203581F4BF
:1007C00021812C3279F424812C3271F48581835477
:1007D000823060F080E0089580E0089580E0089520
:1007E00080E0089580E0089580E0089581E0089514
:1007F000009791F06330710588F0FC01208120356D
:1008000079F421812C3271F424812C3269F48581B0
:100810008F3461F080E0089580E0089580E00895CD
:1008200080E0089580E0089580E0089581E00895D3
:10083000009791F06330710588F0FC01208120352C
:1008400079F421812C3271F424812C3269F4858170
:10085000873561F080E0089580E0089580E0089594
:1008600080E0089580E0089580E0089581E0089593
:10087000CF92DF92EF92FF920F931F93CF93DF936C
:100880004115510509F4AFC0009709F4AEC06630B8
:10089000710508F4ACC0FC012081203509F0A9C025
:1008A00021812C3209F0A7C024812C3209F0A5C087
:1008B0008581873509F0A3C0EA0187EF9CE30E9498
:1008C000BF14883009F49DC087EF9CE30E94BF14D9
:1008D000863009F498C00F942C290E94C05561E01D
:1008E0008DEF9CE30E9434580F9456180E94D11C3F
:1008F000813079F582E00E9473D06B017C01DD24A8
:10090000EE24FF24B701A60182E00F942E17B70151
:10091000A60182E00E945BD00E944E2A811119C07C
:1009200084E1E7E8F9E2A0EDB4E401900D928A9544
:10093000E1F7E0EDF4E401900020E9F73197AF0131
:10094000405D544420E060ED74E48AEA99E30F943A
:100950008B31CE010E94201C80E00E9441D09B017F
:10096000AC016894EE24E2F801ED12E2BE01685E8B
:100970007F4FCE0106960E948E598D8340E050E055
:10098000BA01CE010E948F2E8D81882351F182E021
:100990000E9465D0062F8BE00E9465D021E0611196
:1009A00020E043EB50E4BE016C5C7F4FCE01C69665
:1009B0000E949152CE010E94F61B9E01265A3D4F85
:1009C000AE01475A5D4FBE016C5A7D4FCE018D5A24
:1009D0009D4F0E94162D0E94B03368E0CE010E9408
:1009E000AC148D8111C080E00FC080E00DC080E0AC
:1009F0000BC080E009C080E007C080E005C080E057
:100A000003C080E001C080E0DF91CF911F910F9182
:100A1000FF90EF90DF90CF900895CF92DF92EF920A
:100A2000FF920F93CF93DF934115510509F4B0C0A6
:100A3000009709F4AFC06630710508F4ADC0FC0141
:100A40002081203509F0AAC021812C3209F0A8C0EC
:100A500024812C3209F0A6C0EA018581833409F48F
:100A600093C0843409F0A0C00E9403D10F94F417FE
:100A700087EF9CE30E94BF14883009F497C087EF8A
:100A80009CE30E94BF14863009F492C00F942C2975
:100A90000E94C05561E08DEF9CE30E9434580F9492
:100AA00056180E94D11C813079F582E00E9473D0E3
:100AB0006B017C01DD24EE24FF24B701A60182E056
:100AC0000F942E17B701A60182E00E945BD00E940E
:100AD0004E2A811119C084E1E7E8F9E2A0EDB4E4FF
:100AE00001900D928A95E1F7E0EDF4E40190002089
:100AF000E9F73197AF01405D544420E060ED74E4C4
:100B00008AEA99E30F948B3180E00E9441D09B01E7
:100B1000AC01BE01685E7F4FCE0106960E94C855AB
:100B20008D8340E050E0BA01CE010E948F2E8D816E
:100B3000882341F182E00E9465D0062F8BE00E945D
:100B400065D021E0611120E043EB50E4BE016C5C14
:100B50007F4FCE01C6960E949152CE010E94F61B95
:100B60009E01265A3D4FAE01475A5D4FBE016C5A59
:100B70007D4FCE018D5A9D4F0E94162D68E0CE010B
:100B80000E94AC148D8115C00F94F41781E011C040
:100B900080E00FC080E00DC080E00BC080E009C0A5
:100BA00080E007C080E005C080E003C080E001C0B5
:100BB00080E0DF91CF910F91FF90EF90DF90CF9089
:100BC0000895BF92CF92DF92EF92FF920F931F93FF
:100BD000CF93DF931F92CDB7DEB76115710509F48E
:100BE00064C0DB017C01E9E4F3E48BE7808380E708
:100BF00081838CE282839C91938311969C91948350
:100C000085839FE49683878380E00E94C0D78B0111
:100C10009C0148E0BE016F5F7F4F81E593E40F9434
:100C20000F39E981E85FD12C0F2EFCE2BF2EF02DA9
:100C3000CC24C394CE0EF0E0E75BFC4BB082D3949F
:100C40008D2D0E94C0D78B019C018C2D90E048E037
:100C5000BE016F5F7F4F875B9C4B0F940F39E9811B
:100C6000EC0D83E0D812E4CF81E08E0FF0E0E75B7B
:100C7000FC4B9DE79083482F50E0FA01E75BFC4B6B
:100C80001082898321E069E473E4C7010F948B31FA
:100C90000E944E2A811109C0498150E021E069E497
:100CA00073E48AEA99E30F948B310F90DF91CF912F
:100CB0001F910F91FF90EF90DF90CF90BF9008951C
:100CC000CF93DF9341155105A9F10097A9F1653044
:100CD0007105A0F1FC012081203591F521812C3294
:100CE00089F52281263481F5EA0184818235E9F093
:100CF000833531F0843451F50E942DD181E027C035
:100D00000F942C29BE016C5C7F4FCE01C6960E94C9
:100D1000965087EF9CE30E94992281110F944E29EF
:100D2000CE010E94E6298D8112C0CA01C6960F9499
:100D3000FF0D0DC080E00BC080E009C080E007C05F
:100D400080E005C080E003C080E001C080E0DF916A
:100D5000CF910895FC01892B79F06630710570F010
:100D60008081833569F481818C3261F481E09481E2
:100D70009C3249F080E0089580E0089580E0089575
:100D800080E0089580E008950F93CF93DF9300975C
:100D900009F476C06630710508F474C0FC01608106
:100DA000633509F071C061816C3209F06FC06481F4
:100DB0006C3209F06DC04115510509F46BC0211565
:100DC000310509F469C08581813309F067C0B90133
:100DD000EA01F9011082CA010E948020882309F4E7
:100DE0005FC0CE010E94612081112BC0CE010E9404
:100DF000E62961E0CE010E94112764E0CE010E9445
:100E0000AC1461E0CE010E94462019820E9496A88F
:100E1000E5E8F3E4808190E0DC01AB57BC4B25852D
:100E20003685880F991FFC01EB57FC4B418152819D
:100E30001F960C9161E087EF9CE30E94002581E002
:100E400032C00E944E2A81112DC084E1EBE9F9E203
:100E5000A9E4B3E401900D928A95E1F7E9E4F3E4A3
:100E600001900020E9F73197AF014954534421E044
:100E700069E473E48AEA99E30F948B3181E013C04B
:100E800080E011C080E00FC080E00DC080E00BC0AA
:100E900080E009C080E007C080E005C080E003C0BA
:100EA00081E001C081E0DF91CF910F9108950F9310
:100EB0001F93CF93009709F4C5C16630710508F4FC
:100EC000C3C1DC012C91233509F0C0C111962C91CE
:100ED00011972C3209F0BCC114962C9114972C3226
:100EE00009F0B8C14115510509F4B6C11596EC9148
:100EF0008E2F90E0FC01F097E734F10508F0AEC1C9
:100F00008A018827E450FE4F8F4F0D94C664CA01B2
:100F10000E94BF14843031F0C8010E94BF14893090
:100F200009F09EC1C8010E94D21FC8010F940D1B79
:100F3000C8010E94E6290F942C2960E087EF9CE30A
:100F40000E94112763E0C8010E94AC14F8011182CD
:100F50000E9483A8E5E8F3E4808190E0DC01AB57D0
:100F6000BC4B25853685880F991FFC01EB57FC4B40
:100F7000418152811F960C9161E087EF9CE30E94B2
:100F80000025C1E07CC1CA010E946120882309F4C8
:100F900069C181E0D80111968C9360E0C8010E947C
:100FA000D81460E0C8010E94C6140E944E2A811124
:100FB0005BC180E1EFEAF9E2A9E4B3E401900D92AC
:100FC0008A95E1F7E9E4F3E401900020E9F731972D
:100FD000AF014954534421E069E473E48AEA99E398
:100FE0000F948B31C1E04BC1CA010E94612088235C
:100FF00009F43CC160E0C8010E94D81460E0C80157
:101000000E94C614F801ED5AFD4FD801A75ABD4FF2
:101010008C918083319611968C918083F801118296
:101020000E944E2A811124C180E1EFEBF9E2A9E48C
:10103000B3E401900D928A95E1F7E9E4F3E40190BD
:101040000020E9F73197AF014954534421E069E4A6
:1010500073E48AEA99E30F948B31C1E010C1CA01AD
:101060000E946120C82F882309F409C1C8010E9489
:10107000AE27C1E0811103C1C0E001C1CA010E94D5
:101080006120882329F0C8010E943827C82FF7C0A3
:101090000E9412D8C1E0F3C0CA010E946120C82F8B
:1010A000882309F4ECC00F942C2960E087EF9CE3BF
:1010B0000E94112769E0C8010E94AC14D801119662
:1010C0001C92C8010F941D1BC8010E948A1CC801F4
:1010D0000F94B71F0F94302C61E0C8010E94462086
:1010E000C1E0CDC0CA010E946120C82F811106C095
:1010F000C8010E94BF148A3009F0C1C00F942C2986
:101100000F94632760E0C8010E9411276AE0C801BC
:101110000E94AC1481E0F8018183C8010E9410B3E1
:10112000C8010E945735C8010E94A4B20F94F52D42
:101130000E94E6B261E0C8010E944620C1E09FC063
:10114000CA010E946120882309F494C00F942C29BD
:1011500060E0C8010E94D81460E0C8010E94C61473
:10116000F801E45AFD4F1082C8010E94E4B36AE01E
:10117000C8010E94AC1481E0D80111968C93C1E0A3
:101180007EC0CA010E94BF148930A9F463EB70E4E9
:10119000C8010F94541FC8010F94141B843109F027
:1011A0006BC0C8010F941D1BC8010F94B71F0F948B
:1011B000302CC1E064C0C8010E94BF148A3009F01D
:1011C0005DC0E3EBF0E462817381808191810F94D3
:1011D000145863EB70E4C8010E9441B2C1E04FC0F3
:1011E000CA010F940D1BC8010E948BADC8010E945B
:1011F000E62961E0C8010E94112764E0C8010E944D
:10120000AC1461E0C8010E944620F80111820E94DE
:1012100096A8E5E8F3E4808190E0DC01AB57BC4B95
:1012200025853685880F991FFC01EB57FC4B4181C2
:1012300052811F960C9161E087EF9CE30E9400258C
:10124000C1E01DC0C0E01BC0C0E019C0C0E017C0B5
:10125000C0E015C0C0E013C0C0E011C0C0E00FC0C6
:10126000C1E00DC0C1E00BC0C1E009C0C1E007C0D2
:10127000C1E005C0C1E003C0C1E001C0C0E08C2FE7
:10128000CF911F910F910895FC01892B61F0663079
:10129000710558F080818D3451F481E091819C3248
:1012A00039F080E0089580E0089580E0089580E0BE
:1012B0000895FC01892B61F06630710558F080813A
:1012C000823551F481E091819C3239F080E00895BB
:1012D00080E0089580E0089580E00895FC01892B66
:1012E00061F06530710558F080818A3551F481E0F4
:1012F00091819C3239F080E0089580E0089580E08B
:10130000089580E00895CF92DF92EF92FF920F93BD
:101310001F93CF93DF93CDB7DEB72897CDBFDEBF46
:10132000009709F457C06530710508F455C0FC01F9
:1013300020812A3509F052C021812C3209F050C099
:101340007B018C016C01F2E0CF0ED11CAB0142504D
:1013500051099E012F5F3F4FB6018CE20F94383741
:10136000882309F446C049815A814E5F5F4F498303
:101370005A8343305105B0F142509E012D5F3F4FDB
:1013800060E0C6010F94C035882399F18B819C8160
:10139000039750F589819A8101968E159F0530F546
:1013A0004E2D481B9E012B5F3F4F60E0800F911F29
:1013B0000F944B368823E9F06D817E818F8198856B
:1013C000623071058105910598F48B810E9400EED1
:1013D00081E00FC080E00DC080E00BC080E009C05C
:1013E00080E007C080E005C080E003C080E001C06D
:1013F00080E02896CDBFDEBFDF91CF911F910F9186
:10140000FF90EF90DF90CF9008952F923F924F92F0
:101410005F926F927F928F929F92AF92BF92CF9284
:10142000DF92EF92FF920F931F93CF93DF93CDB78D
:10143000DEB76397CDBFDEBF8C01F62E81E08D83D2
:101440000115110509F423C38093CE2089E10E9480
:1014500065D0672B682B692B09F025C30F943411D5
:10146000B82E811103C0F11020C385C387EF9CE320
:101470000E94D320B82E882309F47DC387EF9CE314
:101480000E94BF148F87F11004C08150823008F48D
:1014900000C32F85243031F487EF9CE30E942C2A6F
:1014A00033E03F870F94F7180F94E01887EF9CE321
:1014B0000E94992281110F944E2987EF9CE30E948C
:1014C000E62982E00E9465D0E62E8FEF8E0D8A30ED
:1014D00008F0E1C2AE014A5F5F4FBE016B5F7F4F14
:1014E0008E2D0E940E228E810E946BED8E81847063
:1014F0000E94DFED8D810F9452130F2EF9E4CF2E51
:10150000F3E4DF2EF02D8BE7D6018C938DE6119658
:101510008C9311978CE212968C93129787E713960F
:101520008C9320E044E050E0B601C8010F948B3169
:101530001F92EF928FEC99E29F938F93DF92CF925D
:101540000F94F366F60101900020E9F73197AF019F
:101550004954534420E0B601C8010F948B31E8E2AE
:10156000F4E587858F9386858F9385858F93848512
:101570008F930F2EF3EDAF2EF9E2BF2EF02DBF9219
:10158000AF92DF92CF920F94F366F60101900020A4
:10159000E9F73197AF014954534420E0B601C8013F
:1015A0000F948B318AE00E9465D09F938F937F9335
:1015B0006F93BF92AF92DF92CF920F94F366F601D2
:1015C00001900020E9F73197AF014954534420E0DE
:1015D000B601C8010F948B318BE00E9465D09F93B8
:1015E0008F937F936F93BF92AF92DF92CF920F94BE
:1015F000F366F60101900020E9F73197AF014954F5
:10160000534420E0B601C8010F948B310F2EF2E451
:10161000CF2EF4E5DF2EF02DCDBFDEBF412C512CB7
:10162000320145010F2EF9E4AF2EF3E4BF2EF02D69
:101630002BC0D6018C9111969C91119712962C91EA
:10164000129713963C91B4E0CB0ED11C3F932F938D
:101650009F938F939F928F92BF92AF920F94F36656
:10166000F50101900020E9F73197AF014954534447
:1016700020E0B501C8010F948B31EFEF4E1A5E0ADE
:101680006E0A7E0ACDBFDEBF0F942D2C90E0A0E045
:10169000B0E0481659066A067B0658F28DE780933B
:1016A000494321E041E050E069E473E4C8010F944C
:1016B0008B3165E087EF9CE30E94AC140F942C29DA
:1016C00087EF9CE30E94EB240E946D5B60E072E078
:1016D00080E090E00E945F5C1092EC401092ED4040
:1016E00086EC93E40E94EDB60E94005E8111FCCF6F
:1016F000B82EF11004C00E94BA1F8823E1F389E0DC
:101700000E9465D06F3171058105910508F59B0137
:10171000AC01012E1CE0220F331F441F551F1A95E8
:10172000D1F7102D2B873C874D875E87CA01B90101
:101730000F9499180F94F62981E00F94462C80E0BD
:1017400090E1A0E0B0E08F839887A987BA873FC077
:101750009B01AC01012E19E0220F331F441F551FBE
:101760001A95D1F7102D2B873C874D875E87CA01CC
:10177000B9010F9499180F94F6290F94762C80E0F4
:1017800092E0A0E0B0E08F839887A987BA871FC056
:10179000412C512C32019F2CCB84DC84ED84FE84BF
:1017A0000F94B32C8823E1F08D810F94202866ECF0
:1017B00073E40E9450B7A82E0F94A22C9FEF491AF1
:1017C000590A690A790AA1100BC0F92C0FC02B85A0
:1017D0003C854D855E85232B242B252BC9F606C021
:1017E0004C145D046E047F04D8F2F92C0F949D2CE8
:1017F00086EC93E40E94B4B7E82E0E94EC5C0F9450
:10180000E025EE2031F06F8587EF9CE30E94AC1459
:10181000B2C18FEE95E40E9402DE882351F0F110F0
:1018200008C06091EE4670E08FEE95E40E9414B817
:1018300009C0E9E4F3E41082118262E070E0CF01B4
:101840000E9414B860E072E080E090E00E94755B56
:101850000E94005E8111FCCF8B859C85AD85BE8585
:10186000892B8A2B8B2B09F4F3C0C12CD12C760148
:101870000F2EF9E42F2EF3E43F2EF02D4F805884E5
:1018800069847A8491E0491A5108610871080E94BC
:1018900003B88093EC409093ED40AE014F5F5F4FF3
:1018A000BC018D810E94EA14882309F463C1C70139
:1018B000B6012F81388549855A850F9488644B017C
:1018C0005C01672B682B692BA1F5C701B6012F813D
:1018D000388549855A850F948864288B398B4A8BC3
:1018E0005B8B89E00E9465D0AB89AF93BA89BF93C7
:1018F000E989EF93F889FF939F938F937F936F9379
:1019000028ED39E23F932F933F922F920F94F36685
:10191000F10101900020E9F73197AF014954534498
:1019200020E0B101C8010F948B311092CE20CDBFC1
:10193000DEBF2F81388549855A85211582E0380719
:101940004105510509F4BAC0211530414105510541
:1019500009F4DDC0D701C60187709927AA27BB27E4
:10196000892B8A2B8B2B09F043C08C818F938B8121
:101970008F938A818F9389818F93A1E5BBE2BF9377
:10198000AF933F922F920F94F366F10101900020E4
:10199000E9F73197AF014954534420E0B101C80140
:1019A0000F948B31C701B6012F81388549855A853F
:1019B0000F9488642F5F3F4F4F4F5F4F6F81788543
:1019C00089859A850F944664CDBFDEBFA701960135
:1019D000285F3F4F4F4F5F4F62177307840795078C
:1019E00019F41092CE20C0C031E03093CE20BCC09C
:1019F0001092CE2084149504A604B70479F4EDE780
:101A0000D101EC9321E041E050E0B101C8010F9415
:101A10008B310FC0ECE2D101EC9304C08091CE2059
:101A2000882339F020E041E050E0B101C8010F9473
:101A30008B31FFEFCF1ADF0AEF0AFF0A2B853C85B7
:101A40004D855E85C216D306E406F50609F01FCF64
:101A50000E94405C0F94E0250F94B83A83EB90E429
:101A60000F94985C6F8587EF9CE30E94AC140F94F1
:101A70006E1987EF9CE30E94992281110F944E29E1
:101A800087EF9CE30E94E629BB24B39474C0B12C79
:101A900072C0B12C70C0B12C6EC087EF9CE30E9465
:101AA000BF148F87F6CCFF24F39487EF9CE30E944A
:101AB000D320B82E882309F45EC0EFCF8C818F939A
:101AC0008B818F938A818F9389818F9341E55BE22C
:101AD0005F934F933F922F920F94F366F101019021
:101AE0000020E9F73197AF014954534420E0B10198
:101AF000C8010F948B3191E09093CE20CDBFDEBF13
:101B0000481459046A047B0409F084CF78CF8C818F
:101B10008F938B818F938A818F9389818F93E1E556
:101B2000FBE2FF93EF933F922F920F94F366F10144
:101B300001900020E9F73197AF014954534420E068
:101B4000B101C8010F948B3131E03093CE20CDBF6D
:101B5000DEBF481459046A047B0409F05BCF4FCF01
:101B6000ECE2D101EC935ACF84149504A604B70497
:101B7000B9F745CFB82E8B2D6396CDBFDEBFDF9171
:101B8000CF911F910F91FF90EF90DF90CF90BF907A
:101B9000AF909F908F907F906F905F904F903F900D
:101BA0002F900895CF92DF92EF92FF921F93CF93E1
:101BB000DF936115710509F474C04630510508F4CE
:101BC00072C0DB01EC91ED3409F06FC01196EC911D
:101BD000EC3209F06CC02115310509F46AC0009798
:101BE00009F469C069017A01EB012D81203341F4C8
:101BF00040E060E00ADC11E0811160C010E05EC0EE
:101C0000233541F5C6010E94E020182F882309F4EE
